:100000000C94540A0C94750A0C94750A0C94CD0F38
:100010000C9407100C94750A0C94750A0C94750ACC
:100020000C94750A0C94750A0C94750A0C94750A54
:100030000C94750A0C94750A0C94750A0C94391377
:100040000C94750A0C94750A0C94750A0C94750A34
:100050000C94750A0C94C96D0C94750A0C94750A6D
:100060000C94750A0C94446E0C94750A0C94750AE1
:100070000C94750A0C94750A0C94750A0C94750A04
:100080000C9436830C94750A0C94750A0C94750ABA
:100090000C94736E0C94750A0C94750A0C94750A82
:1000A0000C94750A0C94750A0C94750A0C94750AD4
:1000B0000C94750A0C94750A0C94750A0C94750AC4
:1000C0000C94750A0C94750A0C94750A0C94750AB4
:1000D0000C94750A0C94750A0C94750A0C94750AA4
:1000E0000C94750A0C940F750C9405750C94197585
:1000F0000C94A3740C9423750C94FB740C94EF74FF
:100100000C94E3740C94750A0C94750A0C94750A9B
:100110000C94750A0C94750A0C94750A0C94750A63
:100120000C94750A0C94750A0C94750A0C94750A53
:100130000C94750A5B897A89E989DA8AFA8A1A8BBA
:10014000228BCF8A084AD73B3BCE016E84BCBFFDD1
:10015000C12F3D6C74319ABD56833DDA3D00C77F97
:1001600011BED9E4BB4C3E916BAAAABE0000008030
:100170003F07634236B79BD8A71A39685618AEBAFC
:10018000AB558C1D3CB7CC5763BD6DEDFD753EF690
:10019000177231BF000000803F08000000BE9224AB
:1001A00049123EABAAAA2ABECDCCCC4C3E000000E0
:1001B00080BEABAAAAAA3E00000000BF00000080DB
:1001C0003F0000000000084178D3BB4387D1133DB6
:1001D000190E3CC3BD4282AD2B3E68EC8276BED97F
:1001E0008FE1A93E4C80EFFFBE01C4FF7F3F0000BE
:1001F000000000000C94674F0C94586F0C94E3813E
:100200000C94367E0C947A890C945B890C94CF7D87
:100210000C94DE810C94437E0C9482820C949F7526
:100220000C949E710C9461910C943B7E0C94007321
:100230000C9408150C94EC700C9411830C949E8D06
:100240000C949D820C94997C0C9425700C94407EA7
:100250000C942C7E0C941A8B0C94E9890C94228BB0
:100260000C945C7B0C94E3700C94BF7B0C94D46E68
:100270000C94FA8A0C94E6810C94C54F0C94FB7F85
:100280000C94BE4E0C942C6F0C94AD720C94EA7BC3
:100290000C9447720C94305F0C945B0E0C94DA8AC9
:1002A0000C94D2100C942A740C94DB7D0C9408836B
:1002B0000C94317E0C94AC760C940F7C0C94827B65
:1002C0000C94CF8A0C94F6150C941A700C94337B12
:1002D0000C94411D0C94828C0C94FD380C94567C2B
:1002E0000C94CD8B0C94410E6E616E00696E6600AD
:1002F00000407A10F35A00A0724E18090010A5D4DD
:10030000E80000E87648170000E40B54020000CA39
:100310009A3B000000E1F50500008096980000007F
:1003200040420F000000A0860100000010270000DE
:100330000000E803000000006400000000000A0064
:10034000000000000100000000002C76D888DC6767
:100350004F0823DFC1DFAE59E1B1B796E5E3E453BF
:10036000C63AE651997696E8E6C28426EB898C9BDC
:1003700062ED407C6FFCEFBC9C9F40F2BAA56FA57C
:10038000F490055A2AF75C936B6CF9676DC11BFCFE
:10039000E0E40D47FEF520E6B500D0ED902E030019
:1003A000943577050080841E080000204E0A000066
:1003B00000C80C333333330F986E12831141EF8D25
:1003C0002114893BE65516CFFEE6DB18D1844B3865
:1003D0001BF77C1D901DA4BBE424203284725E2296
:1003E0008100C9F124ECA1E53D274E414E494E491B
:1003F0005459494E46CDCCCC3D0AD7233C17B7D1F2
:100400003877CC2B329595E6241FB14F0A00002097
:10041000410000C84200401C4620BCBE4CCA1B0E16
:100420005AAEC59D74256300496E76616C6964207F
:1004300069326320737065656420696E204545509C
:10044000524F4D2E2053657474696E6720313020F1
:100450006B6269742F730025730A00776474206ED1
:100460006F7420656E61626C65640A005854414C7B
:100470005F5452494D3D25640025730A0025730AD7
:10048000005465737420362025730A005465737414
:1004900020352025730A0054657374203420257399
:1004A0000A005465737420332025730A0054657361
:1004B0007420322025730A0054657374203120257E
:1004C000730A006368616E3D25640A007478707772
:1004D000723D25640A003530306B0A003235306BCE
:1004E0000A003131356B0A0035366B0A0033386B40
:1004F0000A0025730A00765F6C6F773D252D332E39
:1005000032660A0025730A0073656E743D252D75E9
:10051000206475703D252D752069676E6F72656466
:100520003D252D752074746C5F7A65726F3D252DA5
:10053000750A0025372E33662025372E33660025B1
:10054000352E326620004572726F72203020566F51
:100550006C74004E6F7420737570706F7274656484
:100560000A004572726F72203020566F6C7400451D
:1005700072726F72203020566F6C740062756C6BF3
:100580005F64656C61793D252D750062756C6B3D0E
:10059000252D750056616C7565206E6F7420616C39
:1005A0006C6F7765640062756C6B3A206D61783DA5
:1005B00025752073746172743D25752C20656E64F9
:1005C0003D25752C20696E5F7573653D25750A00A4
:1005D0007062323D25730A007062313D25730A0056
:1005E000256C7500416C6C6F776564207370656570
:1005F0006420312F31302F3130302F343030206BA8
:100600006269742F730025630074746C3D252D643A
:10061000200074746C3D252D6420004E6577207495
:10062000746C3D252D6420002563004D5335363113
:100630003120503D252D372E326620252D372E3284
:10064000666D0A00424D5030383520256C642043D9
:100650002000424D5030383520256C6420506120F8
:1006600020252D372E32666D00256300545F4845E6
:1006700041545F4944583D252D352E3266200054A3
:100680005F4445573D252D352E3266200041483DBB
:10069000252D352E32662000545F53485432583D84
:1006A000252D352E3266200052485F53485432586B
:1006B0003D252D352E32662000545F52483D252DB4
:1006C000342E3166200052483D252D342E316620CF
:1006D0000025630025630025630025630025630072
:1006E0007265706F72745F616C6C3D007265706FE3
:1006F00072743D00256300256300256300256300B7
:10070000204F534343414C3D2564200020467573E0
:10071000653A2065653D253032782068663D253094
:100720003278206C663D25303278206C623D253071
:100730003278004D43553D2530366C7800256300F6
:1007400074785F6C656E3D252D6C752C765F6C6FD3
:10075000773D252D6C752C73687432783D252D6C92
:10076000752C62756C6B3D252D6C75002563004FF3
:100770004B0A0025630025630025630025630025DF
:100780006300256300256300256300646562756767
:100790005F616C6C3D0064656275673D0064656215
:1007A00075673D0025730A00646565700A006E6F09
:1007B0006E650A00707772733D007764743D25732F
:1007C0000A007062323D25730A007062313D257364
:1007D0000A00696E74725F7365635F70313D252D29
:1007E000372E33660A00696E74725F70313D252DB5
:1007F0006C640A00696E74725F7365635F70303D8C
:10080000252D372E33660A00696E74725F70303D95
:10081000252D6C640A00765F6D63753D252D352EA0
:1008200032660A00745F6D63753D252D352E326684
:100830000A00707077723D25730A006465627567FF
:100840003D0072636D643D25730A0025730A0061E3
:1008500075746F0A006C6F675F6D6F64653D00753E
:1008600073625F7077723D25730A0072656C6179FF
:100870003D25730A0074746C3D252D640A005249AD
:100880004D455F616464723D252D642E252D640AFB
:10089000006E65696768626F725F7461626C655F44
:1008A00073697A653D25640A00765F6C6F773D2534
:1008B0002D332E32660A00747870773D25640A0065
:1008C0006368616E3D25640A0069643D00693263B6
:1008D0005F6275733D006932635F73706565643D87
:1008E000252D6C750A007478743D25730A005379C0
:1008F0007374656D2053756D6D6172790A002530D2
:10090000366C780041744D65676132353652465217
:10091000320041744D6567613132385246523200BF
:1009200041744D6567613634524652320041744D10
:1009300065676131323852464131004D43553D00C3
:100940006D61736B3D002C00696E74657276616C2D
:100950003D252D750023252D642C00705F626D658B
:100960003238300072685F626D6532383000745F13
:10097000626D65323830007062320070623100742E
:100980005F686561745F69647800745F64657700AF
:10099000616800705F6D73353631310072685F7366
:1009A0006874327800745F73687432780070610024
:1009B000700061643400616433006164320061641A
:1009C0003100613300613200613100765F696E0091
:1009D00072680065727200757074696D65007031BF
:1009E0005F6C73740070315F740070310070305F41
:1009F0006C73740070305F7400703000765F6D63EC
:100A00007500745F6D637500743100740069640073
:100A100065363400747874002D002B006175746F96
:100A2000006E6F6E650062756C6B00706F7765723B
:100A30005F736176655F6C656472790072656C6185
:100A4000795F6C65647900636F6D706173730061C9
:100A50006363656C007072657300705F707772001D
:100A60006165730070315F6C6564790070305F6C34
:100A7000656472006576656E74006C6564006F77FE
:100A800000706B740074785F6C6564790072785FD5
:100A90006C656472006F706572006E6F6E65002524
:100AA00030327800765F6164343D252D382E36660D
:100AB000002000765F6164333D252D382E366600B8
:100AC0002000765F6164323D252D382E3666002089
:100AD00000765F6164313D252D382E36660020009A
:100AE000765F6C696768743D252D382E3666002068
:100AF00000765F61323D252D372E3366002000766B
:100B00005F61313D252D372E3366002000765F6909
:100B10006E3D252D352E326600204E657665722D90
:100B20007573656420737461636B203E20256420B7
:100B300062797465730A00757074696D653D252D61
:100B4000642D646179732D253032643A2530326426
:100B50003A253032642D686F7572730A00746573BC
:100B600074205B6F66667C317C327C337C347C35F0
:100B70005D20202020202020202D207465737420EB
:100B80006D6F6465730A0D007478205B706B742060
:100B90007061796C6F61645D20202020202020200E
:100BA000202020202D2073656E6420726164696F9F
:100BB00020706B74206B6579626F6172640A0D003E
:100BC000776474205B6F6E7C6F66667C746573748B
:100BD0005D20202020202020202020202D20776133
:100BE000746368646F670A0D00765F6C6F77205BD3
:100BF000765F6C6F775D2020202020202020202031
:100C000020202020202D206C6F7765737420726562
:100C1000706F727420766F6C746167650A0D007571
:100C200070677220202020202020202020202020DB
:100C300020202020202020202020202D20726562CE
:100C40006F6F742076696120626F6F746C6F61647E
:100C500065720A0D0075617274205B33386B7C35E8
:100C6000366B7C3131356B7C3235306B7C353030D6
:100C70006B5D202D20736574207465726D2F756116
:100C800072742073706565640A0D00626F6F742062
:100C90002020202020202020202020202020202054
:100CA000202020202020202D207265626F6F740A82
:100CB0000D0070777273205B646565707C6E6F6E7B
:100CC000655D2020202020202020202020202D2095
:100CD0006D637520736C656570206D6F64650A0DBA
:100CE000007265737420656570726F6D202020201E
:100CF000202020202020202020202020202D207295
:100D00006573746F726520656570726F6D0A0D0092
:100D100070707772205B6F6E7C6F66665D2020203E
:100D20002020202020202020202020202D20707214
:100D30006F6772616D6D61626C65207077720A0D0C
:100D40000070623220205B6F6E7C6F66665D2020D3
:100D5000202020202020202020202020202D207036
:100D6000726F6772616D6D61626C652070696E2073
:100D700062320A0D0070623120205B6F6E7C6F66FC
:100D8000665D2020202020202020202020202020E0
:100D9000202D2062756C6B204750494F2070696E82
:100DA0000A0D00747874205B737472696E675D203D
:100DB0002020202020202020202020202020202D26
:100DC00020536574207265706F7274207465787436
:100DD00020737472696E670A0D0074787077205BF7
:100DE00031352D305D202020202020202020202083
:100DF0002020202020202D205458205077722E2093
:100E000048696768657374203020283364426D290F
:100E10000A0D0074746C205B302D31355D2020206C
:100E20002020202020202020202020202020202DB5
:100E30002074696D652D746F2D6C69766520666F01
:100E400072207061636B6574730A0D0073732020E8
:100E50002020202020202020202020202020202092
:100E600020202020202020202D2073797374656D90
:100E70002073756D6D6172790A0D007273202020E8
:100E80002020202020202020202020202020202062
:100E9000202020202020202D20726164696F207383
:100EA000746174730A0D007269205B236E5D205BB0
:100EB000696E745D2020202020202020202020200A
:100EC0002020202D207265706F727420696E746509
:100ED0007276616C0A0D0072636D64205B6F6E7CCC
:100EE0006F66665D202020202020202020202020EA
:100EF0002020202D20616C6C6F7720636D6420664C
:100F0000726F6D206E65746F726B0A0D00726520D2
:100F10005B236E5D205B2B7C2D5D205B6D61736BB5
:100F20007C6175746F2C6D61736B5D202D206D6F0E
:100F30007465207265706F7274207365742F6D6FA5
:100F4000646966790A0D006F772020202020202018
:100F50002020202020202020202020202020202091
:100F60002020202D206F6E652D77697265207365B6
:100F70006E736F72730A0D006C6F67205B6175741E
:100F80006F7C6F6E7C6F66665D20202020202020A5
:100F9000202020202D206D6F7465732064617461A2
:100FA000206F6E205553420A0D006E65205B666C03
:100FB0007573685D20202020202020202020202004
:100FC0002020202020202D206E65696768626F72C6
:100FD000207461626C650A0D006572722020202009
:100FE0002020202020202020202020202020202001
:100FF00020202020202D206572726F722073746172
:1010000074730A0D006D637520202020202020209D
:1010100020202020202020202020202020202020D0
:10102000202D206D637520696E666F0A0D00693290
:1010300063205B70726F62657C73706565642023EA
:101040006E5D20202020202020202D20693263206A
:1010500070726F6265206275737C7365742062754F
:10106000732073706565640A0D006964205B7265A6
:101070007365745D20202020202020202020202047
:101080002020202020202D2069642068616E646C5F
:10109000696E670A0D0068756D20202020202020D1
:1010A0002020202020202020202020202020202040
:1010B00020202D2068756D69646974792073656ED0
:1010C000736F720A0D0072656C6179205B6F6E7CC4
:1010D0006F66667C73746174735D2020202020200D
:1010E00020202D2072656C6179206E6574776F7297
:1010F0006B207265706F7274730A0D006465205BFB
:101100006D61736B5D202020202020202020202076
:1011100020202020202020202D2064656275670A71
:101120000D006368616E205B31312D32365D202009
:1011300020202020202020202020202020202D20A2
:101140006368616E2031312D32362028322E3430E2
:10115000352D32343830204D687A290A0D0063610C
:101160006C69205B5B765F696E7C61317C61325DAE
:1011700020766F6C747C72657365747C6E6F6E65BF
:101180005D202D2063616C6962726174650A0D00D7
:1011900062756C6B205B5B73686F777C666C7573D4
:1011A000685D205B73657420746872736820646581
:1011B0006C61795D5D20202D2062756C6B696E67B6
:1011C000207061636B657473200A0D006164632095
:1011D000202020202020202020202020202020200F
:1011E00020202020202020202D2073686F7720765B
:1011F0005F696E2C2061312C20613220766F6C7417
:10120000616765730A0D00752020202020202020B2
:1012100020202020202020202020202020202020CE
:101220002020202D20757074696D650A0D007620D0
:1012300020202020202020202020202020202020AE
:10124000202020202020202020202D207665727351
:10125000696F6E0A0D0068202020202020202020A9
:10126000202020202020202020202020202020207E
:1012700020202D2068656C700A0D00256300756EB6
:101280006B6E6F776E20636D640A00484D4335388E
:101290003833002573002573000A002025730020D1
:1012A00025362E32662000253032780074656D7048
:1012B0005F65787465726E3D252D362E326600208E
:1012C0002573002025362E3266204F6E2D426F6129
:1012D000726400253032780074656D705F626F61F2
:1012E00072643D252D362E32660042756C6B20727D
:1012F000656D3A2073746172743D25752C20656E9E
:10130000643D25752C20696E5F7573653D25750AF2
:101310000042756C6B206164643A2073746172746E
:101320003D25752C20656E643D25752C20696E5F0A
:101330007573653D25750A0042756C6B2074687283
:101340006573683A2074696D65723D25750A0050B1
:101350003A20256C642050612020252D372E3266DE
:10136000206D0A004932433A20004F6E6C696E6569
:101370000A00526F7574696E6720456E61626C6514
:10138000640A0052504C20456E61626C65640A002C
:1013900025732025732C206368616E6E656C202593
:1013A00075202C20636865636B207261746520254D
:1013B0007520487A20747820706F776572202575C3
:1013C0000A000A2A2A2A2A2A2A2A426F6F74696E78
:1013D000672025732A2A2A2A2A2A2A0A00726E6777
:1013E000206973737565732025640A004545505262
:1013F0004F4D20697320636F72727570742C207268
:101400006577726974696E672077697468206465AE
:101410006661756C74732E0A006C6F63616C686F23
:1014200073740041544D454741323536726672320D
:1014300000020000FFFE000001452025642E256407
:1014400020636C6F636B20256C752063707520259D
:101450006C75206C706D20256C752069727120256B
:101460006C7520676C656420256C7520796C6564EB
:1014700020256C7520726C656420256C752074784D
:1014800020256C75206C697374656E20256C752041
:1014900073656E736F727320256C75207365726946
:1014A000616C20256C750A0011241FBECFEFD1E8B6
:1014B000DEBFCDBF00E00CBF1BE0A0E0B2E0E2EB7E
:1014C000FCE301E00BBF02C007900D92A432B1070C
:1014D000D9F72BE3A4E2BBE001C01D92A930B2070B
:1014E000E1F70E94DA6C0C94579E0C9400002F9246
:1014F0003F924F925F926F927F928F929F92AF92A4
:10150000BF92CF92DF92EF92FF920F931F93CF93F0
:10151000DF93CDB7DEB760970FB6F894DEBF0FBE8E
:10152000CDBF7C011B016A01FC01178216828381F9
:1015300081FF44C39E012F5F3F4F3901F701938123
:10154000F10193FD859193FF81911F01882309F497
:1015500031C3853239F493FD859193FF81911F0149
:10156000853239F4B70190E00E94339B5601650142
:10157000E5CF10E0512C912CFFE1F915D8F08B321A
:1015800079F038F4803279F08332A1F4F92DF061EA
:101590002EC08D3261F0803369F4292D21602DC079
:1015A000392D3260932E892D8460982E2AC0E92D22
:1015B000E86015C097FC2DC020ED280F2A3088F474
:1015C00096FE06C03AE0139F200D1124122F19C079
:1015D0008AE0589E200D1124522EE92DE0629E2EA5
:1015E00010C08E3231F496FCE5C2F92DF0649F2EC6
:1015F00008C08C3621F4292D2068922E02C088362E
:1016000041F4F10193FD859193FF81911F018111B7
:10161000B3CF9BEB980F933020F4992D9061805EAF
:1016200007C09BE9980F933008F066C1992D9F7E03
:1016300096FF16E09F73992E853619F49064992EC3
:1016400008C0863621F4392F3068932E02C011115C
:10165000115097FE07C01C3350F444244394410EAC
:1016600027E00BC0183038F027E017E005C027E06E
:101670009CE3492E02C0212F412C560184E0A80E84
:10168000B11CF6016081718182819381042DA301D7
:101690000E94AA996C01F981FC87F0FF02C0F3FF58
:1016A00006C091FC06C092FE06C000E205C00DE235
:1016B00003C00BE201C000E08C858C7019F00111B1
:1016C0005AC29BC297FE10C04C0CFC85F4FF04C0AC
:1016D0008A81813309F44A94141474F528E024159E
:1016E00078F588E0482E2CC096FC2AC0812F90E027
:1016F0008C159D059CF03CEFC3163FEFD30674F0AC
:10170000892D8068982E0AC0E2E0F0E0EC0FFD1F02
:10171000E10FF11D8081803319F411501111F4CFC4
:1017200097FE0EC044244394410E812F90E0C816CA
:10173000D9062CF41C1904C04424439401C010E0C1
:1017400097FE06C01C141D0434F4C601019605C0A2
:1017500085E090E002C081E090E001110196112344
:1017600031F0212F30E02F5F3F4F820F931F252D47
:1017700030E08217930714F4581A01C0512C892DB8
:10178000897049F4552039F0B70180E290E00E9459
:10179000339B5A94F7CF002329F0B701802F90E0B4
:1017A0000E94339B93FC09C0552039F0B70180E3B8
:1017B00090E00E94339B5A94F7CF97FE4CC04601AD
:1017C000D7FE02C0812C912CC60188199909F3011A
:1017D000E80FF91FFE87ED87960124193109388B30
:1017E0002F87012F10E01195019511093FEF831606
:1017F000930629F4B7018EE290E00E94339BC8144F
:10180000D9044CF08F8598898815990524F4ED85C5
:10181000FE85818101C080E3F1E08F1A91082D855A
:101820003E852F5F3F4F3E872D87801691062CF017
:10183000B70190E00E94339BD9CFC814D90441F47A
:101840009A81963320F4953319F43C8534FF81E373
:10185000B70190E04EC08A81813319F09C859F7E4C
:101860009C87B70190E00E94339B111105C094FC46
:1018700018C085E690E017C0B7018EE290E00E94A4
:10188000339B1E5F82E001E0080FF301E80FF11DBA
:101890008081B70190E00E94339B802F0113F3CF2A
:1018A000E6CF85E490E0B7010E94339BD7FC06C0E9
:1018B000C114D10441F4EC85E4FF05C0D194C19476
:1018C000D1088DE201C08BE2B70190E00E94339B0A
:1018D00080E32AE0C216D1042CF08F5FFAE0CF1A21
:1018E000D108F7CFB70190E00E94339BB701C60142
:1018F000C0960E94339B54C1833631F0833779F010
:10190000833509F056C020C0560132E0A30EB11C49
:10191000F6018081898301E010E0630112C0560165
:10192000F2E0AF0EB11CF601C080D18096FE03C07C
:10193000612F70E002C06FEF7FEFC6010E94DF9A57
:101940008C01F92DFF7714C0560122E0A20EB11CC4
:10195000F601C080D18096FE03C0612F70E002C006
:101960006FEF7FEFC6010E94949A8C01F92DF06809
:101970009F2EF3FD1AC0852D90E008171907A8F4D3
:10198000B70180E290E00E94339B5A94F4CFF601B5
:1019900097FC859197FE81916F01B70190E00E94BD
:1019A000339B51105A94015011090115110579F713
:1019B000F7C0843611F0893661F5560197FE09C0EB
:1019C00024E0A20EB11CF6016081718182819381B5
:1019D0000AC0F2E0AF0EB11CF60160817181072EE2
:1019E000000C880B990BF92DFF769F2E97FF09C0ED
:1019F00090958095709561957F4F8F4F9F4FF068C0
:101A00009F2E2AE030E0A3010E94479CC82EC618F2
:101A10003FC0092D853721F40F7E2AE030E01DC03C
:101A2000097F8F3691F018F4883559F0C3C080379C
:101A300019F0883711F0BEC0006104FF09C00460CE
:101A400007C094FE08C0066006C028E030E005C06C
:101A500020E130E002C020E132E0560107FF09C07A
:101A600084E0A80EB11CF6016081718182819381AE
:101A700008C0F2E0AF0EB11CF6016081718180E018
:101A800090E0A3010E94479CC82EC6180F77902EA5
:101A900096FE0BC0092D0E7FC11650F494FE0AC0AD
:101AA00092FC08C0092D0E7E05C0DC2C092D03C058
:101AB000DC2C01C0D12E04FF0DC0FE01EC0DF11D88
:101AC0008081803311F4097E09C002FF06C0D394DF
:101AD000D39404C0802F867809F0D39403FD11C0FD
:101AE00000FF06C01C2DD51480F4150D1D190DC066
:101AF000D51458F4B70180E290E00E94339BD39450
:101B0000F7CFD51410F45D1801C0512C04FF10C09C
:101B1000B70180E390E00E94339B02FF17C001FDF4
:101B200003C088E790E002C088E590E0B7010CC0F0
:101B3000802F867859F001FF02C08BE201C080E25D
:101B400007FD8DE2B70190E00E94339BC11638F487
:101B5000B70180E390E00E94339B1150F7CFCA9405
:101B6000F301EC0DF11D8081B70190E00E94339BE1
:101B7000C110F5CF15C0F4E0F51560F584E0581AF2
:101B800093FE1FC0011127C02C8523FF2AC008EE39
:101B900012E0392D3071932EF8018491811124C007
:101BA000552009F4E4CCB70180E290E00E94339B19
:101BB0005A94F6CFF7018681978126C08FEF9FEF69
:101BC00023C0B70180E290E00E94339B5A945110E9
:101BD000F8CFD8CF512CB701802F90E00E94339BD3
:101BE000D3CF0CEE12E0D5CF91108052B70190E028
:101BF0000E94339B0F5F1F4FCFCF23E0251510F4BA
:101C000083E0BDCF512CC0CF60960FB6F894DEBFF5
:101C10000FBECDBFDF91CF911F910F91FF90EF903D
:101C2000DF90CF90BF90AF909F908F907F906F90FC
:101C30005F904F903F902F9008958115910511F07E
:101C40000197F1F7089584EB97E09F938F930E949B
:101C5000839B8091660290916702A0916802B09187
:101C600069020F900F9093FF03C08EEA97E002C0C5
:101C700088EA97E09F938F930E94839B0F900F9029
:101C80000895E091F81DEF73F0E0E75BF14E80837B
:101C90008091F81D8F5F8093F81D8091A536886034
:101CA0008093A5364CE452E061E1CA010E949E781F
:101CB00080E090E00895CF93DF93EC0180917D1454
:101CC00090917E14A0917F14B091801486FF1DC066
:101CD0008E811F928F938D811F928F938C811F9283
:101CE0008F938B811F928F938A811F928F9389EE9E
:101CF00092E09F938F930E946F9B8DB79EB70C9637
:101D00000FB6F8949EBF0FBE8DBFBE018FE69BE05D
:101D10000E949579BE0188E092E0DF91CF910C940A
:101D2000F07A52985A981DBAE9E6F0E08081806214
:101D30008083EA9A53985B98EB9A808180688083CD
:101D4000E8E6F0E08081816080830895EEEAFEE1BC
:101D50001182128210820895CF92DF92EF92FF9249
:101D60000F931F93CF93DF93EC019B018091AE1EE5
:101D7000843108F0BBC08091B01E64E10E944C9099
:101D80009093B01EC090CB31D090CC31E090CD314B
:101D9000F090CE31092F10E08DE8989FD0011124EA
:101DA000A255B14E1396CD92DD92ED92FC9216970C
:101DB0004115510559F0FA018081FD01EA57FF4FA5
:101DC0008083FA018181A957BF4F8C932097A9F096
:101DD00089819DE8909FF001919FF00D1124E255BB
:101DE000F14EDF01A657BF4F8C93E557FF4F888117
:101DF0008F70808388818F70808321153105E1F198
:101E0000D90116964C9116975DE8509FC001519FDD
:101E1000900D11248255914EFC01E757FF4F4083EE
:101E200015964C9115973197408334961B964D919A
:101E30005D916D917C911E97452F562F672F7727C7
:101E4000518340837C01BEE8EB0EF11CF901238530
:101E5000348545855685A4E6B0E00E94E790672F5B
:101E6000782F892F992724E630E040E050E00E9447
:101E70008090D7016D937C938DE8809FD001819FE6
:101E8000B00D1124AB54B14EFE0132968FE7019094
:101E90000D928A95E1F78091B01E8F5F8093B01EFE
:101EA0009091AE1E9F5F9093AE1E40917D14509115
:101EB0007E1460917F147091801460FF2DC01F927A
:101EC0009F931F928F938091AF1E1F928F9381E1FA
:101ED00093E19F938F930E94839BEDB7FEB7389653
:101EE0000FB6F894FEBF0FBEEDBF16C08091DB3178
:101EF0009091DC31A091DD31B091DE310196A11DD0
:101F0000B11D8093DB319093DC31A093DD31B09330
:101F1000DE3180E090E002C081E090E0DF91CF917F
:101F20001F910F91FF90EF90DF90CF900895209137
:101F3000AE1E222361F18091AF1E8F5F215020934E
:101F4000AE1E64E10E944C909093AF1E40917D14B0
:101F500050917E1460917F147091801460FF1AC0BC
:101F60001F922F938091B01E1F928F931F929F9369
:101F70008AEE92E19F938F930E94839B8DB79EB7C9
:101F800008960FB6F8949EBF0FBE8DBF03C080E0C9
:101F900090E0089581E090E008951F920F920FB6AF
:101FA0000F9211248F939F93AF93BF9380916800FA
:101FB00080FF24C08091743690917536A09176365A
:101FC000B09177360196A11DB11D80937436909320
:101FD0007536A0937636B093773680917D149091C4
:101FE0007E14A0917F14B091801487FF07C074986D
:101FF00082E090E09093920280939102BF91AF9122
:102000009F918F910F900FBE0F901F9018951F9268
:102010000F920FB60F9211248F939F93AF93BF939C
:102020008091680080FF24C0809178369091793645
:10203000A0917A36B0917B360196A11DB11D809397
:10204000783690937936A0937A36B0937B36809128
:102050007D1490917E14A0917F14B091801490FF14
:1020600007C0739882E090E090939202809391026F
:10207000BF91AF919F918F910F900FBE0F901F90C6
:10208000189580937C0080917B00877F80937B00F4
:1020900080917C00806C80937C0085E080937A0046
:1020A00080917A00806880937A0080917B0087FF1E
:1020B000FCCF80917B0085FFFCCF80917A0080640B
:1020C00080937A0080917A0086FDFCCF109279008F
:1020D0001092780084E090E060E070E020917A0057
:1020E000206420937A0020917A0026FDFCCF209175
:1020F000780030917900620F731F019779F7109281
:102100007C0080917A008F7780937A00769567952E
:102110007695679580E090E00E942A94089580E08B
:102120000E9441102091890230918A0240918B02D5
:1021300050918C020E94249621EE3AE744E95EE336
:102140000E94959208950F931F93CF93DF930FE111
:1021500010E0CBE5DEE00093510182E991E00E94BE
:102160001D0E8091510185FD0DC00031110521F03A
:102170002CF0CB54D10903C0C4ECD9E0E297015054
:102180001109E9CFBE0180E090E00E942A9420E08E
:1021900030E04AE754E40E947893DF91CF911F9199
:1021A0000F910895CF93DF93EC0188819981009777
:1021B00099F08B37924121F01982188283E011C087
:1021C000623171F40E94A3106093C7317093C831DB
:1021D0008093C9319093CA318BE792E199838883C8
:1021E00081E0DF91CF91089580917B00886080939A
:1021F0007B0089EC80937C0085E080937A0080915D
:102200007A00806880937A0080917B0087FFFCCF02
:1022100080917B0085FFFCCF80917A008064809361
:102220007A0080917A0086FDFCCF80917A008064EC
:1022300080937A0080917A0086FDFCCF60917800CF
:102240007091790080917A008F7780937A0080E096
:1022500090E00E942A9427ED33EA40E95FE30E9470
:10226000249626E636E648E853E40E9494920895C0
:10227000AF92BF92CF92DF92EF92FF921F93CF93D4
:10228000DF93CDB7DEB729970FB6F894DEBF0FBE48
:10229000CDBF5C01109277148FEF898781E0E82E23
:1022A0008EE1F82E10E06E0189E0C80ED11C898500
:1022B0008823D1F11830D1F1BE016F5F7F4FC60185
:1022C0000E94EE6289858F3F11F08E3F19F4809352
:1022D00077142AC0CE010196A114B10479F40E94AA
:1022E000076380939636FE013196AEE8B6E381919E
:1022F0008D93EC15FD05D9F781E019C00E940763A5
:10230000F7018087FE01319680E090E02191D701AE
:10231000A80FB91F2C93019688309105B9F71F5F5C
:10232000F9E0EF0EF11CC3CF812F01C088E02996A0
:102330000FB6F894DEBF0FBECDBFDF91CF911F91D6
:10234000FF90EF90DF90CF90BF90AF9008952F92C5
:102350003F924F925F926F927F928F929F92AF9235
:10236000BF92CF92DF92EF92FF920F931F93CF9382
:10237000DF93EC015B01009711F427E003C00197A4
:1023800049F426E04AE250E06BE270E089E290E036
:102390000E94CE61CE010E9438119E0128583B4E0A
:1023A0006901F9018083CD2B69F0C1E0DEE1E12C08
:1023B000F12C9BE9292E92E1392E29E9822E22E186
:1023C000922EC2C08EE896E30E949463BC01990FDE
:1023D000880B990B0E942C946B017C01AB2801F1B6
:1023E00020E030E048EC52E40E9478939F938F9372
:1023F0007F936F9388ED92E19F938F930E94839BCD
:1024000089E992E19F938F930E94839B2DB73EB7FA
:10241000285F3F4F0FB6F8943EBF0FBE2DBFCBC015
:10242000CEE8D6E386E9A82E86E3B82E03ED12E1C6
:1024300089911F928F931F930F930E94839B0F90FC
:102440000F900F900F90AC16BD0691F720E030E092
:1024500048EC52E4C701B6010E9478939F938F9392
:102460007F936F9383EC92E19F938F930E94839B62
:102470000F900F900F900F900F900F9080919636C5
:10248000811103C08AE993E002C088E193E09F9341
:102490008F938FEB92E19F938F930E94839B89E9A7
:1024A00092E19F938F930E94839B0F900F900F90C8
:1024B0000F900F900F907FC000E010E0FE01E00F42
:1024C000F11F80811F928F93E7EAF2E1FF93EF9370
:1024D0000E94839B0F5F1F4F0F900F900F900F90E4
:1024E0000830110559F720E030E048EC52E4C30110
:1024F000B2010E9478939F938F937F936F938FE99C
:1025000092E19F938F930E94839B0F900F900F9067
:102510000F900F900F90888581114AC08AE993E04F
:102520009F938F933F922F920E94839B9F928F92B3
:102530000E94839BFFEFEF1AFF0A29960F900F90DE
:102540000F900F900F900F90F601808190E0E816A9
:10255000F9068CF5CE010E949463BC01990F880B9B
:10256000990B0E942C942B013C01A114B10409F495
:10257000A3CF20E030E048EC52E40E9478939F9390
:102580008F937F936F938CEA92E19F938F930E9436
:10259000839B89E992E19F938F930E94839B8DB7E0
:1025A0009EB708960FB6F8949EBF0FBE8DBF03C0AE
:1025B00088E193E0B5CFDF91CF911F910F91FF900C
:1025C000EF90DF90CF90BF90AF909F908F907F90D3
:1025D0006F905F904F903F902F900895CF93DF932F
:1025E0001F921F92CDB7DEB7EEE8F6E381818983B3
:1025F00087818A83CE0101960E94E27F0F900F901F
:10260000DF91CF910895CF93DF93EC0120918E3627
:1026100030918F364091903650919136609192363C
:10262000709193368091943690919536AFEF0E94D9
:102630008892E1F427E04AE250E06BE270E089E240
:1026400090E00E94CE6180E090E00E943811C8586E
:10265000DB4E888349E050E06EE070E08EE896E360
:102660000E943A9EDF91CF910C94EE12DF91CF91B0
:1026700008951F920F920FB60F9211240BB60F926E
:10268000FF920F931F932F933F934F935F936F93FB
:102690007F938F939F93AF93BF93CF93DF93EF93EA
:1026A000FF938091A53682608093A5368091660263
:1026B00086FD2B9A8091660287FD2B9A809191026C
:1026C000909192021816190614F4749A739A8091D4
:1026D0007D1490917E14A0917F14B091801485FF99
:1026E00002C0749873988091060290910702019736
:1026F0009093070280930602892B09F04FC18091C5
:10270000320B9091330B01969093330B8093320BE5
:102710008091CB319091CC31A091CD31B091CE311F
:102720000196A11DB11D8093CB319093CC31A09324
:10273000CD31B093CE3180E190E090930702809349
:1027400006028091660280FD02C01D9B05C01092AA
:102750007C1410927B1406C081E090E090937C146E
:1027600080937B1480917D1490917E14A0917F14AE
:10277000B091801497FF08C080917B1490917C14D5
:10278000892B49F0749A739808EA1DE1C0EED1E3F1
:10279000FF24F39441C0739A7498F6CF8091320B62
:1027A0009091330B0196BF010E945890892BE1F55F
:1027B000D80112964C91417020E030E050E060E08A
:1027C00070E080E090E0A0E00E94889269F1779844
:1027D00080917D1490917E14A0917F14B09180140B
:1027E00092FF05C074981092920210929102F80123
:1027F0006085718561157105C1F4D80118966D91D8
:102800007C9119976115710511F5065F1F4F25968B
:10281000B1E3C43FDB0779F1D8011896ED91FC9143
:102820001997309721F3BACFBF018091320B909165
:10283000330B01960E945890892BF9F61C821B825B
:10284000AE0162E184E292E00E949E78D6CF809150
:10285000320B9091330B0E945890892BB1F6F8827D
:102860001A8309831C821B82AE0162E182E492E03A
:102870000E949E78CACF60916C0270916D026115C2
:102880007105A1F18091320B9091330B0E94589009
:10289000892B61F58091743690917536A0917636CA
:1028A000B09177364091BD295091BE296091BF29E2
:1028B0007091C029841B950BA60BB70B8093D01D7C
:1028C0009093D11DA093D21DB093D31D80917436E7
:1028D00090917536A0917636B09177368093BD2968
:1028E0009093BE29A093BF29B093C02960916A023A
:1028F00070916B0261157105A1F18091320B90917D
:10290000330B0E945890892B61F580917836909115
:102910007936A0917A36B0917B364091C129509199
:10292000C2296091C3297091C429841B950BA60B01
:10293000B70B8093D41D9093D51DA093D61DB09353
:10294000D71D8091783690917936A0917A36B091E2
:102950007B368093C1299093C229A093C329B09359
:10296000C4298091660286FD2B9880916602909121
:102970006702A0916802B091690291FF0FC00E94A6
:10298000DC718A3119F0C1E0C80F01C0CBE00E94B0
:102990001A708C2F0E94ED710E94E37040E050E0AD
:1029A00060E08BEA92E00E949E78FF91EF91DF91C8
:1029B000CF91BF91AF919F918F917F916F915F91D7
:1029C0004F913F912F911F910F91FF900F900BBE50
:1029D0000F900FBE0F901F9018958091F81D909149
:1029E000DF31891B08950E94ED14882371F0E09176
:1029F000DF31EF73F0E0E75BF14E808190E02091F2
:102A0000DF312F5F2093DF3108958FEF9FEF08951F
:102A1000CF93DF93EC011092630B1092620B8881CD
:102A200099810097C1F08D3E934021F01982188260
:102A300083E0B8C0613109F0B4C00E94F314992753
:102A400090935E0B80935D0B8D30910509F444C02B
:102A50008F3F910549F40E94ED148111EECF8DEE68
:102A600093E0998388839DC08231910509F45AC00F
:102A70008F37910509F052C080915B0B90915C0BF0
:102A8000181619060CF56091033B7091043B88E021
:102A900090E00E94339B6091033B7091043B80E285
:102AA00090E00E94339B6091033B7091043B88E06F
:102AB00090E00E94339B80915B0B90915C0B01979F
:102AC00090935C0B80935B0B80915B0B90915C0B04
:102AD0008F37910509F0BFCF1092DF311092F81DAA
:102AE00080915B0B90915C0BFC01EC50FE4C1082D2
:102AF0009093630B8093620B10925C0B10925B0BB4
:102B00008091973690919836009709F4A4CF40E0D1
:102B100050E0609175140E949E789DCF8830910599
:102B200071F5AACF6091033B7091043B8DE090E07A
:102B30000E94339B10925A0B1092590B8091590BA3
:102B400090915A0B20915B0B30915C0B821793078D
:102B50000CF0BACFFC01EC50FE4C80816091033B3D
:102B60007091043B90E00E94339B8091590B9091AF
:102B70005A0B019690935A0B8093590BDFCF6091BB
:102B8000033B7091043B0E94339B80915B0B9091BF
:102B90005C0B20915D0BFC01EC50FE4C20830196F8
:102BA0008FCF81E0DF91CF91089580917B14909138
:102BB0007C14892BD1F08091660290916702A091DC
:102BC0006802B091690293FD10C00E941A7083B729
:102BD000817F866083BFF89483B7816083BF7894D8
:102BE000889583B78E7F83BF78940895CF93DF93C2
:102BF000FC01208131812115310551F0223B324108
:102C000029F0FC011182108283E015C0653891F42F
:102C1000EC010E941A6F0E94D51540E050E065E873
:102C20008091E2159091E3150E949E7882EB92E1EB
:102C30009983888381E0DF91CF910895CF93DF93CB
:102C4000EB01892B61F05F934F9386E992E19F93AB
:102C50008F930E94839B0F900F900F900F90DF93A4
:102C6000CF9383E992E19F938F930E94839B0F9070
:102C70000F900F900F90DF91CF910895CF93DF9336
:102C8000D62FC42F0E9457648D2F0E9488648C2FEA
:102C90000E948864DF91CF910C948064CF92DF9280
:102CA000EF92FF920F931F93CF93DF93C82FD62FEE
:102CB000F42E152F022F0E9457648D2F0E948864D6
:102CC0008C2F81600E947E64CF2DD12F10E0E12CEB
:102CD000F12C680181E0C81AD108E016F10671F004
:102CE000CE14DF0419F40E94A36402C00E94996408
:102CF00088838FEFE81AF80A2196EFCFDF91CF9102
:102D00001F910F91FF90EF90DF90CF900C94806413
:102D1000CF92DF92EF92FF920F931F93CF93DF93A7
:102D20001F92CDB7DEB70E941A6F80EB0E9423641A
:102D300081111CC00E9480648091C52D9091C62D88
:102D400081609093C62D8093C52D81E293E09F937F
:102D50008F9383E992E19F938F930E94839B0F90BF
:102D60000F900F900F9001E010E002C000E010E023
:102D70008EB18470F82E729A64E278E680E090E07A
:102D80000E9400640E941A6F8EE40E9423648111E5
:102D900017C00E9480648091C52D9091C62D8260DD
:102DA0009093C62D8093C52D68018FEFC81AD80A5D
:102DB00043EB59E069E273E0C8010E941E168601E8
:102DC000F11001C0729864E278E680E090E00E9421
:102DD00000640E941A6F8EEE0E942364811159C014
:102DE00019820E94806421E030E0AE014F5F5F4FA6
:102DF00060ED70E08EEE90E00E944E168981853580
:102E0000A9F48091C52D9091C62D84609093C62D14
:102E10008093C52D78018FEFE81AF80A43EB59E04B
:102E200061E373E0C8010E941E168701898188351D
:102E3000A9F48091C52D9091C62D80619093C62DE7
:102E40008093C52D78018FEFE81AF80A43EB59E01B
:102E500068E373E0C8010E941E16870189818036ED
:102E6000C1F48091C52D9091C62D80629093C62D9E
:102E70008093C52D78018FEFE81AF80A43EB59E0EB
:102E80006FE373E0C8010E941E1681E00E948D6707
:102E9000870164E278E680E090E00E9400640E948E
:102EA0001A6F86EA0E942364811117C00E94806411
:102EB0008091C52D9091C62D80649093C62D8093EE
:102EC000C52D78018FEFE81AF80A43EB59E066E464
:102ED00073E0C8010E941E16870164E278E680E074
:102EE00090E00E9400640E941A6F8CE30E942364A9
:102EF00081111FC00E9480648091C52D9091C62DC4
:102F000080689093C62D8093C52D78018FEFE81AC5
:102F1000F80A43EB59E06EE473E0C8010E941E1604
:102F20008BE892E19F938F930E94839B0F900F9069
:102F3000870164E278E680E090E00E9400640E94ED
:102F40001A6F82ED0E942364811117C00E94806471
:102F50008091C52D9091C62D91609093C62D809340
:102F6000C52D78018FEFE81AF80A43EB59E066E5C2
:102F700073E0C8010E941E16870164E278E680E0D3
:102F800090E00E9400640E941A6F80E80E9423640F
:102F9000811117C00E9480648091C52D9091C62D2B
:102FA00098609093C62D8093C52D78018FEFE81A15
:102FB000F80A43EB59E06FE573E0C8010E941E1662
:102FC000870164E278E680E090E00E9400640E945D
:102FD0001A6F80ED0E942364811117C00E948064E3
:102FE0008091C52D9091C62D94609093C62D8093AD
:102FF000C52D78018FEFE81AF80A43EB59E065E632
:1030000073E0C8010E941E16870164E278E680E042
:1030100090E00E9400640E941A6F8CEE0E9423646C
:10302000811117C00E9480648091C52D9091C62D9A
:1030300090619093C62D8093C52D78018FEFE81A8B
:10304000F80A43EB59E06DE673E0C8010E941E16D2
:10305000870187E0E82EF12C64E278E680E090E0DA
:103060000E9400640E941A6F8CE70E942364811101
:1030700013C00E9480648091C52D9091C62D9260EE
:103080009093C62D8093C52D43EB59E064E773E020
:10309000C8010E941E1604C081E0E81AF108E1F69A
:1030A0000E94806489E992E19F938F930E94839BA1
:1030B0000F900F900F90DF91CF911F910F91FF9084
:1030C000EF90DF90CF900895AF92BF92CF92DF92B2
:1030D000EF92FF920F931F93CF93DF93CDB7DEB79D
:1030E00060970FB6F894DEBF0FBECDBFF82EE42E6A
:1030F0006623E9F18E010F5F1F4F80E1F801119205
:103100008A95E9F728E0A80168E980EB0E944E164D
:10311000FF2041F08DE793E09F938F930E946F9B78
:103120000F900F905E01F8E0AF0EB11C94E8C92E2D
:1031300093E0D92EF80181918F011F928F93DF9236
:10314000CF920E946F9B0F900F900F900F900A15D7
:103150001B0581F788851F928F9389ED93E09F93DC
:103160008F930E946F9B0F900F900F900F90EE2007
:10317000E9F18E010F5F1F4F80E1F80111928A95EE
:10318000E9F720E1A80160E880EB0E944E16FF20DD
:1031900041F089E893E09F938F930E946F9B0F907B
:1031A0000F906E01F0E1CF0ED11C84E8E82E83E091
:1031B000F82EF80181918F011F928F93FF92EF9269
:1031C0000E946F9B0F900F900F900F90C016D1062A
:1031D00081F788891F928F9389ED93E09F938F9356
:1031E0000E946F9B0F900F900F900F9060960FB6FC
:1031F000F894DEBF0FBECDBFDF91CF911F910F912D
:10320000FF90EF90DF90CF90BF90AF9008950F9315
:103210001F93CF93DF931F921F92CDB7DEB71A8211
:10322000198222E0AE014F5F5F4F6AEA8EEE0E9484
:103230004E1609E81EE189819A81982789279827E7
:10324000F8019183808322E0AE014F5F5F4F6CEA0B
:103250008EEE0E944E1689819A8198278927982799
:10326000F8019383828322E0AE014F5F5F4F6EEAE5
:103270008EEE0E944E1689819A8198278927982779
:10328000F8019583848322E0AE014F5F5F4F60EBCE
:103290008EEE0E944E1689819A8198278927982759
:1032A000F801938B828B22E0AE014F5F5F4F62EBA0
:1032B0008EEE0E944E1689819A8198278927982739
:1032C000F801958B848B22E0AE014F5F5F4F64EB7A
:1032D0008EEE0E944E1689819A8198278927982719
:1032E000F801978B868B22E0AE014F5F5F4F66EB54
:1032F0008EEE0E944E1689819A81982789279827F9
:10330000F8019783868322E0AE014F5F5F4F68EB41
:103310008EEE0E944E1689819A81982789279827D8
:10332000F8019187808722E0AE014F5F5F4F6AEB23
:103330008EEE0E944E1689819A81982789279827B8
:10334000F8019587848722E0AE014F5F5F4F6CEBF9
:103350008EEE0E944E1689819A8198278927982798
:10336000F8019787868722E0AE014F5F5F4F6EEBD3
:103370008EEE0E944E1689819A8198278927982778
:10338000F801918B808B0F900F90DF91CF911F915F
:103390000F9108952F923F924F925F926F927F927A
:1033A0008F929F92AF92BF92CF92DF92EF92FF9255
:1033B0000F931F93CF93DF93CDB7DEB769970FB607
:1033C000F894DEBF0FBECDBF182FD62E042F2F8B43
:1033D0009E012F5F3F4F790183E0F90111928A9599
:1033E000E9F78091AD1E811105C00E94071981E0A7
:1033F0008093AD1EDD2009F46DC04EE264EF8EEEC9
:103400000E943E1662E174E380E090E00E94006456
:1034100022E0A70166EF8EEE0E944E1629813A81C6
:10342000322723273227A90160E070E080919F1E98
:103430009091A01E9A01AB01281B390B410951093B
:10344000A0919D1EB0919E1E0E94E7906B017C0191
:103450003FE0F594E794D794C7943A95D1F76091FB
:10346000971E7091981ECB01770FAA0BBB0BBC0166
:10347000CD014BE0660F771F881F991F4A95D1F742
:103480002091991E30919A1E4901330FAA08BB085A
:10349000A50194012C0D3D1D4E1D5F1D0E94A290A3
:1034A000C20ED31ED092941EC092931EF8E0CF0E8F
:1034B000D11C54E0D594C7945A95E1F70D2C000C1B
:1034C000EE08FF08C092A11ED092A21EE092A31E99
:1034D000F092A41E812F8295880F880F807C8C5CCF
:1034E0008A87212F30E039872887A3E0B0E0012EBA
:1034F00002C0AA0FBB1F0A94E2F72AE63AE00E9434
:10350000E0909B01AC012E5F3F4F4F4F5F4F2B87E9
:103510003C874D875E8780E593ECA0E0B0E09C019E
:10352000AD0104C055954795379527951A95D2F763
:103530002B8B3C8B4D8B5E8B10E0412C512C320140
:1035400088E090E0AC01E885F9854E1B5F0B598F50
:10355000488F101709F439C14A8564EF8EEE0E9436
:103560003E166B857C858D859E850E94006423E0D8
:10357000AE014F5F5F4F66EF8EEE0E944E162090B9
:10358000931E3090941EF0EA2F1AFFE03F0A91013B
:10359000D1010E94C9906C837D838E839F83E091CB
:1035A0008B1EF0918C1EF88BEF87E091891EF091B5
:1035B0008A1EFA8BE98BE0918D1EF0918E1EA091F0
:1035C0008F1EB091901E9B01AC018CE055954795E4
:1035D000379527958A95D1F70E94F2906C01FF24C8
:1035E000D7FCF094EF2C9101DF010E94C990DC011F
:1035F000CB013DE0B595A795979587953A95D1F77D
:103600008C0D9D1DAE1DBF1D0296A11DB11D42E07A
:10361000B595A795979587954A95D1F79C01AD01EA
:1036200030584F4F5F4FA0919B1EB0919C1E0E943F
:10363000E7904B015C015FE0B694A7949794879460
:103640005A95D1F78981CA80D12CE12CF12CFE2C1E
:10365000ED2CDC2CCC24E82A8B81C82A088C04C0F1
:10366000F594E794D794C7940A94D2F7A091911E49
:10367000B091921E2C813D814E815F810E94F2901B
:103680009B01AC0177E155954795379527957A953C
:10369000D1F72C833D834E835F839101AF85B88939
:1036A0000E94C990DC01CB01EBE0B595A7959795F9
:1036B0008795EA95D1F72C813D814E815F81820FFC
:1036C000931FA41FB51FE989FA89AF01FF0F660B8D
:1036D000770BF2E0440F551F661F771FFA95D1F75D
:1036E000840F951FA61FB71F088404C0880F991F59
:1036F000AA1FBB1F0A94D2F70296A11DB11D22E09A
:10370000B595A795979587952A95D1F7A701960125
:10371000281B390B4A0B5B0B6B897C898D899E8931
:103720000E943C9097FD0BC0660F771F881F991F62
:10373000A50194010E94809049015A010AC0A50187
:1037400094010E94809049015A01880C991CAA1C7E
:10375000BB1C9927B7FC9A958B2D7A2D692D9B015F
:10376000AC010E943C909B01AC01AEEDBBE00E941D
:10377000E7906B017C01A3E4B3EEA50194010E94E4
:10378000F590BB2797FDB095AB2F6701FF24D7FCC1
:10379000F094EF2CC80ED91EEA1EFB1EFFECCF0ED4
:1037A000FEE0DF1EE11CF11C44E0F594E794D794A1
:1037B000C7944A95D1F78C0C9D1CAE1CBF1C480CBD
:1037C000591C6A1C7B1C1F5FC4CE112381F0212F62
:1037D00030E040E050E0C301B2010E9480902093AD
:1037E000A51E3093A61E4093A71E5093A81E2F8996
:1037F000222389F16091A51E7091A61E8091A71EBB
:103800009091A81E611571058105910521F10E9415
:103810002C9420E836EE45EC57E40E94789321E0A2
:103820003EED42E45EE30E9491969B01AC0160E0B4
:1038300070E080E89FE30E9494922BE43AE34DEB22
:1038400057E30E9478936093A91E7093AA1E8093F9
:10385000AB1E9093AC1E69960FB6F894DEBF0FBEF8
:10386000CDBFDF91CF911F910F91FF90EF90DF902F
:10387000CF90BF90AF909F908F907F906F905F9010
:103880004F903F902F9008950F931F93CF93DF9306
:1038900000D000D0CDB7DEB78E010F5F1F4F86E09E
:1038A000F80111928A95E9F780919F1D811113C04B
:1038B00040E061E386EA0E943E164AE06CE286EA56
:1038C0000E943E1681E080939F1D68EF7CE780E0B8
:1038D00090E00E94006448E06DE286EA0E943E1695
:1038E00068EF7CE780E090E00E94006426E0A80199
:1038F00062E386EA0E944E1647E06DE286EA0E9485
:103900003E1689819A818093991D90939A1D2B81EF
:103910003C8120939B1D30939C1D4D815E81409383
:103920009D1D50939E1D5F934F933F932F939F93A5
:103930008F938DE893E09F938F930E946F9B0FB6B8
:10394000F894DEBF0FBECDBF26960FB6F894DEBF4B
:103950000FBECDBFDF91CF911F910F9108958F9230
:103960009F92AF92BF92CF92DF92EF92FF920F930E
:103970001F93CF93DF9300D000D0CDB7DEB78E0179
:103980000F5F1F4F86E0F80111928A95E9F741E039
:1039900062E08CE30E943E1648E560E08CE30E9402
:1039A0003E1664E278E680E090E00E94006426E043
:1039B000A80163E08CE30E944E1643E062E08CE3D2
:1039C0000E943E1609811A81102701271027E9E776
:1039D000FDE111830083EB80FC80FE24EF24FE24B4
:1039E000F382E282CD80DE80DC24CD24DC24D5820B
:1039F000C482B801012E000C880B990B0E942C94F4
:103A00004B015C01B7010F2C000C880B990B0E9435
:103A10002C94A50194010E94149320EE3EE245E609
:103A200052E40E94249620E030E044E353E40E94F4
:103A300095929F938F937F936F93DF92CF92FF9294
:103A4000EF921F930F938BE993E09F938F930E94C4
:103A50006F9B0FB6F894DEBF0FBECDBF26960FB694
:103A6000F894DEBF0FBECDBFDF91CF911F910F91B4
:103A7000FF90EF90DF90CF90BF90AF909F908F908E
:103A80000895CF93DF93EC01888199810097A9F184
:103A90008739924121F01982188283E083C080E443
:103AA0009BE00E946F76892BA1F180917D1490910B
:103AB0007E14A0917F14B091801493FD2CC080914E
:103AC0007D1490917E14A0917F14B091801493FD89
:103AD00053C080917D1490917E14A0917F14B09179
:103AE000801494FD51C080917D1490917E14A0911A
:103AF0007F14B091801495FD4EC040E850E060E026
:103B000070E080E49BE00E94517687E992E199831E
:103B1000888381E047C08091C52D82FFD0CF21E00E
:103B200048E061E083E00E94CA198091AC1E8F9347
:103B30008091AB1E8F938091AA1E8F938091A91EB6
:103B40008F938091A81E8F938091A71E8F93809151
:103B5000A61E8F938091A51E8F938FE493E19F9370
:103B60008F930E94839B8DB79EB70A960FB6F894E9
:103B70009EBF0FBE8DBFA3CF8091C52D85FFA9CF5E
:103B800081E00E948368A5CF8091C52D86FFABCFD1
:103B90000E94441CA8CF8091C52D87FFAECF0E9404
:103BA000AF1CABCFDF91CF910895CF93DF93C82F98
:103BB0008CEE0E947E648C2F0E9488646AE67AE014
:103BC00080E090E00E9400648DEE0E947E640E947E
:103BD0009964D82F0E94A364C82F0E9480648C2F00
:103BE00090E09D2BDF91CF9108951F93CF93DF93AA
:103BF000C82F8CEE0E947E648C2F0E94886464E241
:103C000078E680E090E00E9400648CEE0E947E6482
:103C100080E00E9488646AE67AE080E090E00E949A
:103C200000648DEE0E947E640E949964182F0E94A9
:103C30009964C82F0E94A364D82F0E9480648C2F9F
:103C400090E0A0E0B0E0BA2FA92F982F8827A12BF1
:103C5000BC01CD016D2BDF91CF911F9108952F9263
:103C60003F924F925F926F927F928F929F92AF920C
:103C7000BF92CF92DF92EF92FF920F931F93CF9359
:103C8000DF93CDB7DEB7CE54D1090FB6F894DEBFBF
:103C90000FBECDBF8091040290910502892BE1F106
:103CA00010920502109204028CEE0E947E648EE156
:103CB0000E9488640E94806466E37CE980E090E072
:103CC0000E94006482EA0E94D51D9093310B80937C
:103CD000300B84EA0E94D51D90932F0B80932E0BFE
:103CE00086EA0E94D51D90932D0B80932C0B88EAB9
:103CF0000E94D51D90932B0B80932A0B8AEA0E9479
:103D0000D51D9093290B8093280B8CEA0E94D51D1A
:103D10009093270B8093260B88E40E94F51D6AAFD1
:103D20007BAF8CAF9DAF88E50E94F51D2091280BDD
:103D30003091290B4B015C01A90160E070E080E04B
:103D400090E0DC0127962FAF279728965FAF289742
:103D500029966FAF29972A967FAF2A972B968FAF18
:103D60002B972C969FAF2C972D96AFAF2D972E9615
:103D7000BFAF2E97AB0160E070E080E090E008E01C
:103D80000E942A922A833983B42FA52FF62FE72F7A
:103D90008C019401A50160E070E080E090E0AA80D1
:103DA000B980CB2EDA2EEF2EFE2E0E9476922901BC
:103DB0004A016DA37CA389839A83315041095F4FE7
:103DC0006F4F7F4F8F4F9F4F66246394712C211547
:103DD0003F4F4F4F5140610571058105910509F035
:103DE00010F4612C712C13014091260B5091270B7C
:103DF00052016401EDA0FCA009811A819A0140E002
:103E000050E060E070E080E090E00E94FA90F22ED6
:103E1000032F142FB52FF62FE72FD82EE92EA0E071
:103E20000E94889284F42150310940485F4F6F4FBF
:103E30007F4F8F4F9F4FF22E032F142FB52FF62F4A
:103E4000E72FD82EE92E2F2D302F412F5B2F6F2FEC
:103E50007E2F8D2D9E2D07E10E9443922C8F3D8F4A
:103E60004E8F5F8F68A379A38AA39BA32053384FFB
:103E70004F4F5F4F6F4F7F4F8F4F9F4F2C8B3D8B1F
:103E80004E8B5F8B688F798F8A8F9B8F2056304F38
:103E90004F4F5F4F6F4F7F4F8F4F9F4F243D3043AA
:103EA00041055105610571058105910529F020F055
:103EB0001301EFEF2E1A3E0A40912A0B50912B0B63
:103EC00052016401EDA0FCA009811A819A0140E031
:103ED00050E060E070E080E090E00E94FA90F22E06
:103EE000032F142FB52FF62FE72FD82EE92EA0E0A1
:103EF0000E9488925CF4AFE70E946A92F22E032F30
:103F0000142FB52FF62FE72FD82EE92E2F2D302F77
:103F1000412F5B2F6F2F7E2F8D2D9E2D07E00E944E
:103F200043922B833C833A01B62FA72FF82FE92F1A
:103F3000A0902E0BB0902F0B950140E050E060E078
:103F400070E080E090E000E10E942A9259016A014D
:103F50007B018C012B813C81A3016B2F7A2F8F2F4A
:103F60009E2F0E9461922B833C8349875A876B87DF
:103F70007C878D879E872E5F3F4F434051096E4F50
:103F80007F4F8F4F9F4F22303105494F5F4F644025
:103F900071058105910521F018F02FEF221A320AE0
:103FA0004091300B5091310B5E834D8340912C0B2F
:103FB00050912D0B52016401EDA0FCA009811A81E2
:103FC0009A0140E050E060E070E080E090E00E9404
:103FD000FA90F22E032F142FB52FF62FE72FD82E9D
:103FE000E92EA0E00E94889284F421503F4F4F4F69
:103FF0005F4F6F4F7F4F8F4F9F4FF22E032F142F26
:10400000B52FF62FE72FD82EE92E2F2D302F412F49
:104010005B2F6F2F7E2F8D2D9E2D08E00E944392E7
:104020002F8338873A01B62FA72FF82FE92F6D81FC
:104030007E81C12CD12C9B01A60160E070E080E064
:1040400090E00FE00E942A9259016A017B018C01E5
:104050002F813885A3016B2F7A2F8F2F9E2F0E94DF
:1040600061922D833F8348875F87688B798B8A8B2A
:104070009B8B2F5F3F4F414051096F4F7F4F8F4FB9
:104080009F4F213030484C4F5F476240710581059A
:10409000910521F018F0BFEF2B1A3B0A2C893D89BE
:1040A0004E895F89688D798D8A8D9B8D2F3C374035
:1040B00041055105610571058105910511F00CF06F
:1040C000D3C152016401EDA0FCA009811A819201C3
:1040D000A401B701C8010E94FA90122F3A834983C4
:1040E000B52FF62FE72FF82E092FA0E00E94889217
:1040F00084F421503109410950486F4F7F4F8F4F51
:104100009F4F122F3A834983B52FF62FE72FF82EB2
:10411000092F212F3A8149815B2F6F2F7E2F8F2D01
:10412000902F0FE10E9443922EAF3FAF21964FAFE9
:10413000219722965FAF229723966FAF23972496FD
:104140007FAF249725968FAF259726969FAF26970A
:1041500045E0A42EB12CC12CD12CE12CF12C00E097
:1041600010E02C8D3D8D4E8D5F8D68A179A18AA1C7
:104170009BA10E94FA90AC8CBD8CCE8CDF8CE8A009
:10418000F9A00AA11BA10E94FA90122F3BAB4AABE7
:10419000B52FF62FE72F7C01922EA32EB42EC52E1D
:1041A000D62E072F782E8F2CA0E00E9488925CF4E8
:1041B000A1E00E946A92922EA32EB42EC52ED62E76
:1041C000072F782E892E292D3A2D4B2D5C2D6D2D04
:1041D000702F872D982D01E00E9443922AA73BA7BC
:1041E0004CA75DA76EA77FA788AB99AB29833A83BD
:1041F0004CA35DA36EA37FA388A799A7212F3BA9FA
:104200004AA95B2F6F2F7E2FC701A0E00E948892E2
:1042100054F4A3E00E946A92122F3BAB4AABB52F35
:10422000F62FE72F7C01212F3BA94AA95B2F6F2F87
:104230007E2FC70102E00E9443922AAB3BAB4CABFE
:104240005DAB6EAB7FAB88AF99AF2F962FAF2F973B
:1042500027963FAF2797B42FA52FF62FE72F4C01B6
:104260002C893D894E895F89688D798D8A8D9B8DDA
:1042700024323A4F4F4F5F4F6F4F7F4F8F4F9F4FBB
:104280000CF088C02C8D3D8D4E8D5F8D68A179A17D
:104290008AA19BA12455324F4F4F5F4F6F4F7F4FE5
:1042A0008F4F9F4F29013A014B018D8F9C8F27E043
:1042B000A22EB12CC12CD12CE12CF12C00E010E06D
:1042C00092010E94FA905201630174010D8D1C8DC0
:1042D0000E94FA90AAA4BBA4CCA4DDA4EEA4FFA4DF
:1042E00008A919A90E94619229833A834CA35DA36E
:1042F0006EA37FA388A799A73BE0A32EB12CC12C66
:10430000D12CE12CF12C00E010E09201A301B401CA
:104310008D8D9C8D0E94FA905201630174010D8D68
:104320001C8D0E94FA90122F3D8F4C8FB52FF62FC7
:10433000E72FF82E092FA0E00E9488925CF4A1E0FC
:104340000E946A92122F3D8F4C8FB52FF62FE72FC8
:10435000F82E092F212F3D8D4C8D5B2F6F2F7E2F37
:104360008F2D902F01E00E944392AAA8BBA8CCA851
:10437000DDA8EEA8FFA808AD19AD0E9461922F96A6
:104380002FAF2F9727963FAF2797B42FA52FF62F44
:10439000E72F4C012B813C8149855A856B857C85B3
:1043A0008D859E85A980BA80CCA0DDA0EEA0FFA05F
:1043B00008A519A50E9476922B833C8349875A87CA
:1043C0006B877C878D879E872D813F8148855F85A0
:1043D000688979898A899B892F96AFAC2F97279610
:1043E000BFAC2797CB2EDA2EEF2EFE2E84010E9433
:1043F00076922D833F8348875F87688B798B8A8B82
:104400009B8B2C893D894E895F89688D798D8A8D3A
:104410009B8DAEACBFAC2196CFAC21972296DFAC82
:1044200022972396EFAC23972496FFAC24972596EA
:104430000FAD259726961FAD26970E94769220569F
:10444000304F4F4F5F4F6F4F7F4F8F4F9F4F243DE8
:10445000304341055105610571058105910521F044
:1044600018F0BFEF2B1A3B0A4AAD5BAD6CAD7DADCA
:104470009A01AB0160E070E0CB0127962FAF279740
:1044800028963FAF289729964FAF29972A965FAF76
:104490002A972B966FAF2B972C967FAF2C972D9644
:1044A0008FAF2D972E969FAF2E97AD80BF80C8847B
:1044B000DF84E888F9880A891B8960E070E080E081
:1044C00090E00E94FA90122F3A834983B52FF62F7D
:1044D000E72FF82E092FA0E00E94889284F4215043
:1044E0003109404E5F4F6F4F7F4F8F4F9F4F122FBD
:1044F0003A834983B52FF62FE72FF82E092F212F66
:104500003A8149815B2F6F2F7E2F8F2D902F05E1F0
:104510000E944392AB80BC80C984DA84EB84FC8423
:104520000D851E850E947692122F3A834983B52FFE
:10453000F62FE72FF82E092FA0E00E94889284F42E
:10454000215030484F4F5F4F6F4F7F4F8F4F9F4FDE
:10455000122F3A834983B52FF62FE72FF82E092F14
:10456000212F3A8149815B2F6F2F7E2F8F2D902F26
:104570000FE00E94439259016A017B018C01722E67
:104580006B2CB42FAD2DF62F5F2C4C01285E3340E1
:10459000410951096109710981099109283D304D8D
:1045A00041405105610571058105910509F010F43F
:1045B000232869F09501A601B701C8010E94E39183
:1045C000722E632EB42FA52FF62F572E4C01272DB8
:1045D000362D4B2F5A2F6F2F752DC4010E94249416
:1045E00020E030E048EC52E40E947893C25BDF4F59
:1045F0000FB6F894DEBF0FBECDBFDF91CF911F91F4
:104600000F91FF90EF90DF90CF90BF90AF909F9071
:104610008F907F906F905F904F903F902F90089574
:104620004F925F926F927F928F929F92AF92BF92C2
:10463000CF92DF92EF92FF922B013C0169017A0148
:1046400023EC35EF4CE851E4C701B6010E942496F3
:104650004B015C0128EB3EE143E753E4C701B6019F
:104660000E9495929B01AC01C501B4010E94789310
:104670000E94F2934B015C0120E030E048EC52E4F0
:10468000C301B2010E94789321E835E943EC50E47C
:104690000E942496A50194010E9424964B015C017E
:1046A00023E333E948E853E4C701B6010E94959239
:1046B0009B01AC01C501B4010E94789323E333EB65
:1046C00048E553E40E942496FF90EF90DF90CF904E
:1046D000BF90AF909F908F907F906F905F904F9022
:1046E00008954F925F926F927F928F929F92AF92B6
:1046F000BF92CF92DF92EF92FF9269017A010E94FE
:1047000098954B015C0123EC35EF4CE851E4C7016F
:10471000B6010E9424962B013C0128EB3EE143E7C1
:1047200053E4C701B6010E9495929B01AC01C301FD
:10473000B2010E9478936B017C0120E030E040E000
:1047400050E4C501B4010E94949222E93CE54EED8B
:104750005EE30E9478939B01AC01C701B6010E9401
:1047600095926B017C0128EB3EE143E753E40E9404
:1047700024964B015C01A701960163EC75EF8CE870
:1047800091E40E9494929B01AC01C501B4010E9486
:104790007893FF90EF90DF90CF90BF90AF909F9075
:1047A0008F907F906F905F904F9008954F925F929F
:1047B0006F927F928F929F92AF92BF92CF92DF9231
:1047C000EF92FF922B013C0169017A0123EC35EF56
:1047D0004CE851E4C701B6010E9424964B015C01EC
:1047E00028EB3EE143E753E4C701B6010E949592EE
:1047F0009B01AC01C501B4010E9478930E94F29321
:104800004B015C0120E030E048EC52E4C301B2010E
:104810000E947893A50194010E94249620E030E044
:1048200040E251E40E94949224EE38E34EE05FE3CC
:104830000E942496A70196010E949592FF90EF9006
:10484000DF90CF90BF90AF909F908F907F906F90B0
:104850005F904F90089580E80E947E6481110DC0A2
:104860008EEF0E948864811108C066E37CE980E0D5
:1048700090E00E9400640C9480640E9480648091A7
:10488000D7319091D831A091D931B091DA310196D8
:10489000A11DB11D8093D7319093D831A093D93108
:1048A000B093DA310895FC01DC01AC014E5F5F4F3B
:1048B00090E031E38D91982788E0292F220F97FF10
:1048C00003C0922F932701C0922F8150B1F7A417F4
:1048D000B50781F721E030E08281891711F020E0EF
:1048E00030E0C9010895DF92EF92FF920F931F937A
:1048F000CF93DF930E942B2480E80E947E64811175
:104900006DC08AEF0E948864811168C08FE00E94A8
:104910008864811163C06AE67AE080E090E00E94DA
:10492000006481E80E947E64811158C00E949964ED
:10493000D82F0E9499640E949964182F0E9499644C
:104940000E949964082F0E9499640E94A364F82E23
:1049500080E80E947E64811141C08CEF0E948864CF
:1049600081113CC089EC0E948864811137C06AE6DD
:104970007AE080E090E00E94006481E80E947E641A
:104980000E949964E82E0E949964D82E0E9499642E
:104990000E949964C82F0E94A3641F92DF921F9205
:1049A000EF921F92FF921F920F931F921F931F92DD
:1049B000DF931F928F931F92CF9380EB93E09F938F
:1049C0008F930E946F9B0E9480648DB79EB7429622
:1049D0000FB6F8949EBF0FBE8DBF17C00E948064B3
:1049E0008091D7319091D831A091D931B091DA31FD
:1049F0000196A11DB11D8093D7319093D831A0931A
:104A0000D931B093DA310E942B2420E030E040E02D
:104A100050E060E070E080E090E0DF91CF911F9186
:104A20000F91FF90EF90DF900895EF92FF920F9318
:104A30001F93CF93DF9300D0CDB7DEB78C0180E812
:104A40000E947E64811154C00115110551F085EE5C
:104A50000E94886481114CC062E07EE281E090E0B7
:104A600009C083EE0E948864811142C062E375E749
:104A700083E090E00E94006481E80E947E648111DE
:104A800037C00E949964E82E89830E949964F82EA9
:104A90008A830E94A3648B830E948064CE01019666
:104AA0000E945324892B21F16F2D70E07E296C7FA9
:104AB00080E090E0012B69F00E942A9420E030E031
:104AC0004AEF5AE30E94249620E030E040EC50E4A4
:104AD0000CC00E942A9422E538EB4FE25BE30E946F
:104AE000249626E636E64BE352E40E9494921BC0DD
:104AF0000E9480648091D7319091D831A091D931B2
:104B0000B091DA310196A11DB11D8093D7319093F8
:104B1000D831A093D931B093DA310E942B2460EFC1
:104B20007FEF89E794E40F900F900F90DF91CF9182
:104B30001F910F91FF90EF9008950F931F93CF93C4
:104B4000DF93729A8091660283FF08C08EE40E9410
:104B50002364811165C0C0E5D0E009C0C0E5D0E0A4
:104B60008FED97E00E941D0E2197D1F7EFCF8FEDCB
:104B700097E00E941D0E2197D1F78FE40E942364D5
:104B80000E949964D82FDF730E949964082F0E94B5
:104B90009964C82F0E94A364182F0E94806480919A
:104BA000660283FF72986D2F70E0762F6627600F84
:104BB000711D80E090E00E942A9420E134E048ECEE
:104BC0005BE30E9424966093B9297093BA2980937D
:104BD000BB299093BC296C2F70E0762F6627610F5C
:104BE000711D769567957695679580E090E00E94B7
:104BF0002A9424EA3CEF44E25CE30E94249620E0FD
:104C000030E040E252E40E9494926093A6367093A2
:104C1000A7368093A8369093A93680E090E002C032
:104C200081E090E0DF91CF911F910F9108957298EC
:104C3000729A8EE40E94236480EA0E94886480E075
:104C40000E94886480E00E9488648FE40E9423644C
:104C50000E9499648EE40E94236480E80E94886424
:104C600080E00E94886480E00E9488640E948064E2
:104C700080E090E008958EE792E19F938F930E94E9
:104C8000839B809180020F900F90882361F01F9288
:104C90008F938BE792E19F938F930E94839B0F905A
:104CA0000F900F900F90089586E592E19F938F9358
:104CB0000E94839B8EE292E19F938F930E94839B3D
:104CC00087E092E19F938F930E94839B8CEC91E10C
:104CD0009F938F930E94839B80E991E19F938F9391
:104CE0000E94839B8EE591E19F938F930E94839B0B
:104CF00082E291E19F938F930E94839B8CEF90E1DE
:104D00009F938F930E94839B86EC90E19F938F9358
:104D10000E94839B8091C52D9091C62D82709870C2
:104D20002DB73EB72E5E3F4F0FB6F8943EBF0FBE75
:104D30002DBF892B41F086E990E19F938F930E94CC
:104D4000839B0F900F908AE690E19F938F930E9430
:104D5000839B8EE290E19F938F930E94839B85E0DB
:104D600090E19F938F930E94839B89ED9FE09F9397
:104D70008F930E94839B8AEA9FE09F938F930E9468
:104D8000839B88E79FE09F938F930E94839B87E498
:104D90009FE09F938F930E94839B8DE09FE09F9362
:104DA0008F930E94839B87ED9EE09F938F930E9439
:104DB000839B87EA9EE09F938F930E94839B8BE760
:104DC0009EE09F938F930E94839B8CE49EE09F9331
:104DD0008F930E94839B83E19EE09F938F930E9419
:104DE000839B8AED9DE09F938F930E94839B83EA30
:104DF0009DE09F938F930E94839B85E79DE09F9307
:104E00008F930E94839B8DB79EB780960FB6F894C0
:104E10009EBF0FBE8DBF81E49DE09F938F930E9444
:104E2000839B80E19DE09F938F930E94839B81EE03
:104E30009CE09F938F930E94839B82EB9CE09F93C7
:104E40008F930E94839B8BE89CE09F938F930E949B
:104E5000839B85E59CE09F938F930E94839B8FE1CA
:104E60009CE09F938F930E94839B89EE9BE09F938E
:104E70008F930E94839B80EC9BE09F938F930E9473
:104E8000839B88E89BE09F938F930E94839B8DE593
:104E90009BE09F938F930E94839B2DB73EB72A5E22
:104EA0003F4F0FB6F8943EBF0FBE2DBF08958FED54
:104EB00093E00C94AB9B4F925F926F927F928F9294
:104EC0009F92AF92BF92CF92DF92EF92FF92CF93D9
:104ED000DF93CDB7DEB728970FB6F894DEBF0FBECD
:104EE000CDBF8091CB319091CC31A091CD31B0919B
:104EF000CE3189839A83AB83BC834090CB31509071
:104F0000CC316090CD317090CE318091CB31909189
:104F1000CC31A091CD31B091CE318D839E83AF83C2
:104F2000B8876091CB317091CC318091CD31909127
:104F3000CE312CE3822E912CA12CB12CA501940111
:104F40000E9480907F936F9330E1C32E3EE0D32E7A
:104F5000E12CF12C6D817E818F819885A7019601CE
:104F60000E948090A50194010E9480903F932F930E
:104F700040E8842E41E5942EAA24A394B12CC301C9
:104F8000B201A50194010E948090A70196010E94A0
:104F900080903F932F9369817A818B819C81A501B9
:104FA00094010E9480903F932F9387E39BE09F930F
:104FB0008F930E94839B0FB6F894DEBF0FBECDBFC8
:104FC00028960FB6F894DEBF0FBECDBFDF91CF910C
:104FD000FF90EF90DF90CF90BF90AF909F908F9019
:104FE0007F906F905F904F900895E9E0FBE38081A0
:104FF00091818234924479F0E950FB43FF93EF931F
:1050000089E19BE09F938F930E94839B0F900F9069
:105010000F900F9008953A96E53F81E8F80738F32E
:105020000895CF93DF93EC018C9A0E948F109F9389
:105030008F937F936F938DE09BE09F938F930E945C
:10504000839B0F900F900F900F900F900F902097D1
:1050500019F089E992E102C08BE09BE09F938F9366
:105060000E94839B0F900F9081E00E94411020913D
:1050700085023091860240918702509188020E94F9
:1050800024969F938F937F936F938FEF9AE09F93D4
:105090008F930E94839B0F900F900F900F900F9013
:1050A0000F90209719F089E992E102C08DEF9AE004
:1050B0009F938F930E94839B0F900F9082E00E949A
:1050C00041102091810230918202409183025091DF
:1050D00084020E9424969F938F937F936F9381EF16
:1050E0009AE09F938F930E94839B0F900F900F9055
:1050F0000F900F900F90209719F089E992E102C06C
:105100008FEE9AE09F938F930E94839B0F900F9056
:1051100083E00E9441109F938F937F936F9380EE63
:105120009AE09F938F930E94839B8C980F900F908F
:105130000F900F900F900F90209719F089E992E14E
:1051400002C08EED9AE09F938F930E94839B0F90F5
:105150000F908091C52D9091C62D92FF88C021E0BF
:1051600042E161E080ED0E94EA659F938F937F9317
:105170006F9381ED9AE09F938F930E94839B0F9092
:105180000F900F900F900F900F90209719F089E9D2
:1051900092E102C08FEC9AE09F938F930E94839BD1
:1051A0000F900F9021E042E162E080ED0E94EA65FD
:1051B0009F938F937F936F9382EC9AE09F938F934B
:1051C0000E94839B0F900F900F900F900F900F9065
:1051D000209719F089E992E102C080EC9AE09F9350
:1051E0008F930E94839B0F900F9021E042E163E038
:1051F00080ED0E94EA659F938F937F936F9383EB7B
:105200009AE09F938F930E94839B0F900F900F9033
:105210000F900F900F90CD2B19F089E992E102C009
:1052200081EB9AE09F938F930E94839B0F900F9046
:1052300021E042E164E080ED0E94EA659F938F9354
:105240007F936F9384EA9AE09F938F930E94839B4E
:105250000F900F900F900F900F900F9089E992E1AF
:105260009F938F930E94839B0F900F9002C0CD2B32
:10527000A9F3DF91CF9108950F931F93CF93DF93FD
:10528000882389F049E050E06FEF70E08EE896E304
:105290000E94B99A49E050E06EE070E08EE896E333
:1052A0000E943A9E13C0CEE8D6E30FE91AE0899136
:1052B0001F928F931F930F930E94839B0F900F90C9
:1052C0000F900F9086E3C639D80789F789E992E1F4
:1052D0009F938F930E94839B0F900F90DF91CF91AC
:1052E0001F910F910895882311F0299A0895299804
:1052F0000895882311F02A9A08952A980895CF9244
:10530000DF92EF92FF92CF93DF936B017C0160FFFE
:1053100011C08CE194E09F938F9383E992E19F9376
:105320008F930E94839B0F900F900F900F9081E0BE
:1053300090E002C080E090E0C1FE09C0EC0121963F
:1053400043EB59E061E274E00E941E16CE01C2FEFA
:1053500009C0EC01219643EB59E069E274E00E9438
:105360001E16CE01C3FE09C0EC01219643EB59E0A5
:1053700061E374E00E941E16CE01C4FE09C0EC0178
:10538000219643EB59E060EF75E00E941E16CE01B6
:10539000C5FE09C0EC01219643EB59E065E374E0DA
:1053A0000E941E16CE01C6FE09C0EC01219643EBF9
:1053B00059E069E374E00E941E16CE01C7FE09C0E1
:1053C000EC01219643EB59E06FE374E00E941E1656
:1053D000CE01D0FE09C0EC01219643EB59E067E411
:1053E00074E00E941E16CE01D1FE09C0EC01219688
:1053F00043EB59E06FE474E00E941E16CE01D2FE2A
:1054000009C0EC01219643EB59E063E574E00E948A
:105410001E16CE012091C52D3091C62D24703071FD
:10542000232B59F0D3FE09C0EC01219643EB59E040
:1054300069E574E00E941E16CE012091C52D26FF5D
:105440000BC0D4FE09C0EC01219643EB59E06EE598
:1054500074E00E941E16CE012091C52D27FF0BC0BF
:10546000D5FE09C0EC01219643EB59E064E674E0F7
:105470000E941E16CE01D6FE09C0EC01219643EB18
:1054800059E06CE674E00E941E16CE01D7FE09C0FA
:10549000EC01219643EB59E067E774E00E941E1689
:1054A000CE01E0FE0CC043EB59E068E874E0DF9108
:1054B000CF91FF90EF90DF90CF900C941E16CD28E7
:1054C000CE28CF2841F48AE99AE09F938F930E94D7
:1054D000839B0F900F90DF91CF91FF90EF90DF9023
:1054E000CF900895CF92DF92EF92FF92CF93DF9308
:1054F000EC01C12CD12C7601209709F4A3C065E9F9
:105500007AE0CE010E948B9A892B11F46894C0F83E
:105510006DE87AE0CE010E948B9A892B11F4689491
:10552000C1F865E87AE0CE010E948B9A892B11F4CC
:105530006894C2F861E87AE0CE010E948B9A892BC8
:1055400011F46894C3F86EE77AE0CE010E948B9A5A
:10555000892B11F46894C4F86AE77AE0CE010E94BE
:105560008B9A892B11F46894C5F864E77AE0CE0130
:105570000E948B9A892B11F46894C6F86CE67AE045
:10558000CE010E948B9A892B11F46894C7F864E6C7
:105590007AE0CE010E948B9A892B11F46894D0F89E
:1055A00060E67AE0CE010E948B9A892B11F4689410
:1055B000D1F86AE57AE0CE010E948B9A892B11F42A
:1055C0006894D2F865E57AE0CE010E948B9A892B27
:1055D00011F46894D3F86FE47AE0CE010E948B9ABC
:1055E000892B11F46894D4F867E47AE0CE010E9424
:1055F0008B9A892B11F46894D5F86CE37AE0CE018C
:105600000E948B9A892B11F46894D6F86BE27AE0A9
:10561000CE010E948B9A892B11F46894D7F866E228
:105620007AE0CE010E948B9A892B11F46894E0F8FD
:1056300060917E0270917F0280E090E00E949F9ACC
:10564000EC015ACFC701B601DF91CF91FF90EF90E7
:10565000DF90CF900895AF92BF92CF92DF92EF92FA
:10566000FF920F931F93CF93DF93122FD32FC42F4B
:10567000052FF62ED72EE82EC92E217030E040E0FF
:1056800050E060E070E080E090E0A0E00E9488924E
:1056900089F08DE894E09F938F9383E992E19F9343
:1056A0008F930E94839B0F900F900F900F90E1E0DB
:1056B000F0E002C0E0E0F0E08091C52D80FF19C06D
:1056C000212F247030E040E050E060E070E080E0A6
:1056D00090E0A0E00E94889261F05F018FEFA81A2D
:1056E000B80A43EB59E061E974E0CF010E941E164D
:1056F000F501212F227030E040E050E060E070E0E2
:1057000080E090E0A0E00E94889261F05F018FEF5E
:10571000A81AB80A43EB59E065E974E0CF010E948A
:105720001E16F501212F287030E040E050E060E0C7
:1057300070E080E090E0A0E00E94889261F05F015C
:105740008FEFA81AB80A43EB59E06DEA74E0CF0175
:105750000E941E16F501212F207130E040E050E03C
:1057600060E070E080E090E0A0E00E94889261F04C
:105770005F018FEFA81AB80A43EB59E068E974E0BB
:10578000CF010E941E16F501212F207230E040E06B
:1057900050E060E070E080E090E0A0E00E9488923D
:1057A00061F05F018FEFA81AB80A43EB59E06BE98B
:1057B00074E0CF010E941E16F501212F207430E005
:1057C00040E050E060E070E080E090E0A0E00E9407
:1057D000889261F05F018FEFA81AB80A43EB59E095
:1057E00061EA74E0CF010E941E16F501212F207896
:1057F00030E040E050E060E070E080E090E0A0E069
:105800000E94889261F05F018FEFA81AB80A43EBFB
:1058100059E067EA74E0CF010E941E16F50120E00E
:105820003D2F317040E050E060E070E080E090E0BB
:10583000A0E00E94889261F05F018FEFA81AB80A79
:1058400043EB59E06AEA74E0CF010E941E16F501AD
:1058500020E03D2F327040E050E060E070E080E0FA
:1058600090E0A0E00E94889261F05F018FEFA81A9B
:10587000B80A43EB59E06FEA74E0CF010E941E16AC
:10588000F50120E03D2F347040E050E060E070E032
:1058900080E090E0A0E00E94889261F05F018FEFCD
:1058A000A81AB80A43EB59E066EB74E0CF010E94F6
:1058B0001E16F50120E03D2F387040E050E060E01A
:1058C00070E080E090E0A0E00E94889261F05F01CB
:1058D0008FEFA81AB80A43EB59E069EB74E0CF01E7
:1058E0000E941E16F50120E03D2F307140E050E08F
:1058F00060E070E080E090E0A0E00E94889261F0BB
:105900005F018FEFA81AB80A43EB59E06EEB74E021
:10591000CF010E941E16F50120E03D2F307240E0BD
:1059200050E060E070E080E090E0A0E00E948892AB
:1059300061F05F018FEFA81AB80A43EB59E065ECFC
:1059400074E0CF010E941E16F50120E030E040E037
:1059500050E06F2D647070E080E090E0A0E00E9465
:10596000889261F05F018FEFA81AB80A43EB59E003
:105970006CEC74E0CF010E941E16F5018091C52DDC
:1059800081FF19C020E03D2F307440E050E060E01E
:1059900070E080E090E0A0E00E94889261F05F01FA
:1059A0008FEFA81AB80A43EB59E060ED74E0CF011D
:1059B0000E941E16F5018091C52D9091C62D93FF72
:1059C00019C020E030E040E0502F507160E070E0FE
:1059D00080E090E0A0E00E94889261F05F018FEF8C
:1059E000A81AB80A43EB59E063ED74E0CF010E94B6
:1059F0001E16F5018091C52D9091C62D93FF19C0FB
:105A000020E030E040E0502F507260E070E080E035
:105A100090E0A0E00E94889261F05F018FEFA81AE9
:105A2000B80A43EB59E066ED74E0CF010E941E1600
:105A3000F5018091C52D9091C62D93FF19C020E0EE
:105A400030E040E0502F507460E070E080E090E083
:105A5000A0E00E94889261F05F018FEFA81AB80A57
:105A600043EB59E06CED74E0CF010E941E16F50186
:105A700020E03D2F307840E050E060E070E080E0D2
:105A800090E0A0E00E94889261F05F018FEFA81A79
:105A9000B80A43EB59E067EE74E0CF010E941E168E
:105AA000F50120E030E04C2F417050E060E070E004
:105AB00080E090E0A0E00E94889261F05F018FEFAB
:105AC000A81AB80A43EB59E06CEE74E0CF010E94CB
:105AD0001E16F50120E030E04C2F427050E060E0EF
:105AE00070E080E090E0A0E00E94889261F05F01A9
:105AF0008FEFA81AB80A43EB59E06FEE74E0CF01BC
:105B00000E941E16F50120E030E04C2F447050E05A
:105B100060E070E080E090E0A0E00E94889261F098
:105B20005F018FEFA81AB80A43EB59E062EF74E007
:105B3000CF010E941E16F50120E030E040E050E069
:105B40006F2D687070E080E090E0A0E00E94889285
:105B500061F05F018FEFA81AB80A43EB59E065EFD7
:105B600074E0CF010E941E16F50120E030E040E015
:105B700050E06F2D607170E080E090E0A0E00E9446
:105B8000889261F05F018FEFA81AB80A43EB59E0E1
:105B900069EF74E0CF010E941E16F5018091C52DBA
:105BA0009091C62D92FF19C020E030E04C2F487034
:105BB00050E060E070E080E090E0A0E00E94889219
:105BC00061F05F018FEFA81AB80A43EB59E06DEF5F
:105BD00074E0CF010E941E16F5018091C52D9091B1
:105BE000C62D92FF19C020E030E04C2F407150E0EC
:105BF00060E070E080E090E0A0E00E94889261F0B8
:105C00005F018FEFA81AB80A43EB59E061E075E035
:105C1000CF010E941E16F5018091C52D9091C62DD1
:105C200092FF19C020E030E04C2F407250E060E05D
:105C300070E080E090E0A0E00E94889261F05F0157
:105C40008FEFA81AB80A43EB59E065E075E0CF0181
:105C50000E941E16F5018091C52D9091C62D92FFD0
:105C600019C020E030E04C2F407450E060E070E05C
:105C700080E090E0A0E00E94889261F05F018FEFE9
:105C8000A81AB80A43EB59E069E075E0CF010E9419
:105C90001E16F5018091C52D82FF19C020E030E06D
:105CA0004C2F407850E060E070E080E090E0A0E0B1
:105CB0000E94889261F05F018FEFA81AB80A43EB47
:105CC00059E06DE776E0CF010E941E16F501809144
:105CD000C52D82FF19C020E030E040E0502F517008
:105CE00060E070E080E090E0A0E00E94889261F0C7
:105CF0005F018FEFA81AB80A43EB59E06DE075E039
:105D0000CF010E941E16F5018091C52D9091C62DE0
:105D100093FF19C020E030E040E0502F527060E067
:105D200070E080E090E0A0E00E94889261F05F0166
:105D30008FEFA81AB80A43EB59E060E175E0CF0194
:105D40000E941E16F5018091C52D9091C62D93FFDE
:105D500019C020E030E040E0502F547060E070E067
:105D600080E090E0A0E00E94889261F05F018FEFF8
:105D7000A81AB80A43EB59E068E175E0CF010E9428
:105D80001E16F5018091C52D9091C62D94FF19C066
:105D900020E030E040E0502F587060E070E080E09C
:105DA00090E0A0E00E94889261F05F018FEFA81A56
:105DB000B80A43EB59E061E275E0CF010E941E167C
:105DC000F5018091C52D85FF19C020E030E040E04D
:105DD00050E06F2D607270E080E090E0A0E00E94E3
:105DE000889261F05F018FEFA81AB80A43EB59E07F
:105DF0006AE275E0CF010E941E16F5018091C52D63
:105E000085FF19C020E030E040E050E06F2D607465
:105E100070E080E090E0A0E00E94889261F05F0175
:105E20008FEFA81AB80A43EB59E063E375E0CF019E
:105E30000E941E16F5018091C52D85FF1EC020E031
:105E400030E040E050E06F2D607870E080E090E05E
:105E5000A0E00E94889289F043EB59E06DE375E081
:105E6000CF01DF91CF911F910F91FF90EF90DF90C5
:105E7000CF90BF90AF900C941E16212F3D2F4C2F2A
:105E8000502F6F2D7D2D8E2D9C2DA0E00E9488928D
:105E900041F481E29AE09F938F930E94839B0F903D
:105EA0000F90DF91CF911F910F91FF90EF90DF90B6
:105EB000CF90BF90AF900895AF92BF92DF92EF92D4
:105EC000FF920F931F93CF93DF93EC015B01FB01D4
:105ED00010826CE17AE00E948B9A892B89F580917F
:105EE000C52D1DE440E8F42E82FF03C034E8E32E04
:105EF00002C024E0E22E00E0D12C81FF02C090EC31
:105F0000F92E26E04AE250E06BE270E089E290E090
:105F10000E94CE6181E090E00E94381181111DE560
:105F20008091C52D9091C62D93FF02C0177F06E08A
:105F300094FD086085FF09C0177F80EED82E05C04C
:105F400010E0F12CE12C00E0D12C6AE17AE0CE01E6
:105F50000E948B9A892B61F481E0F5018083609126
:105F60007E0270917F0280E090E00E949F9AEC0197
:105F700068E17AE0CE010E948B9A892B61F48FEF61
:105F8000F501808360917E0270917F0280E090E055
:105F90000E949F9AEC01209709F456C164E17AE0CF
:105FA000CE010E948B9A892B09F4116060E17AE09E
:105FB000CE010E948B9A892B09F414606DE07AE07F
:105FC000CE010E948B9A892B09F412606BE07AE073
:105FD000CE010E948B9A892B09F4186068E07AE060
:105FE000CE010E948B9A892B09F4106162E07AE05D
:105FF000CE010E948B9A892B09F410626CEF79E034
:10600000CE010E948B9A892B09F4106469EF79E024
:10601000CE010E948B9A892B09F4106864EF79E015
:10602000CE010E948B9A892B19F4FF2DF160FF2E6F
:106030006DEE79E0CE010E948B9A892B19F48F2D99
:106040008260F82E6AEE79E0CE010E948B9A892B4D
:1060500019F4EF2DE460FE2E65EE79E0CE010E948A
:106060008B9A892B19F4FF2DF860FF2E6EED79E0E5
:10607000CE010E948B9A892B19F48F2D8061F82E06
:1060800067ED79E0CE010E948B9A892B19F4EF2DF0
:10609000E062FE2E63ED79E0CE010E948B9A892B9F
:1060A00019F4FD2DF460DF2E60ED79E0CE010E9441
:1060B0008B9A892B19F48F2D8064F82E6BEC79E084
:1060C000CE010E948B9A892B19F4EF2DE068FE2EE9
:1060D00068EC79E0CE010E948B9A892B19F4FE2D91
:1060E000F160EF2E65EC79E0CE010E948B9A892B4E
:1060F00019F48E2D8260E82E62EC79E0CE010E94C8
:106100008B9A892B19F4EE2DE460EE2E6EEB79E07C
:10611000CE010E948B9A892B19F4FE2DF860EF2E88
:106120006AEB79E0CE010E948B9A892B19F48E2DAF
:106130008061E82E66EB79E0CE010E948B9A892B74
:1061400019F4EE2DE062EE2E62EB79E0CE010E94B2
:106150008B9A892B19F4FE2DF064EF2E60EB79E019
:10616000CE010E948B9A892B19F48E2D8068E82E1F
:106170006DEA79E0CE010E948B9A892B09F40160C7
:1061800065EA79E0CE010E948B9A892B09F40260BE
:106190006CE979E0CE010E948B9A892B09F40460A6
:1061A00063E979E0CE010E948B9A892B09F408609B
:1061B00060E979E0CE010E948B9A892B09F4006195
:1061C0006AE879E0CE010E948B9A892B09F400627B
:1061D0006FE779E0CE010E948B9A892B09F4006465
:1061E0006BE779E0CE010E948B9A892B19F4ED2D93
:1061F000E860DE2E67E779E0CE010E948B9A892B5A
:1062000019F4FD2DF061DF2E6EE679E0CE010E94DB
:106210008B9A892B19F48D2D8062D82E64E679E053
:10622000CE010E948B9A892B19F4ED2DE064DE2EAD
:106230006BE579E0CE010E948B9A892B09F0A2CE02
:10624000FD2DF068DF2E9ECE212F3F2D4E2D502F9D
:106250006D2D70E080E090E0DF91CF911F910F9164
:10626000FF90EF90DF90BF90AF9008953F924F92D4
:106270005F926F927F928F929F92AF92BF92CF92D6
:10628000DF92EF92FF920F931F93CF93DF93582EDD
:10629000C8EADDE100E010E085E5E82E89E0F82EAF
:1062A000852D8170382E852D8270482E90E4C92E60
:1062B00099E0D92E28E4A22E29E0B22E36E4832ECE
:1062C00039E0932E49E9642E42E1742E552051F0B5
:1062D0001F930F93FF92EF920E94839B0F900F905A
:1062E0000F900F903320A1F089858F9388858F932D
:1062F000BF92AF920E94839B0F900F900F900F90D0
:106300004420C1F09F928F920E94839B0F900F9028
:10631000442081F0DF92CF920E94839B28813981B3
:106320004A815B816C817D818E819F810E942B2BB4
:106330000F900F907F926F920E94839B0F5F1F4F71
:106340002A960F900F900430110509F0BFCFDF910E
:10635000CF911F910F91FF90EF90DF90CF90BF9062
:10636000AF909F908F907F906F905F904F903F90F5
:1063700008958BE399E09F938F930E94839B809174
:10638000B5299091B629A091B729B091B8290F905D
:106390000F90813027EA92072EE1A207B10519F488
:1063A0008DE299E01DC0823026EA92072EE1A20715
:1063B000B10519F480E299E013C0823027EA920710
:1063C0002EE1A207B10519F482E199E009C08230FB
:1063D00028EA92072EE1A207B10549F484E099E08A
:1063E0009F938F930E94839B0F900F900895BF936C
:1063F000AF939F938F938EEF98E09F938F930E941C
:10640000839B0F900F900F900F900F900F90089517
:106410008EEE98E09F938F930E94839B0E94572754
:106420000E94B93189E992E19F938F930E94839BE7
:106430008FE89DE19F938F9386EE98E09F938F93D3
:106440000E94839B60916002709161028091620260
:106450009091630228EE33E040E050E00E9480908B
:106460005F934F933F932F9386ED98E09F938F9385
:106470000E94839B8DEC98E09F938F930E94839B57
:106480000E9488168091C52D2DB73EB7205F3F4FE3
:106490000FB6F8943EBF0FBE2DBF80FF05C041E090
:1064A00061E081E00E94641889EC98E09F938F93EB
:1064B0000E94839B80E00E943C290E945B27809180
:1064C00065021F928F9380EC98E09F938F930E94B8
:1064D000839B80917A141F928F9387EB98E09F9310
:1064E0008F930E94839B809190028F9380918F0263
:1064F0008F9380918E028F9380918D028F9389EA82
:1065000098E09F938F930E94839B1F9280E48F93C8
:1065100081E998E09F938F930E94839B8091E83854
:106520001F928F938091E7381F928F938EE798E0A8
:106530009F938F930E94839B809164021F928F93FD
:1065400085E798E09F938F930E94839B80916602DA
:1065500090916702A0916802B09169022DB73EB791
:10656000225E3F4F0FB6F8943EBF0FBE2DBF96FD83
:1065700003C089E495E002C086E495E09F938F9381
:106580008BE698E09F938F930E94839B83E00E9409
:1065900036310F900F900F900F901D9903C089E432
:1065A00095E002C086E495E09F938F938FE598E095
:1065B0009F938F930E94839B85E598E09F938F9391
:1065C0000E94839B809166020F900F900F900F9016
:1065D0000F900F9081FF09C08FE498E09F938F93F5
:1065E0000E94839B0F900F9013C080FD03C089E42D
:1065F00095E002C086E495E09F938F938BE498E04A
:106600009F938F930E94839B0F900F900F900F90FA
:106610008091660290916702A0916802B091690230
:1066200097FD03C089E495E002C086E495E09F935E
:106630008F9382E498E09F938F930E94839B8BE3D8
:1066400098E09F938F930E94839B60917D1470913B
:106650007E1480917F14909180140E947F2989E993
:1066600092E19F938F930E94839B8DB79EB708966C
:106670000FB6F8949EBF0FBE8DBF779B03C089E411
:1066800095E002C086E495E09F938F9382E398E0C3
:106690009F938F930E94839B0E94230E0E94F4106D
:1066A0009F938F937F936F9384E298E09F938F9350
:1066B0000E94839B0E94A3109F938F937F936F935D
:1066C00086E198E09F938F930E94839B81E090E006
:1066D0000E9411288091743690917536A09176367B
:1066E000B0917736BF93AF939F938F9388E098E0F4
:1066F0009F938F930E94839B809189368F93809183
:1067000088368F93809187368F93809186368F93CA
:1067100084EF97E09F938F930E94839B80917836BC
:1067200090917936A0917A36B0917B36BF93AF9332
:106730009F938F9386EE97E09F938F930E94839B06
:106740002DB73EB72E5D3F4F0FB6F8943EBF0FBE3C
:106750002DBF80918D368F9380918C368F93809151
:106760008B368F9380918A368F9382ED97E09F933B
:106770008F930E94839B61E070E080E090E00E9434
:10678000A71161E070E081E090E00E94A7110F90F6
:106790000F900F900F900F900F90299903C089E4EC
:1067A00095E002C086E495E09F938F938AEC97E092
:1067B0009F938F930E94839B0F900F900F900F9049
:1067C0002A9903C089E495E002C086E495E09F938E
:1067D0008F9382EC97E09F938F930E94839B80918D
:1067E000660290916702A0916802B09169020F90D1
:1067F0000F900F900F9094FD03C089E495E002C0C4
:1068000086E495E09F938F938AEB97E09F938F9315
:106810000E94839B8091C52D0F900F900F900F9039
:1068200085FF5FC081E00E94836860919936709116
:106830009A3680919B3690919C360E942C9420E051
:1068400030E048EC52E40E9478939F938F937F93BB
:106850006F938DE495E09F938F930E946F9B60915F
:106860009D3670919E3680919F369091A0360E9401
:106870002A9420E030E040E85AE30E9424969F9357
:106880008F937F936F938CE595E09F938F930E94F6
:106890006F9B6091A1367091A2368091A336909142
:1068A000A4360E942A9420E030E040E85BE30E9496
:1068B00024969F938F937F936F938DE695E09F939C
:1068C0008F930E946F9B89E992E19F938F930E941F
:1068D000839B8DB79EB744960FB6F8949EBF0FBEAC
:1068E0008DBF0895F89491E2E0E0F0E090935700B6
:1068F0008491E2E0F0E0909357002491E4E0F0E02E
:1069000090935700E49190E0A0E0B0E0BC015527DF
:106910004427822F90E0A0E0B0E0BA2FA92F982F53
:106920008827840F951FA61FB71F8E0F911DA11DCD
:10693000B11D8093B5299093B629A093B729B09340
:10694000B82978940895CF93DF93CDB7DEB76197D8
:106950000FB6F894DEBF0FBECDBF48E250E062E252
:1069600070E088EA9DE10E941C9E2091A81D309154
:10697000A91D4091AA1D5091AB1D6091AC1D709155
:10698000AD1D8091AE1D9091AF1DAFEF0E9488921A
:1069900091F58DE48093A81D80E88093A91D84E083
:1069A0008093AA1D1092AB1D1092AC1D1092AD1DCC
:1069B0001092AE1D1092AF1D8CE390E09093B11D2C
:1069C0008093B01DE8EAFDE11286138614861586D1
:1069D00016861786108A118A138A128A3A962DE132
:1069E000E63CF20789F748E250E062E270E088EAAC
:1069F0009DE10E943A9E44E050E06EE170E0CE01DD
:106A00000B960E941C9E8B859C85AD85BE858F3F15
:106A10002FEF9207A207B207A9F48AE090E4A0E062
:106A2000B0E08093660290936702A0936802B093EF
:106A3000690244E050E06EE170E086E692E00E9478
:106A40003A9E08C08093660290936702A093680202
:106A5000B09369028091660290916702A0916802EA
:106A6000B0916902A2FF02C02A9A03C080E00E948E
:106A7000792944E050E06AE570E0CE010B960E946F
:106A80001C9E8B859C85AD85BE858F3F2FEF920721
:106A9000A207B20789F410927D1410927E1410920E
:106AA0007F141092801444E050E06AE570E08DE7B6
:106AB00094E10E943A9E08C080937D1490937E14C6
:106AC000A0937F14B093801449E050E06EE070E032
:106AD0008EE896E30E941C9E0E94EE1244E050E075
:106AE0006EE470E0CE010B960E941C9E8B859C8507
:106AF000AD85BE8544E050E06EE470E08F3F9F4F6F
:106B0000AF4FBF4F29F485E892E00E943A9E04C03F
:106B100085E892E00E941C9E44E050E06AE470E048
:106B2000CE010B960E941C9E8B859C85AD85BE85F3
:106B300044E050E06AE470E08F3F9F4FAF4FBF4F9B
:106B400029F481E892E00E943A9E04C081E892E034
:106B50000E941C9E44E050E062E570E0CE010B967E
:106B60000E941C9E8B859C85AD85BE8544E050E0CF
:106B700062E570E08F3F9F4FAF4FBF4F29F489E828
:106B800092E00E943A9E04C089E892E00E941C9E16
:106B900041E050E06DE170E0CE0141960E941C9E04
:106BA000898941E050E06DE170E08F3F29F48AE788
:106BB00094E10E943A9E04C08AE794E10E941C9EE0
:106BC00041E050E06CE170E0CE0141960E941C9ED5
:106BD000898941E050E06CE170E08F3F29F485E65F
:106BE00092E00E943A9E04C085E692E00E941C9EBC
:106BF00041E050E06BE170E0CE0141960E941C9EA6
:106C0000898941E050E06BE170E08F3F29F484E630
:106C100092E00E943A9E04C084E692E00E941C9E8C
:106C20004AE050E064E070E0CE0101960E941C9EB4
:106C300089814AE050E064E070E08F3F29F48FE8FA
:106C40009DE10E943A9E04C08FE89DE10E941C9E37
:106C500044E050E066E570E0CE010B960E941C9E79
:106C60008B859C85AD85BE8544E050E066E570E08F
:106C70008F3F9F4FAF4FBF4F29F48DE892E00E94A6
:106C80003A9E04C08DE892E00E941C9E44E050E0D1
:106C900067E170E0CE010B960E941C9E8B859C855F
:106CA000AD85BE8544E050E067E170E08F3F9F4FC7
:106CB000AF4FBF4F29F480E692E00E943A9E04C095
:106CC00080E692E00E941C9E809160029091610299
:106CD000A0916202B091630281389A41A640B10549
:106CE000A0F088E294E09F938F930E94839B80E1C1
:106CF00097E2A0E0B0E08093600290936102A093DD
:106D00006202B09363020F900F90609160027091E5
:106D1000610280916202909163020E940D6442E0E0
:106D200050E062E070E0CE010F960E941C9E8F85BD
:106D3000988942E050E062E070E08F3F910529F4CD
:106D400083E794E10E943A9E04C083E794E10E94A5
:106D50001C9E42E050E060E070E0CE010F960E9481
:106D60001C9E8F85988942E050E060E070E08F3F84
:106D7000910529F481E794E10E943A9E04C081E7DD
:106D800094E10E941C9E61960FB6F894DEBF0FBE80
:106D9000CDBFDF91CF910895CF92DF92EF92FF9216
:106DA00060917E0270917F0280E090E00E949F9A45
:106DB0006DE775E00E94C09A892B09F010C18DE43F
:106DC0008093A81D80E88093A91D84E08093AA1D6C
:106DD0001092AB1D1092AC1D1092AD1D1092AE1D05
:106DE0001092AF1D8CE390E09093B11D8093B01D85
:106DF000E8EAFDE112861386148615861686178644
:106E0000108A118A138A128A3A968DE1E63CF807B5
:106E100089F748E250E062E270E088EA9DE10E9472
:106E20003A9E8AE090E4A0E0B0E0809366029093FE
:106E30006702A0936802B093690244E050E06EE1FB
:106E400070E086E692E00E943A9E10927D141092C5
:106E50007E1410927F141092801444E050E06AE592
:106E600070E08DE794E10E943A9E82E2C82EDD2414
:106E7000DA948CECE82E8BE3F82EC0928502D09247
:106E80008602E0928702F092880244E050E06EE4CD
:106E900070E085E892E00E943A9EC0928102D09212
:106EA0008202E0928302F092840244E050E06AE4BD
:106EB00070E081E892E00E943A9E87ED94E3AFEEA5
:106EC000BCE38093890290938A02A0938B02B093D3
:106ED0008C0244E050E062E570E089E892E00E94B4
:106EE0003A9E8AE999E9A9E1B0E480938D029093F2
:106EF0008E02A0938F02B093900244E050E066E5CA
:106F000070E08DE892E00E943A9E10927A1480E040
:106F10000E94F27241E050E06DE170E08AE794E196
:106F20000E943A9E8AE1809365020E94DF7141E0EF
:106F300050E06CE170E085E692E00E943A9E8FE0BE
:106F40008093640241E050E06BE170E084E692E0FF
:106F50000E943A9E8AE0EFE8FDE1DF011D928A95EA
:106F6000E9F74AE050E064E070E0CF010E943A9E09
:106F700080E197E2A0E0B0E080936002909361022C
:106F8000A0936202B093630244E050E067E170E0D6
:106F900080E692E00E943A9E10927414109273144C
:106FA00042E050E062E070E083E794E10E943A9EA4
:106FB000109272141092711442E050E060E070E0A0
:106FC00081E794E10E943A9E81E00E943C2980E0A2
:106FD00090E0FF90EF90DF90CF900C940313FF9020
:106FE000EF90DF90CF9008950E94006F6C9A6B9A9B
:106FF0006A9A6F9A729A749A739A779A809880B301
:10700000897F80BB8398849887E080937E00549A20
:107010000E9472340E94A3348091660290916702AC
:10702000A0916802B091690294FD0E940F6F0E94C6
:10703000910E80E090E00E940313609160027091D5
:10704000610280916202909163020E940D640E942D
:10705000A3106093C7317093C8318093C931909366
:10706000CA318091660286FD239A219A229A239A38
:107070000E94A60E1D9B05C010927C1410927B14DA
:10708000089581E090E090937C1480937B140895A0
:10709000CF93DF9390E040917D1450917E146091E6
:1070A0007F147091801441FD08C02091660220FD7C
:1070B00004C021FF92C01D9B90C02DE8289FE001D5
:1070C000299FD00D1124CE018B54914E9F938F9305
:1070D00084E895E09F938F930E946F9BFE01E25599
:1070E000F14EDF01AA57BF4F2C910F900F900F90D8
:1070F0000F9043815481658176818091CB3190914D
:10710000CC31A091CD31B091CE31841B950BA60B23
:10711000B70B2223D1F1BF93AF939F938F93DF01DE
:10712000A257BF4F11968C9111978F938C918F938B
:10713000129711968C9111978F938C918F9313972F
:107140008C911F928F9311978C911F928F9313960E
:107150008C911F928F9311978C911F928F93E95767
:10716000FF4F80811F928F931F922F938AE895E0A3
:107170009F938F930E946F9B8DB79EB746960FB6D5
:10718000F8949EBF0FBE8DBF10C0BF93AF939F9367
:107190008F9381ED95E09F938F930E946F9B0F904B
:1071A0000F900F900F900F900F9089E992E19F93AD
:1071B0008F930E94839B809180020F900F90882371
:1071C00061F01F928F9385E294E09F938F930E94CA
:1071D000839B0F900F900F900F90DF91CF910895A8
:1071E0008091AE1E882341F08091AF1E90E00E94F6
:1071F00048380E94970FF4CF0895CF93DF93EC01A6
:10720000888199818E332FE09207F1F018F4892B51
:10721000C1F04BC086342FE0920709F44CC08A3489
:107220009F4009F042C084E39BE00E946F76892B67
:1072300009F43FC084E39BE00E945B7680E00E94FB
:1072400073298EE39FE02EC0623199F5299A40910F
:107250007114509172145695542F442757954795A1
:1072600060E070E084E39BE00E94517680917D14A1
:1072700090917E14A0917F14B0918014A0FF10C053
:10728000809172148F93809171148F9388E393E1AE
:107290009F938F930E94839B0F900F900F900F905E
:1072A00086E49FE09983888304C01982188283E072
:1072B00019C081E017C084E39BE00E946F76892BA0
:1072C000C1F384E39BE00E945B760E94F03840E2C9
:1072D00050E060E070E084E39BE00E9451768AE435
:1072E0009FE0E0CFDF91CF9108952F923F924F9290
:1072F0005F926F927F928F929F92AF92BF92CF9246
:10730000DF92EF92FF920F931F93CF93DF93CDB74E
:10731000DEB72B970FB6F894DEBF0FBECDBF9B87AD
:107320008A873A01FC0180819181892B11F00C94AC
:10733000A04E60917E0270917F02CA010E949F9AC6
:1073400060E870E0C3010E94DF9A009759F46091F1
:10735000033B7091043B8AE090E00E94339B81E004
:107360000C94A54E8130910561F4F3011081912EAA
:10737000990C9908892CE92CF92C092D492C592CA8
:10738000C0C082309105B9F4F3018081082E000C51
:10739000990B982F88272181820F911D27FD9A959F
:1073A000182F992E892E880C8808E82CF82C082D87
:1073B000482C582CA6C083309105C1F5F3012081DB
:1073C000922F990F990B392F492F592F692F792F08
:1073D000892F00E10E942A9229014A01B62FA72F86
:1073E000382E292E2181922F990F990B392F492F51
:1073F000592F692F792F892F08E00E942A9259016D
:107400006A017B018C019201A4016B2F7A2F832DDD
:10741000922D0E946192A2801A2D110F110BB12E94
:10742000C12ED12EE12EF12E012F59C004970CF45C
:1074300060C0F3012081922F990F990B392F492FAA
:10744000592F692F792F892F08E10E942A9229014B
:107450004A01B62FA72F382E292E2181922F990F5E
:10746000990B392F492F592F692F792F892F00E137
:107470000E942A9259016A017B018C019201A401A8
:107480006B2F7A2F832D922D0E946192A3801A2D4B
:10749000110F110BB12EC12ED12EE12EF12E012F85
:1074A0000E94619229014A01B62FA72F382E292E5A
:1074B0002281922F990F990B392F492F592F692F1C
:1074C000792F892F08E00E942A9259016A017B01D5
:1074D0008C019201A4016B2F7A2F832D922D0E9493
:1074E0006192122F932E842EE52EF62E072F2C015B
:1074F00008C01AE0912C812CE12CF12C00E0412CE9
:10750000512C39E9232E32E1332E3F922F920E94E3
:10751000839B0F900F90212F392D482D5E2D6F2DBD
:10752000702FC2012537F3E63F07FDE64F075105EF
:10753000610571058105910511F40C94D748253733
:10754000E3E63E07EDE64E0751056105710581054D
:10755000910511F008F0B9C12337F2E73F07410563
:107560005105610571058105910511F40C94844B59
:107570002337E2E73E0741055105610571058105A5
:10758000910511F008F0BCC02536F4E63F0741052F
:107590005105610571058105910509F4FAC7253684
:1075A000E4E63E0741055105610571058105910538
:1075B00011F008F042C0A6E70E94889211F40C94E2
:1075C00057450E94889209F070F4A8E60E948892BC
:1075D00011F40C942643A5E70E94889211F40C94B0
:1075E00041450C949E4E212F392D482D5E2D6F2D37
:1075F000702FC2012436F1E63F07410551056105B0
:1076000071058105910511F40C94AC4B2537E2E628
:107610003E0741055105610571058105910509F494
:1076200048C52A333642410551056105710581057A
:10763000910509F43EC30C949E4E212F392D482DFF
:107640005E2D6F2D702FC2012737EFE63E074105F3
:107650005105610571058105910511F40C944149AD
:107660002737FFE63F074105510561057105810593
:10767000910509F0C8F42436E9E63E0741055105B5
:10768000610571058105910511F40C941A452536A3
:107690003E4641055105610571058105910511F4CD
:1076A0000C9479490C949E4E212F392D482D5E2D36
:1076B0006F2D702FC2012536E2E73E0741055105C7
:1076C000610571058105910511F40C94454A29362F
:1076D000F2E73F07410551056105710581059105F7
:1076E00011F40C94334B23333147410551056105A7
:1076F00071058105910511F00C949E4E0C94AC4BD4
:10770000212F392D482D5E2D6F2D702FC20122366D
:10771000F5E63F07F4E64F07510561057105810560
:10772000910509F436C72236E5E63E07E4E64E0742
:107730005105610571058105910511F008F05CC0E6
:107740002133F4E63F07F1E64F0751056105710566
:107750008105910509F4C1C22133E4E63E07E1E663
:107760004E075105610571058105910509F0C0F4C9
:107770002337F3E73F074105510561057105810591
:10778000910511F40C94984B283734474105510565
:10779000610571058105910509F48BC20C949E4E1B
:1077A000212F392D482D5E2D6F2D702FC2012837C6
:1077B000F4E63F07F1E64F075105610571058105C4
:1077C000910509F486C22C36E5E73E07E2E64E074E
:1077D0005105610571058105910509F46AC42336D7
:1077E000344641465105610571058105910511F049
:1077F0000C949E4E0C94AC4B212F392D482D5E2DB0
:107800006F2D702FC2012D36E5E73E07E8E64E07E3
:107810005105610571058105910511F40C94C24B68
:107820002D36F5E73F07F8E64F075105610571056D
:107830008105910509F0E0F42237E2E73E07E5E62D
:107840004E075105610571058105910511F40C94F0
:10785000844823363D46484651056105710581053A
:10786000910511F00C949E4E0E94AF1C0C94A04EFA
:10787000212F392D482D5E2D6F2D702FC2012436FA
:10788000E3E63E07ECE64E0751056105710581050B
:10789000910511F40C94E7472736FFE63F07FCE615
:1078A0004F075105610571058105910511F40C948F
:1078B000EA47233632434946510561057105810582
:1078C000910511F00C949E4E28C2212F392D482D80
:1078D0005E2D6F2D702FC2012037FCE63F07F5E6C5
:1078E0004F07F8E65F07610571058105910509F409
:1078F000ADC62037ECE63E07E5E64E07E8E65E0754
:10790000610571058105910511F008F0E3C0243788
:10791000F8E73F07F4E74F07510561057105810559
:10792000910511F40C94C3452437E8E73E07E4E7DA
:107930004E075105610571058105910511F008F0AB
:107940005EC02033F1E33F07F1E74F0751056105C2
:1079500071058105910511F40C9484482033E1E30D
:107960003E07E1E74E075105610571058105910567
:1079700009F0C0F42133F2E63F07F0E74F07510565
:10798000610571058105910509F4A8C222333246CB
:1079900040475105610571058105910509F4F3C260
:1079A0000C949E4E212F392D482D5E2D6F2D702F5A
:1079B000C2012037F5E63F07F2E74F0751056105A1
:1079C00071058105910511F40C94454A2C36E4E7C4
:1079D0003E074E075105610571058105910511F4BA
:1079E0000C94B54D21333143414751056105710573
:1079F0008105910511F00C949E4E0C94D748212FCF
:107A0000392D482D5E2D6F2D702FC2012B36ECE6DF
:107A10003E07E5E74E07E2E65E0761057105810571
:107A2000910509F446C32B36FCE63F07F5E74F07FF
:107A3000F2E65F07610571058105910509F0E0F443
:107A40002437E4E63E07E7E74E0751056105710577
:107A50008105910511F40C94094E24373F464F4699
:107A60005246610571058105910511F00C949E4EF9
:107A70000C9400000C94A04E212F392D482D5E2D22
:107A80006F2D702FC2012E36E1E63E07E8E64E0765
:107A9000E3E65E07610571058105910511F40C941B
:107AA00097452633F9E63F07F5E74F07F5E65F0709
:107AB000610571058105910509F4CCC529363C465F
:107AC00041465346610571058105910511F00C94FD
:107AD0009E4E99C3212F392D482D5E2D6F2D702F6D
:107AE000C2012437F3E73F07F5E64F07F2E75F07E8
:107AF000610571058105910511F40C94F549243750
:107B0000E3E73E07E5E64E07E2E75E07610571053C
:107B10008105910511F008F063C02337F5E63F07B2
:107B2000F2E74F07F0E75F076105710581059105F1
:107B300011F40C947E4C2337E5E63E07E2E74E074E
:107B4000E0E75E07610571058105910509F0D0F454
:107B50002136FDE63F07F5E74F07F8E65F076105C9
:107B600071058105910511F40C945F49223737475F
:107B700040475047610571058105910509F468C2C8
:107B80000C949E4E212F392D482D5E2D6F2D702F78
:107B9000C2012436FDE63F07F3E64F07F2E75F0731
:107BA000610571058105910509F45FC62136ECE692
:107BB0003E07E5E64E07E2E75E07610571058105D0
:107BC000910509F464C5233732474747504761059B
:107BD00071058105910511F00C949E4E0C94F849A5
:107BE000212F392D482D5E2D6F2D702FC201243786
:107BF000E2E73E07E1E64E07E5E75E07610571054E
:107C00008105910509F48CC62437F2E73F07F1E6B8
:107C10004F07F5E75F07610571058105910509F0DB
:107C2000C8F42437E3E73E07E5E64E07E4E75E07DE
:107C3000610571058105910509F4D0C727373047E3
:107C400048475447610571058105910509F445C709
:107C50000C949E4E212F392D482D5E2D6F2D702FA7
:107C6000C2012F36ECE63E07EFE54E07E6E75E077A
:107C7000610571058105910509F4A2C52C36F1E66F
:107C80003F07F4E74F07F8E75F07610571058105D6
:107C9000910511F40C947C4D2237374640475547E7
:107CA000610571058105910511F00C949E4E0C94AF
:107CB000C34783E080937C3610927E3610927D36E7
:107CC0004CE756E362E182E492E00E949E780C94D5
:107CD000A04E0E94441C0C94A04E21E042E161E0C1
:107CE00080ED0E94EA6521E042E161E080ED0E94C2
:107CF000EA6521E042E161E080ED0E94EA6521E071
:107D000042E161E080ED0E94EA6521E042E161E04C
:107D100080ED0E94EA650C94A04E60917E02709105
:107D20007F0280E090E00E949F9A6DED75E00E94D6
:107D3000C09A892B09F0CEC060917E0270917F02BB
:107D400080E090E00E949F9A8C01009709F49DC00A
:107D500062E773E00E94C09A892BE1F488EE93E019
:107D6000A0E0B0E08093600290936102A093620271
:107D7000B093630268EE73E080E090E00E940D64CF
:107D800044E050E067E170E080E692E00E943A9EB5
:107D90000C94A04E63EE75E0C8010E94C09A892B36
:107DA000E1F480E197E2A0E0B0E08093600290937C
:107DB0006102A0936202B093630260E177E280E027
:107DC00090E00E940D6444E050E067E170E080E6DE
:107DD00092E00E943A9E0C94A04E66EE75E0C801B7
:107DE0000E94C09A892BE1F480EA96E8A1E0B0E015
:107DF0008093600290936102A0936202B093630249
:107E000060EA76E881E090E00E940D6444E050E092
:107E100067E170E080E692E00E943A9E0C94A04EEA
:107E20006AEE75E0C8010E94C09A892BE1F480E8EF
:107E30009AE1A6E0B0E08093600290936102A09383
:107E40006202B093630260E87AE186E090E00E940B
:107E50000D6444E050E067E170E080E692E00E944B
:107E60003A9E0C94A04E84EE95E09F938F930E94CF
:107E7000839B89E992E19F938F930E94839B0F904C
:107E80000F900F900F900C94A04E60916002709133
:107E90006102809162029091630228EE33E040E03B
:107EA00050E00E9480905F934F933F932F9380EE1A
:107EB00095E09F938F930E94839B89E992E19F9322
:107EC0008F930E94839B0FB6F894DEBF0FBECDBF89
:107ED0000C94A04E0E9488160C94A04E60917E02D5
:107EE00070917F0280E090E00E949F9A8C0166E48E
:107EF00075E00E94C09A892BA1F48091660290914E
:107F00006702A0916802B0916902A2608093660244
:107F100090936702A0936802B0936902299A0C9427
:107F2000A04E69E475E0C8010E94C09A892BB1F4A3
:107F30008091660290916702A0916802B0916902F7
:107F4000AD7F8093660290936702A0936802B0931E
:107F5000690280E00E9473290C94A04E299B03C003
:107F600086E495E002C089E495E09F938F9388EDC5
:107F700095E09F938F930E94839B0F900F900F909B
:107F80000F900C94A04E60917E0270917F0280E071
:107F900090E00E949F9A8C0166E475E00E94C09A6E
:107FA000892BE1F48091660290916702A0916802AA
:107FB000B0916902A4608093660290936702A093D7
:107FC0006802B09369022A9A44E050E06EE170E0E2
:107FD00086E692E00E943A9E0C94A04E69E475E019
:107FE000C8010E94C09A892BF1F480916602909199
:107FF0006702A0916802B0916902AB7F809366022C
:1080000090936702A0936802B093690280E00E9497
:10801000792944E050E06EE170E086E692E00E944B
:108020003A9E0C94A04E2A9B03C086E495E002C0C1
:1080300089E495E09F938F9380ED95E09F938F93D4
:108040000E94839B0F900F900F900F900C94A04E66
:1080500060917E0270917F0280E090E00E949F9A82
:108060008C0166E475E00E94C09A892B19F4779818
:108070000C94A04E69E475E0C8010E94C09A892B57
:1080800019F4779A0C94A04E779903C086E495E092
:1080900002C089E495E09F938F9384EA97E09F93D1
:1080A0008F930E94839B0F900F900F900F900C94D2
:1080B000A04E60917E0270917F0280E090E00E946D
:1080C0009F9A8C016EEE75E00E94C09A892BD1F4C4
:1080D0008091AE1E1F928F938091B01E1F928F933E
:1080E0008091AF1E1F928F931F9284E18F9386EA37
:1080F00095E09F938F930E94839B0FB6F894DEBF09
:108100000FBECDBF63EF75E0C8010E94C09A892BF6
:1081100019F40E94F0386DC06DE37AE0C8010E9446
:10812000C09A892BF9F560917E0270917F0280E000
:1081300090E00E949F9A009709F45BC00E948C997E
:108140008531910530F5909374148093731442E057
:1081500050E062E070E083E794E10E943A9E609113
:108160007E0270917F0280E090E00E949F9A0097CB
:1081700009F43FC00E948C999093721480937114FB
:1081800042E050E060E070E081E794E10E943A9EB6
:1081900030C084E995E09F938F930E94839B0F905A
:1081A0000F9027C0809174148F93809173148F93D4
:1081B0008BE895E09F938F930E94839B09E912E1DE
:1081C0001F930F930E94839B809172148F938091D1
:1081D00071148F938CE795E09F938F930E94839BFC
:1081E0001F930F930E94839B0FB6F894DEBF0FBEC0
:1081F000CDBF89E992E19F938F930E94839B0F905B
:108200000F900C94A04E60917E0270917F0280E0EE
:1082100090E00E949F9A8C016CEE74E00E94C09ADC
:10822000892B09F077C060917E0270917F0280E017
:1082300090E00E949F9A8C01009711F40C94A04E3C
:108240006BE37AE00E94C09A892BB1F482E29FEF3F
:10825000ACECBBE38093850290938602A0938702E7
:10826000B093880244E050E06EE470E085E892E06C
:108270000E943A9E0C94A04E69EF75E0C8010E94DE
:10828000C09A892BB1F482E29FEFACECBAE3809301
:10829000850290938602A0938702B093880244E0FF
:1082A00050E06EE470E085E892E00E943A9E0C9403
:1082B000A04EC8010E9488992B013C0120E030E0CB
:1082C000A9010E9473938823D9F081E00E94411094
:1082D0009B01AC01C301B2010E94789360938502B7
:1082E00070938602809387029093880244E050E066
:1082F0006EE470E085E892E00E943A9E0C94A04EF5
:108300008FE695E09F938F930E94839B0F900F9031
:108310000C94A04E6FEE74E0C8010E94C09A892BA5
:1083200009F077C060917E0270917F0280E090E05A
:108330000E949F9A8C01009711F40C94A04E6BE35D
:108340007AE00E94C09A892BB1F482E29FEFACECF4
:10835000BBE38093810290938202A0938302B09347
:10836000840244E050E06AE470E081E892E00E9418
:108370003A9E0C94A04E69EF75E0C8010E94C09A25
:10838000892BB1F482E29FEFACECBAE380938102D7
:1083900090938202A0938302B093840244E050E061
:1083A0006AE470E081E892E00E943A9E0C94A04E4C
:1083B000C8010E9488992B013C0120E030E0A9010E
:1083C0000E9473938823D9F082E00E9441109B01A0
:1083D000AC01C301B2010E94789360938102709353
:1083E0008202809383029093840244E050E06AE426
:1083F00070E081E892E00E943A9E0C94A04E82E6E2
:1084000095E09F938F930E94839B0F900F900C9405
:10841000A04E67EE74E0C8010E94C09A892B09F053
:1084200073C060917E0270917F0280E090E00E94B4
:108430009F9A8C01009711F40C94A04E6BE37AE0A4
:108440000E94C09A892BB1F487ED94E3AFEEBCE3B0
:108450008093890290938A02A0938B02B0938C023E
:1084600044E050E062E570E089E892E00E943A9EC4
:108470000C94A04E69EF75E0C8010E94C09A892B48
:1084800051F483E595E09F938F930E94839B0F9017
:108490000F900C94A04EC8010E9488992B013C01BA
:1084A00020E030E0A9010E947393882319F180E055
:1084B0000E9441104B015C0121EE3AE744E95EE382
:1084C000C301B2010E949492A50194010E94789385
:1084D0006093890270938A0280938B0290938C023E
:1084E00044E050E062E570E089E892E00E943A9E44
:1084F0000C94A04E86E495E09F938F930E94839BFB
:108500000F900F900C94A04E0E948F109F938F930A
:108510007F936F938FE395E09F938F930E94839B4C
:1085200082E00E94411020918102309182024091AC
:108530008302509184020E942496162F072FF82E52
:10854000E92E81E00E944110EF92FF920F931F935A
:1085500020918502309186024091870250918802D5
:108560000E9424969F938F937F936F9383E395E06C
:108570009F938F930E94839B89E992E19F938F93AE
:108580000E94839B0FB6F894DEBF0FBECDBF0C9444
:10859000A04E60917E0270917F0280E090E00E9488
:1085A0009F9A009711F10E94722A00917D141091F8
:1085B0007E1420917F143091801460177107820718
:1085C000930769F160937D1470937E1480937F14F8
:1085D0009093801444E050E06AE570E08DE794E108
:1085E0000E943A9E8DE997E002C086E997E09F934A
:1085F0008F930E94839B60917D1470917E14809173
:108600007F14909180140E947F2989E992E19F93C1
:108610008F930E94839B0F900F900F900F908BE889
:1086200097E09F938F930E94839B6FEF7FEFCB0127
:108630000E947F2989E992E19F938F930E94839BF7
:108640000F900F900F900F900C94A04E0E94542604
:108650000C94A04EF3018481843329F440E061E05E
:1086600080E00E94641880918002882311F40C94A9
:10867000A04E1F928F9388E897E09F938F930E945C
:10868000839B0F900F900F900F900C94A04EF301CE
:108690008481893709F080C060917E0270917F02E9
:1086A00080E090E00E949F9A8C0166E475E00E9451
:1086B000C09A892B51F48091660290916702A09133
:1086C0006802B0916902906410C069E475E0C80165
:1086D0000E94C09A892BD1F4809166029091670222
:1086E000A0916802B09169029F7B8093660290938B
:1086F0006702A0936802B093690244E050E06EE123
:1087000070E086E692E00E943A9E46C06EEF75E009
:10871000C8010E94C09A892B21F58091A71D8F93D3
:108720008091A61D8F938091A51D8F938091A41D8C
:108730008F938091A31D8F938091A21D8F93809121
:10874000A11D8F938091A01D8F9388E095E09F934A
:108750008F930E94839B0FB6F894DEBF0FBECDBFF0
:108760001BC08091660290916702A0916802B0914F
:10877000690296FF03C086E495E002C089E495E0B3
:108780009F938F9384E095E09F938F930E94839BA8
:108790000F900F900F900F9080918002882311F41A
:1087A0000C94A04E1F928F9385E897E09F938F9330
:1087B0000E94839B0F900F900F900F900C94A04EEF
:1087C000F30184818737E9F560917E0270917F0221
:1087D00080E090E00E949F9A0097D9F00E948899CB
:1087E0002B013C0120E030E0A9010E947393882313
:1087F00081F040928D0250928E0260928F027092B0
:10880000900244E050E066E570E08DE892E00E945E
:108810003A9E809190028F9380918F028F938091E6
:108820008E028F9380918D028F9386EF94E09F93B9
:108830008F930E94839B0F900F900F900F900F903B
:108840000F9080918002882311F40C94A04E1F9207
:108850008F9382E897E09F938F930E94839B0F9062
:108860000F900F900F900C94A04E60917E0270912B
:108870007F0280E090E00E949F9A8C0166E475E0A0
:108880000E94C09A40906602509067026090680211
:1088900070906902892B19F4689457F809C069E44B
:1088A00075E0C8010E94C09A892B99F4E89457F8A2
:1088B000409266025092670260926802709269026A
:1088C00044E050E06EE170E086E692E00E943A9E5D
:1088D00013C057FE03C086E495E002C089E495E02A
:1088E0009F938F9382EF94E09F938F930E94839B3B
:1088F0000F900F900F900F9080918002882311F4B9
:108900000C94A04E1F928F938FE797E09F938F93C5
:108910000E94839B0F900F900F900F900C94A04E8D
:1089200060917E0270917F0280E090E00E949F9AA9
:108930008C0164E076E00E94C09A892B11F489E1F1
:1089400008C068E076E0C8010E94C09A892B49F40B
:1089500080E18093C4001092C50082E08093C00043
:1089600055C06CE076E0C8010E94C09A892B11F4D2
:1089700088E0EFCF61E176E0C8010E94C09A892BC0
:1089800039F066E176E0C8010E94C09A892B11F4A3
:1089900083E0DFCF8091C400893141F48DEE94E013
:1089A0009F938F930E94839B0F900F908091C400A0
:1089B000803141F488EE94E09F938F930E94839BD3
:1089C0000F900F908091C400883041F482EE94E0C3
:1089D0009F938F930E94839B0F900F908091C40070
:1089E000833041F48CED94E09F938F930E94839B9E
:1089F0000F900F908091C400883041F486ED94E090
:108A00009F938F930E94839B0F900F908091800281
:108A1000882311F40C94A04E1F928F938CE797E05B
:108A20009F938F930E94839B0F900F900F900F90B6
:108A30000C94A04E60917E0270917F0280E090E0E5
:108A40000E949F9A6BE37AE00E94C09A892B11F4EE
:108A500081E001C080E00E943C298091800288234F
:108A600011F40C94A04E1F928F9389E797E09F9387
:108A70008F930E94839B0F900F900F900F900C94F8
:108A8000A04E0E945B2780918002882311F40C94F1
:108A9000A04E1F928F9386E797E09F938F930E943B
:108AA000839B0F900F900F900F900C94A04E0E94FC
:108AB000572780918002882311F40C94A04E1F92B6
:108AC0008F9383E797E09F938F930E94839B0F90F0
:108AD0000F900F900F900C94A04E60917E027091B9
:108AE0007F0280E090E00E949F9A0E948C998031E2
:108AF00070F480937A140E94F27241E050E06DE1CC
:108B000070E08AE794E10E943A9E0C94A04E809116
:108B10007A141F928F938CEC94E09F938F930E9412
:108B2000839B0F900F900F900F900C94A04E60912C
:108B30007E0270917F0280E090E00E949F9A0E94E6
:108B40008C9995EF980F903170F4809365020E9494
:108B5000DF7141E050E06CE170E085E692E00E9458
:108B60003A9E0C94A04E809165021F928F9383ECE5
:108B700094E09F938F930E94839B0F900F900F9090
:108B80000F900C94A04E60917E0270917F0280E065
:108B900090E00E949F9A009789F04AE050E0BC0163
:108BA0008FE89DE10E94D09A4AE050E064E070E0D6
:108BB0008FE89DE10E943A9E0C94A04E8FE89DE1C3
:108BC0009F938F938BE196E09F938F930E946F9B6F
:108BD0000F900F900F900F900C94A04E60917E021A
:108BE00070917F0280E090E00E949F9A8C0162E782
:108BF00073E00E94C09A892BE1F4219A8091660269
:108C000090916702A0916802B0916902806180939F
:108C1000660290936702A0936802B093690244E0F1
:108C200050E06EE170E086E692E00E943A9E0C947D
:108C3000A04E60EF74E0C8010E94C09A892BE1F455
:108C4000229A8091660290916702A0916802B09189
:108C5000690280628093660290936702A093680223
:108C6000B093690244E050E06EE170E086E692E085
:108C70000E943A9E0C94A04E64E573E0C8010E94E5
:108C8000C09A892BE1F4239A809166029091670241
:108C9000A0916802B091690280648093660290930B
:108CA0006702A0936802B093690244E050E06EE16D
:108CB00070E086E692E00E943A9E0C94A04E63E932
:108CC00074E0C8010E94C09A892BE1F4239A809134
:108CD000660290916702A0916802B0916902806873
:108CE0008093660290936702A0936802B093690232
:108CF00044E050E06EE170E086E692E00E943A9E29
:108D00000C94A04E6CE473E0C8010E94C09A892BB9
:108D100079F581E08093E03188EA9DE19093E2313A
:108D20008093E1311092E4311092E3318091660238
:108D300090916702A0916802B0916902916080935E
:108D4000660290936702A0936802B093690244E0C0
:108D500050E06EE170E086E692E00E943A9E40EEBE
:108D600051E362E182E492E00E949E780C94A04E6E
:108D70006BE773E0C8010E94C09A892B19F5E8EDF2
:108D8000FDE188EF9DE1119211928E179F07D9F7AF
:108D90008091660290916702A0916802B091690289
:108DA00092608093660290936702A0936802B093EA
:108DB000690244E050E06EE170E086E692E00E94D5
:108DC0003A9EBEC769E475E0C8010E94C09A40910E
:108DD0006602509167026091680270916902892B66
:108DE000C1F44F705C7F40936602509367026093BA
:108DF0006802709369022B9A44E050E06EE170E0E3
:108E000086E692E00E943A9E809185360E94ED713E
:108E100097C744FF03C086E495E002C089E495E06B
:108E20009F938F9388EB94E09F938F930E94839BF3
:108E3000809166020F900F900F900F9085FF03C0F6
:108E400086E495E002C089E495E09F938F938DEAD4
:108E500094E09F938F930E94839B809166020F9072
:108E60000F900F900F9086FF03C086E495E002C03C
:108E700089E495E09F938F9382EA94E09F938F9388
:108E80000E94839B809166020F900F900F900F902D
:108E900087FF03C086E495E002C089E495E09F93D4
:108EA0008F9387E994E09F938F930E94839B809197
:108EB000660290916702A0916802B09169020F90DA
:108EC0000F900F900F9090FF03C086E495E002C0D2
:108ED00089E495E09F938F938CE894E09F938F9320
:108EE0000E94839B8091660290916702A091680224
:108EF000B09169020F900F900F900F9091FF03C0F7
:108F000086E495E002C089E495E09F938F9381E821
:108F100094E09F938F930E94839B8091660290912F
:108F20006702A0916802B09169020F900F900F90B4
:108F30000F9091FF05C783E296E00E94AB9B98EDEE
:108F4000E92E9DE1F92E0BE010E02BE2822E26E0C7
:108F5000922EF70180819181F2E0EF0EF11C9F9338
:108F60008F931F930F939F928F920E946F9B0F5F1F
:108F70001F4F0F900F900F900F900F900F900B318D
:108F8000110539F7DDC68FE697E09F938F930E9416
:108F9000839B809180020F900F90882361F01F9235
:108FA0008F938CE697E09F938F930E94839B0F9003
:108FB0000F900F900F90F89498E088E10FB6F89416
:108FC000A895809360000FBE90936000FFCF0E9431
:108FD0009B65B6C660917E0270917F0280E090E052
:108FE0000E949F9A8C0166E475E00E94C09A892BCA
:108FF000E9F40E94E3708091660290916702A0916B
:109000006802B09169028D7F8160809366029093BF
:109010006702A0936802B093690244E050E06EE1F9
:1090200070E086E692E00E943A9E8AC669E475E0A6
:10903000C8010E94C09A892BE1F40E941A708091A5
:10904000660290916702A0916802B09169028C7FDC
:109050008093660290936702A0936802B0936902BE
:1090600044E050E06EE170E086E692E00E943A9EB5
:1090700067C666E376E0C8010E94C09A892BE9F4CE
:109080000E941A708091660290916702A091680216
:10909000B09169028E7F826080936602909367022E
:1090A000A0936802B093690244E050E06EE170E082
:1090B00086E692E00E943A9E43C68091660281FF56
:1090C0000FC086E396E09F938F938DE794E09F9384
:1090D0008F930E94839B0F900F900F900F9030C63C
:1090E00080FF03C086E495E002C089E495E09F9389
:1090F0008F9389E794E09F938F930E94839B0F90B7
:109100000F900F900F901CC68091DE318F9380914D
:10911000DD318F938091DC318F938091DB318F93A0
:109120008091DA318F938091D9318F938091D831AA
:109130008F938091D7318F938091D6318F93809187
:10914000D5318F938091D4318F938091D3318F9388
:109150008091D2318F938091D1318F938091D03192
:109160008F938091CF318F9380E497E09F938F937B
:109170000E94839B89E992E19F938F930E94839B36
:10918000809180020FB6F894DEBF0FBECDBF88235A
:1091900009F4D6C51F928F938DE397E09F938F9329
:1091A0000E94839B0F900F900F900F90C9C5F89469
:1091B00089E021E030E0F90180935700C895E02C68
:1091C00020E030E0F90180935700C895F02C7894A6
:1091D000F89423E030E0F90180935700C895002D02
:1091E00022E030E0F90180935700C895102D789463
:1091F0008091B8298F938091B7298F938091B62958
:109200008F938091B5298F9383E397E09F938F93FA
:109210000E94839B1F92EF921F92FF921F920F93C7
:109220001F921F938CE097E09F938F930E94839BE4
:109230000E94F527809166001F928F9380E097E04F
:109240009F938F930E94839B89E992E19F938F93D1
:109250000E94839B809180020FB6F894DEBF0FBE00
:10926000CDBF882309F46CC51F928F938DEF96E0D4
:109270009F938F930E94839B0F900F900F900F905E
:109280005FC560E070E080E090E00E94A71160E0C0
:1092900070E081E090E00E94A71180918002882315
:1092A00009F44EC51F928F938AEF96E09F938F9398
:1092B0000E94839B0F900F900F900F9041C50E94CA
:1092C00017263F922F920E94839B809180020F90DD
:1092D0000F90882309F434C51F928F9387EF96E08F
:1092E0009F938F930E94839B0F900F900F900F90EE
:1092F00027C560917E0270917F0280E090E00E941D
:109300009F9A63EF75E00E94C09A892B31F5F8941B
:109310008FE69BE00E9475798C01892B69F0C8016A
:109320000F960E945677B80188E092E00E94F07A8A
:10933000C8010E94D679F0CF8FE69BE00E94C979E0
:10934000892B29F08FE69BE00E948979F5CF8FE683
:109350009BE00E947179789436C08FE69BE00E9472
:1093600075798C018BE3E82E86E0F82E0115110546
:1093700051F1F80186811F928F9380851F928F9300
:1093800085811F928F9381851F928F9387811F9272
:109390008F9384811F928F9383811F928F938281F9
:1093A0001F928F9382851F928F93FF92EF920E945C
:1093B0006F9BC8010E94D6798C010FB6F894DEBF6E
:1093C0000FBECDBFD3CF80918002882309F4B8C4EB
:1093D0001F928F9384EF96E09F938F930E94839BBD
:1093E0000F900F900F900F90ABC40E94CC36A8C482
:1093F00060917E0270917F0280E090E00E949F9ACF
:109400008C016AE776E00E94C09A892BD1F48091A2
:10941000660290916702A0916802B0916902977FFD
:109420008093660290936702A0936802B0936902EA
:1094300044E050E06EE170E086E692E00E943A9EE1
:109440007FC469EF75E0C8010E94C09A892BD1F4EE
:109450008091660290916702A0916802B0916902C2
:1094600098608093660290936702A0936802B0931D
:10947000690244E050E06EE170E086E692E00E940E
:109480003A9E5EC40E94230E5BC460917E0270917E
:109490007F0280E090E00E949F9AFC0120812332AD
:1094A000C1F44AE050E060E070E001960E944D9700
:1094B0007B836A8360917E0270917F0280E090E0FE
:1094C0000E949F9A2A813B81243031050CF09CC078
:1094D00002C01B821A82009709F496C01982BE014D
:1094E0006F5F7F4F0E945C2F19013A014B01B82F2B
:1094F000A92F8AE02A813B81829FF001839FF00D92
:109500001124E855F24E4080518032813C838381A2
:109510008D8394819E8325812F833681388787812F
:1095200089879101A301B4018B2F9A2F5201CC801E
:10953000DD80EE80FF80088519850E947F9209F406
:1095400066C08981811103C0208231822AC0181629
:1095500084F4422853289C81692A2D81722A3E81F5
:10956000832A8F81982A9885B92B2985A22B40823E
:1095700017C0209430946094709480949094B09527
:10958000A095242053203C8163228D8178229E81E6
:1095900089222F8192223885B3238985A8232082AE
:1095A00051826282738284829582B683A78348E265
:1095B00050E062E270E088EA9DE10E943A9E8CEE03
:1095C00096E09F938F930E94839B8AE02A813B8140
:1095D000829FF001839FF00D1124E855F24E208107
:1095E00031814281538164817581868197810E9496
:1095F0002B2B89E992E19F938F930E94839B0F907D
:109600000F900F900F9003C082E00E94363180EEE1
:1096100096E09F938F930E94839B2FEF3FEF4FEF36
:109620005FEF6FEF7FEF8FEF9FEF0E942B2B89E9AA
:1096300092E19F938F930E94839B809180020F9071
:109640000F900F900F90882309F47AC31F928F9385
:109650008DED96E09F938F930E94839B0F900F90C8
:109660000F900F906DC360917E0270917F0280E039
:1096700090E00E949F9AFC0120812332A1F44AE0ED
:1096800050E060E070E001960E944D978B01609180
:109690007E0270917F0280E090E00E949F9A0430E9
:1096A0001105ECF402C000E010E00097C1F04AE0C0
:1096B00050E060E070E00E947B982AE0209FF0017B
:1096C000219FF00D1124E855F24E7187608748E222
:1096D00050E062E270E088EA9DE10E943A9E81E0FB
:1096E0000E94363180918002882309F429C31F9299
:1096F0008F938AED96E09F938F930E94839B0F90A8
:109700000F900F900F901CC30E94DF798091800210
:10971000882309F415C31F928F9387ED96E09F93DA
:109720008F930E94839B0F900F900F900F9008C310
:109730000E94083280918002882309F401C31F929D
:109740008F9384ED96E09F938F930E94839B0F905D
:109750000F900F900F90F4C280E090E00E941128CB
:1097600080918002882309F4EBC21F928F9381EDD0
:1097700096E09F938F930E94839B0F900F900F9082
:109780000F90DEC28091C52D81FF2DC00E949D25C6
:10979000892B49F58091BC298F938091BB298F93A8
:1097A0008091BA298F938091B9298F9386EC96E0A6
:1097B0009F938F930E94839B8091A9368F93809172
:1097C000A8368F938091A7368F938091A6368F937A
:1097D00089EB96E09F938F930E94839B0FB6F8943A
:1097E000DEBF0FBECDBF89E992E19F938F930E94A8
:1097F000839B8091C52D9091C62D0F900F9093FF64
:1098000063C081E090E00E9415251B012C0180E0DF
:1098100090E00E9415257B018C010E9473245F92C9
:109820004F923F922F9288EA96E09F938F930E94E7
:10983000839B1F930F93FF92EF9288E996E09F938B
:109840008F930E94839B370148019701A801710102
:109850008201B101C2010E9410239F938F937F93D5
:109860006F938DE896E09F938F930E94839B262DA4
:10987000372D482D592D622D7F2D842D912F0E943B
:1098800071239F938F937F936F938FE796E09F93BE
:109890008F930E94839B262D372D482D592D622DA5
:1098A0007F2D842D912F0E94D6239F938F937F939A
:1098B0006F938CE696E09F938F930E94839B0FB6E5
:1098C000F894DEBF0FBECDBF89E992E19F938F93DD
:1098D0000E94839B809180020F900F90882309F44F
:1098E0002FC21F928F9389E696E09F938F930E94D9
:1098F000839B0F900F900F900F9022C28091C52DE7
:1099000082FF43C021E048E061E083E00E94CA1981
:109910008091AC1E8F938091AB1E8F938091AA1E75
:109920008F938091A91E8F938091A81E8F93809111
:10993000A71E8F938091A61E8F938091A51E8F9353
:1099400082E596E09F938F930E94839B3F922F9294
:109950000E94839B8091A41E8F938091A31E8F935E
:109960008091A21E8F938091A11E8F9384E496E034
:109970009F938F930E94839B3F922F920E94839B81
:109980000FB6F894DEBF0FBECDBF8091C52D85FF09
:109990005CC081E00E9483686091993670919A362C
:1099A00080919B3690919C360E942C9420E030E070
:1099B00048EC52E40E9478939F938F937F936F9328
:1099C0008DE495E09F938F930E946F9B60919D36ED
:1099D00070919E3680919F369091A0360E942A9475
:1099E00020E030E040E85AE30E9424969F938F9352
:1099F0007F936F938CE595E09F938F930E946F9B6D
:109A00006091A1367091A2368091A3369091A436D0
:109A10000E942A9420E030E040E85BE30E94249614
:109A20009F938F937F936F938DE695E09F938F9392
:109A30000E946F9B89E992E19F938F930E94839B81
:109A40000FB6F894DEBF0FBECDBF8091C52D9091AB
:109A5000C62D94FF3FC00E942F1E20E030E048EC4E
:109A600052E4162F072FF82EE92E0E94249620E8A4
:109A700036EE45EC57E40E94789321E03EED42E457
:109A80005EE30E9491969B01AC0160E070E080E88B
:109A90009FE30E9494922BE43AE34DEB57E30E943C
:109AA00078939F938F937F936F93EF92FF920F938F
:109AB0001F938BE296E09F938F930E94839B89E98B
:109AC00092E19F938F930E94839B0FB6F894DEBF21
:109AD0000FBECDBF80918002882309F431C11F924F
:109AE0008F9388E296E09F938F930E94839B0F90C1
:109AF0000F900F900F9024C160917E0270917F02B1
:109B000080E090E00E949F9A6FE776E00E94C09A02
:109B1000892B99F460917E0270917F0280E090E041
:109B20000E949F9A009709F40BC10E948C99909112
:109B30005201892B8093520103C1809152018F7091
:109B40001F928F938CE694E09F938F930E94839B48
:109B500089E992E19F938F930E94839B0F900F90CE
:109B60000F900F900F900F90EBC060917E0270915C
:109B70007F0280E090E00E949F9A009711F14AE0F6
:109B800050E060E070E00E944D97603198F460937F
:109B900064021F926F938BE196E09F938F930E94D4
:109BA000839B41E050E06BE170E084E692E00E942C
:109BB0003A9E11C0809164021F928F9382E196E0D9
:109BC00006C0809164021F928F9389E096E09F9374
:109BD0008F930E94839B0F900F900F900F9089E9B5
:109BE00092E19F938F930E94839B809180020F90BC
:109BF0000F90882309F4A4C01F928F9386E096E00B
:109C00009F938F930E94839B0F900F900F900F90C4
:109C100097C060917E0270917F0280E090E00E9488
:109C20009F9A8C0166E475E00E94C09A892BE1F44A
:109C30000E940F6F8091660290916702A091680266
:109C4000B091690290618093660290936702A0933D
:109C50006802B093690244E050E06EE170E086E68D
:109C600092E00E943A9E6CC069E475E0C8010E94CF
:109C7000C09A892B99F5F8940E941C6F0FB6F8943E
:109C8000A8958091600088618093600010926000C8
:109C90000FBE84B7877F84BF809160008861809306
:109CA0006000109260007894809166029091670243
:109CB000A0916802B09169029F7E809366029093A2
:109CC0006702A0936802B093690244E050E06EE13D
:109CD00070E086E692E00E943A9E32C064E876E048
:109CE000C8010E94C09A409166025091670260913B
:109CF000680270916902892B69F454FF02C0F894DC
:109D0000FFCF8BE594E09F938F930E94839B0F90EE
:109D10000F9016C054FF03C086E495E002C089E4AA
:109D200095E09F938F9387E594E09F938F930E9494
:109D3000839B0F900F900F900F9002C00E943B26C4
:109D4000EA85FB851182108283E02B960FB6F8948A
:109D5000DEBF0FBECDBFDF91CF911F910F91FF905E
:109D6000EF90DF90CF90BF90AF909F908F907F90BB
:109D70006F905F904F903F902F900895CF93DF9317
:109D8000EC0188819981009741F08037924109F474
:109D900090C01982188283E097C00E94F4378091A6
:109DA000660280FD05C081FF01C01D9B0E941A70E4
:109DB000809170008C7F809370008091B6008062EB
:109DC0008093B6001092B20082E08093B10080913F
:109DD000B6008770E1F78091700081608093700019
:109DE00061E47EE080E090E00E94E96E0E945727E7
:109DF00080E00E943C2984E693E19F938F930E9428
:109E0000839B0E9488168091C52D9091C62D0F903E
:109E10000F9091FD0E9447658091C52D9091C62DB0
:109E200093FD0E942B248091C52D9091C62D92FF09
:109E300006C021E04CE061E080ED0E94EA6580917F
:109E40007A140E94F272809165020E94DF710E9472
:109E5000DC7180935F0B809165020E94DF718091BD
:109E60007A141F928F9380915F0B1F928F9389E8D2
:109E700096E09F938F930E946F9B1092610B1092BC
:109E8000600B0F900F900F900F900F900F9086E542
:109E900092E0909398368093973683E290E0909387
:109EA00076148093751480E792E19983888381E02A
:109EB0000BC06332E1F744EF51E360E070E080E60D
:109EC0009BE00E947539E3CFDF91CF9108950F9306
:109ED0001F93CF93DF93EC018A01888199810097CA
:109EE00011F18538924121F01982188283E020C057
:109EF0006231E9F4A80162E170E080E69BE00E9433
:109F0000753984E080937C3610927E3610927D36CF
:109F10001093803600937F364CE756E362E182E48B
:109F200092E00E949E7885E892E19983888381E09F
:109F3000DF91CF911F910F9108958436910514F10F
:109F40009F938F938FED96E09F938F930E946F9BCB
:109F50008091CF319091D031A091D131B091D23157
:109F60000196A11DB11D8093CF319093D031A09364
:109F7000D131B093D2310F900F900F900F9081E0BC
:109F800090E0089580E090E008952F923F924F92E4
:109F90005F926F927F928F929F92AF92BF92CF9279
:109FA000DF92EF92FF920F931F93CF93DF93CDB782
:109FB000DEB7C959D1090FB6F894DEBF0FBECDBFC9
:109FC000CE56DF4F99838883C259D040F62E8A013E
:109FD00023E8621304C084E69BE00E941D7ECE56F7
:109FE000DF4FA881B981C259D0408D919C918D31AC
:109FF000B2E19B0711F40C94E95E38F4009781F00C
:10A000008E31904109F4E7C4DBC48F3222E192071C
:10A0100009F4B5C48633924111F40C94F15ED0C4B6
:10A0200045EB59E061E870E084E69BE00E94027E27
:10A030008EE190E19BC48C010F5F1F4FE3E0F0E0E5
:10A04000EC0FFD1FE00FF11F1082C8010E949D4F11
:10A05000892B71F720E030E040E050E0C157DF4F3E
:10A060006881CF58D040627070E080E090E0A0E05E
:10A070000E94889209F0A4C7C557DF4F2881CB58AA
:10A08000D040287030E040E050E060E070E080E0D8
:10A0900090E0A0E00E94889299F127E04AE250E027
:10A0A0006BE270E089E290E00E94CE618EE896E378
:10A0B0000E949463BC01990F880B990B0E942C9409
:10A0C00020E030E048EC52E40E9478939F938F9315
:10A0D0007F936F9383E197E09F938F931F9287E71E
:10A0E0008F93CE01800F911F03969F938F930E94B1
:10A0F000DB9B080F191F0FB6F894DEBF0FBECDBF54
:10A10000C557DF4F2881CB58D040207130E040E068
:10A1100050E060E070E080E090E0A0E00E94889273
:10A12000E9F126E04AE250E06BE270E089E290E07B
:10A130000E94CE6181E090E00E94381180937914F2
:10A1400081E09EE10E949463BC01990F880B990BFA
:10A150000E942C9420E030E048EC52E40E94789376
:10A160009F938F937F936F938DE197E09F938F934E
:10A170001F9287E78F93C801029621E030E02C0FF1
:10A180003D1F820F931F9F938F930E94DB9B080FAD
:10A19000191F0FB6F894DEBF0FBECDBF2E2D30E0D5
:10A1A00040E050E060E070E080E090E0A0E00E94DD
:10A1B000889201F10E94F4109F938F937F936F9385
:10A1C00088E297E09F938F931F9287E78F93C80150
:10A1D0000296A1E0B0E0AC0FBD1F8A0F9B1F9F93BA
:10A1E0008F930E94DB9B080F191F0FB6F894DEBFF8
:10A1F0000FBECDBFC557DF4F2881CB58D04020744C
:10A2000030E040E050E060E070E080E090E0A0E00E
:10A210000E94889231F18091CA318F938091C93127
:10A220008F938091C8318F938091C7318F9386E34C
:10A2300097E09F938F931F9287E78F93C8010296B1
:10A2400021E030E02C0F3D1F820F931F9F938F93CF
:10A250000E94DB9B080F191F0FB6F894DEBF0FBEDC
:10A26000CDBFC557DF4F2881CB58D040207830E094
:10A2700040E050E060E070E080E090E0A0E00E940C
:10A28000889241F1F8948091743690917536A0913E
:10A290007636B09177367894BF93AF939F938F9330
:10A2A00084E497E09F938F931F9287E78F93C80171
:10A2B0000296A1E0B0E0AC0FBD1F8A0F9B1F9F93D9
:10A2C0008F930E94DB9B080F191F0FB6F894DEBF17
:10A2D0000FBECDBF20E0C457DF4F3881CC58D040EF
:10A2E000317040E050E060E070E080E090E0A0E09D
:10A2F0000E94889209F075C620E0C457DF4F38816C
:10A30000CC58D040327040E050E060E070E080E037
:10A3100090E0A0E00E94889209F0C3C620E0C457F4
:10A32000DF4F3881CC58D040347040E050E060E0DE
:10A3300070E080E090E0A0E00E94889209F0E2C620
:10A3400020E0C457DF4F3881CC58D040387040E00F
:10A3500050E060E070E080E090E0A0E00E94889231
:10A3600009F000C720E0C457DF4F3881CC58D040F7
:10A37000307140E050E060E070E080E090E0A0E00C
:10A380000E94889209F04EC720E0C457DF4F388101
:10A39000CC58D040307240E050E060E070E080E0A7
:10A3A00090E0A0E00E94889209F06CC720E030E0C5
:10A3B00040E050E0C157DF4F6881CF58D040647013
:10A3C00070E080E090E0A0E00E94889209F088C7E9
:10A3D00020E0C956DF4F3881C759D04040E050E0F7
:10A3E00060E070E080E090E0A0E00E94889209F0D8
:10A3F000E5C720E0C856DF4F3881C859D04040E05B
:10A4000050E060E070E080E090E0A0E00E94889280
:10A4100011F00C940D5AC357DF4F5881CD58D040DE
:10A420005170E52E20E030E0452F50E060E070E014
:10A4300080E090E0A0E00E94889211F00C943C5AD9
:10A4400020E030E0C357DF4F4881CD58D040427004
:10A4500050E060E070E080E090E0A0E00E94889230
:10A4600011F00C94705A20E030E04F2D50E060E085
:10A4700070E080E090E0A0E00E94889211F00C94DF
:10A48000A45A20E030E040E050E0C157DF4F68813F
:10A49000CF58D040687070E080E090E0A0E00E946B
:10A4A000889211F00C94CF5A20E030E040E050E068
:10A4B000C157DF4F6881CF58D040607170E080E0B5
:10A4C00090E0A0E00E94889211F00C94FB5A20E0EA
:10A4D00030E0C357DF4F4881CD58D040487050E03E
:10A4E00060E070E080E090E0A0E00E94889211F0CF
:10A4F0000C94275B20E030E0C357DF4F4881CD58F4
:10A50000D040407150E060E070E080E090E0A0E07A
:10A510000E94889211F00C945C5B20E030E0C357FD
:10A52000DF4F4881CD58D040407250E060E070E08D
:10A5300080E090E0A0E00E94889211F00C94915B82
:10A5400020E030E0C357DF4F4881CD58D040407401
:10A5500050E060E070E080E090E0A0E00E9488922F
:10A5600011F00C94C65BC357DF4FF881CD58D04033
:10A57000F078DF2E20E030E04F2F50E060E070E018
:10A5800080E090E0A0E00E94889211F00C94FB5BC8
:10A59000C257DF4F2881CE58D0402170C22E20E014
:10A5A00030E040E05C2D60E070E080E090E0A0E012
:10A5B0000E94889211F40C94045F8091C52D82FF53
:10A5C00006C021E046E061E083E00E94CA1920E075
:10A5D00030E04D2D50E060E070E080E090E0A0E0E1
:10A5E0000E94889211F40C94435C8091C52D82FFE7
:10A5F00002C00C94085C20E030E040E0C257DF4F1E
:10A600005881CE58D040527060E070E080E090E019
:10A61000A0E00E94889211F00C94785C20E030E079
:10A6200040E0C257DF4F5881CE58D040547060E0B0
:10A6300070E080E090E0A0E00E94889211F00C941D
:10A64000AB5C20E030E040E0C257DF4F5881CE588D
:10A65000D040507160E070E080E090E0A0E00E94A7
:10A66000889211F00C94DE5C20E030E040E0C257AC
:10A67000DF4F5881CE58D040507260E070E080E0EB
:10A6800090E0A0E00E94889211F00C941D5D20E003
:10A6900030E040E0C257DF4F5881CE58D040507470
:10A6A00060E070E080E090E0A0E00E94889211F00D
:10A6B0000C945C5D20E030E040E0C257DF4F5881F1
:10A6C000CE58D040587060E070E080E090E0A0E0AC
:10A6D0000E94889211F00C949B5D20E030E040E0F5
:10A6E00050E0C157DF4F6881CF58D040607270E0B2
:10A6F00080E090E0A0E00E94889211F40C94CC5D80
:10A700008091C52D85FD02C00C94CC5D81E00E9436
:10A7100083686091993670919A3680919B369091BA
:10A720009C360E942C9420E030E048EC52E40E94D9
:10A7300078939F938F937F936F938DEC98E09F9383
:10A740008F931F9287E78F93C801029641E050E0F4
:10A750004C0F5D1F840F951F9F938F930E94DB9B6F
:10A76000080F191FC8010E949D4F0FB6F894DEBF55
:10A770000FBECDBF892B09F05BCCE1E020E030E0DB
:10A7800040E050E0C157DF4F6881CF58D04060743F
:10A7900070E080E090E0A0E00E94889211F00C94BC
:10A7A000CF5D20E030E040E050E0C157DF4F6881EE
:10A7B000CF58D040607870E080E090E0A0E00E9448
:10A7C000889211F00C94125E20E030E040E0C75611
:10A7D000DF4F5881C959D04060E070E080E090E0E0
:10A7E000A0E00E94889211F00C94545E20E030E0CA
:10A7F0004E2D50E060E070E080E090E0A0E00E942C
:10A80000889211F00C94895EC557DF4F2881CB5890
:10A81000D040C457DF4F3881CC58D040C357DF4FAA
:10A820004881CD58D040C257DF4F5881CE58D040D4
:10A83000C157DF4F6881CF58D040CC56DF4F788169
:10A84000C459D040CB56DF4F8881C559D040CA5635
:10A85000DF4F9881C659D040A0E00E94889211F045
:10A860000C94B65E80916402806189838091580B5C
:10A870008A83FE01E00FF11F138280917D14909175
:10A880007E14A0917F14B0918014F80133967F015B
:10A8900080FF0CC0FF92EF9388E199E09F938F9324
:10A8A0000E946F9B0F900F900F900F90B701CE01F9
:10A8B00001960E94627F8091660282FF0AC024E7AF
:10A8C00032E3A701BE016F5F7F4F8EE692E00E94E8
:10A8D000AD6480917D1490917E14A0917F14B0910D
:10A8E000801482FD73980E94E37084E69BE00E94CE
:10A8F0001F7E8091660290916702A0916802B091DC
:10A90000690290FD02C00C949A5E0F5F1F4F0E9477
:10A91000DC71E82E89E10E94ED71809166029091D0
:10A920006702A0916802B091690290FD02C00C9488
:10A93000965E73988091580B8F5F8093580B8A8333
:10A94000B8016F5F7F4FCE0101960E94627F84E65F
:10A950009BE00E941F7E40E050E065E88091E21598
:10A960009091E3150E949E788DE192E1CE56DF4FE3
:10A97000A881B981C259D0408D939C931EC08CE4AC
:10A980009BE00E946F76892BC1F00E94E37080915A
:10A99000660287FD2B9840E450E060E070E08CE4B4
:10A9A0009BE00E94517686E392E1CE56DF4FE8812C
:10A9B000F981C259D0409183808381E00C94145F67
:10A9C000CE56DF4FA881B981C259D0401D921C924A
:10A9D00083E00C94145FB2E1FB12EFCF809066022B
:10A9E00090906702A0906802B090690291FC20CB21
:10A9F000F80180818130E1F50180F281E02D208134
:10AA0000C557DF4F2883CB58D0403181C457DF4F23
:10AA10003883CC58D0404281C357DF4F4883CD584C
:10AA2000D0405381C257DF4F5883CE58D0408481E5
:10AA3000C157DF4F8883CF58D0409581CC56DF4F28
:10AA40009883C459D040A681CB56DF4FA883C559FF
:10AA5000D040B781CA56DF4FB883C659D040608412
:10AA60007184C057DF4F19821882C059D04085C009
:10AA7000823041F5F8010380F481E02DC057DF4FAB
:10AA8000F983E883C059D040612C712CF1E0C5579F
:10AA9000DF4FF883CB58D040C457DF4F1882CC58D3
:10AAA000D040C357DF4F1882CD58D04020E8C2575E
:10AAB000DF4F2883CE58D040C157DF4F1882CF5880
:10AAC000D0404CC0833039F1843009F0B1CA612CD8
:10AAD000712CC057DF4F19821882C059D04035E021
:10AAE000C557DF4F3883CB58D040C457DF4F18824B
:10AAF000CC58D040C357DF4F1882CD58D040C257F2
:10AB0000DF4F1882CE58D04042E0C157DF4F488314
:10AB1000CF58D04023C0612C712CC057DF4F198211
:10AB20001882C059D04055E0C557DF4F5883CB58E5
:10AB3000D040C457DF4F1882CC58D040C357DF4FA6
:10AB40001882CD58D040C257DF4F1882CE58D0401F
:10AB500081E0C157DF4F8883CF58D040CC56DF4FBC
:10AB60001882C459D040CB56DF4F1882C559D04007
:10AB7000CA56DF4F1882C659D04020908D023090BF
:10AB80008E0240908F0250909002C090C731D090BA
:10AB9000C831E090C931F090CA312DEC3CEC4CE466
:10ABA0005EE3C201B1010E949592A70196010E9445
:10ABB000739318165CF0E894A0F880926602909265
:10ABC0006702A0926802B092690253C0A701960181
:10ABD000C201B1010E94519518160CF04AC0809133
:10ABE000D3319091D431A091D531B091D631019625
:10ABF000A11DB11D8093D3319093D431A093D53151
:10AC0000B093D631A0FC14CA6894A0F88092660272
:10AC100090926702A0926802B092690295E4C557CB
:10AC2000DF4F9883CB58D040A0E2C457DF4FA883B2
:10AC3000CC58D040C357DF4F1882CD58D040C257B0
:10AC4000DF4F1882CE58D040B4E0C157DF4FB883F1
:10AC5000CF58D040CC56DF4F1882C459D040CB5685
:10AC6000DF4F1882C559D040CA56DF4F1882C659E7
:10AC7000D040C357DF4FE881CD58D040E470FE2E5E
:10AC800020E030E04E2F50E060E070E080E090E0A7
:10AC9000A0E00E94889209F08C9AC557DF4FF88196
:10ACA000CB58D040F072EF2E2F2F30E040E050E034
:10ACB00060E070E080E090E0A0E00E94889211F0F7
:10ACC0000E94F410C457DF4F2881CC58D040207424
:10ACD000C956DF4F2883C759D04020E0C956DF4FFF
:10ACE0003881C759D04040E050E060E070E080E03B
:10ACF00090E0A0E00E94889211F00E949D25C45728
:10AD0000DF4F3881CC58D0403078C856DF4F388379
:10AD1000C859D04020E040E050E060E070E080E0C2
:10AD200090E0A0E00E94889251F00E948F10609302
:10AD30008136709382368093833690938436C557DC
:10AD4000DF4F2881CB58D040217030E040E050E008
:10AD500060E070E080E090E0A0E00E948892F1F076
:10AD60008FE89DE19F938F9383EF96E09F938F935E
:10AD70001F9287E78F93CE0103969F938F930E9434
:10AD8000DB9B6C010E949D4F0FB6F894DEBF0FBE97
:10AD9000CDBF892B09F04CC9860102C000E010E04C
:10ADA000C557DF4F2881CB58D040227030E040E0BB
:10ADB00050E060E070E080E090E0A0E00E948892C7
:10ADC000D9F1C80102966BEF76E0A1E0B0E0AC0FDC
:10ADD000BD1F8A0F9B1F0E94C99A0D5F1F4F3EE83F
:10ADE000C32E36E3D32E46E9842E46E3942E54E850
:10ADF000A52E53E0B52E67E7562EF60181916F011F
:10AE00001F928F93BF92AF921F925F92C8010296DA
:10AE100021E030E02C0F3D1F820F931F9F938F93F3
:10AE20000E94DB9B080F191F0FB6F894DEBF0FBE00
:10AE3000CDBF8C149D0409F7C557DF4F2881CB582F
:10AE4000D040247030E040E050E060E070E080E00E
:10AE500090E0A0E00E94889209F446C0C8010296E2
:10AE60006FEF76E0A1E0B0E0AC0FBD1F8A0F9B1F33
:10AE70000E94C99A0C5F1F4F6E01BAE7CB0ED11C1E
:10AE800080E1F60111928A95E9F728E0A60168E9C8
:10AE900080EB0E944E164601F8E08F0E911C94E85C
:10AEA000A92E93E0B92E27E7522ED6018D916D0180
:10AEB0001F928F93BF92AF921F925F92C80102962A
:10AEC000E1E0F0E0EC0FFD1F8E0F9F1F9F938F932B
:10AED0000E94DB9B080F191F0FB6F894DEBF0FBE50
:10AEE000CDBFC814D90409F7C257DF4F3881CE58F7
:10AEF000D0403078C756DF4F3883C959D04020E062
:10AF000030E040E0C756DF4F5881C959D04060E07B
:10AF100070E080E090E0A0E00E948892E1F48091EF
:10AF20007B1490917C149F938F9384E097E09F9380
:10AF30008F931F9287E78F93CE01800F911F039607
:10AF40009F938F930E94DB9B080F191F0FB6F894F5
:10AF5000DEBF0FBECDBF20E030E040E050E0C15783
:10AF6000DF4F6881CF58D040617070E080E090E0A2
:10AF7000A0E00E94889209F46DC8E3E0F0E0EC0FD5
:10AF8000FD1FE00FF11F80E28083DE01A00FB11FE3
:10AF9000BD016C5F7F4FE4EFF1E3045F11439F015C
:10AFA0002D5F3F4FC8018E0F9F1F43813196442371
:10AFB00009F441C8D9018C91DB018D93BD01EFCF1C
:10AFC000CE01800F911F6BE077E003960E94C99A33
:10AFD000095F1F4FC8010E949D4F892B09F028C8A7
:10AFE0004BC86114710409F487C9F8942090743631
:10AFF00030907536409076365090773678948091C0
:10B00000F91D9091FA1DA091FB1DB091FC1DA201AC
:10B010009101281B390B4A0B5B0BCA01B9010E9435
:10B020002A944B015C01B30180E090E00E942A94D5
:10B030009B01AC01C501B4010E947893B62EC72EC6
:10B04000D82EE92E9F938F937F936F938FE497E091
:10B050009F938F931F9287E78F93CE01800F911F4D
:10B0600003969F938F930E94DB9B080F191F8B2DD4
:10B070009C2DAD2DBE2D8093863690938736A09360
:10B080008836B09389362092F91D3092FA1D40928D
:10B09000FB1D5092FC1D0FB6F894DEBF0FBECDBF56
:10B0A0002BC96114710409F439C9F8948091D01D39
:10B0B0009091D11DA091D21DB091D31D78949F93F2
:10B0C0008F9380916D028F9380916C028F938CE5AA
:10B0D00097E09F938F931F9287E78F93C801029603
:10B0E000A1E0B0E0AC0FBD1F8A0F9B1F9F938F9311
:10B0F0000E94DB9B080F191F0FB6F894DEBF0FBE2E
:10B10000CDBF0CC9F8948091783690917936A09192
:10B110007A36B0917B367894BF93AF939F938F9399
:10B120008CE697E09F938F931F9287E78F93C801D8
:10B13000029621E030E02C0F3D1F820F931F9F935A
:10B140008F930E94DB9B080F191FC8010E949D4F1F
:10B150000FB6F894DEBF0FBECDBF892B11F00C9453
:10B160001850EEC86114710409F4FCC8F8942090DA
:10B1700078363090793640907A3650907B36789495
:10B180008091FD1D9091FE1DA091FF1DB091001EAC
:10B19000A2019101281B390B4A0B5B0BCA01B901B3
:10B1A0000E942A944B015C01B30180E090E00E9470
:10B1B0002A949B01AC01C501B4010E947893B62E7C
:10B1C000C72ED82EE92E9F938F937F936F9387E797
:10B1D00097E09F938F931F9287E78F93CE01800F05
:10B1E000911F03969F938F930E94DB9B080F191F5B
:10B1F0008B2D9C2DAD2DBE2D80938A3690938B3652
:10B20000A0938C36B0938D362092FD1D3092FE1D9A
:10B210004092FF1D5092001E0FB6F894DEBF0FBE85
:10B22000CDBFA0C8672809F4AFC8F8948091D41D99
:10B230009091D51DA091D61DB091D71D78949F9364
:10B240008F9380916B028F9380916A028F9384E831
:10B2500097E09F938F931F9287E78F93C801029681
:10B26000A1E0B0E0AC0FBD1F8A0F9B1F9F938F938F
:10B270000E94DB9B080F191F0FB6F894DEBF0FBEAC
:10B28000CDBF82C88091CB319091CC31A091CD318E
:10B29000B091CE31BF93AF939F938F9384E997E0A2
:10B2A0009F938F931F9287E78F93C801029621E0A7
:10B2B00030E02C0F3D1F820F931F9F938F930E94AE
:10B2C000DB9B080F191FC8010E949D4F0FB6F89411
:10B2D000DEBF0FBECDBF892B11F00C94185066C88D
:10B2E0008091D6318F938091D5318F938091D431D5
:10B2F0008F938091D3318F938091D2318F938091AE
:10B30000D1318F938091D0318F938091CF318F93B2
:10B310008FE997E09F938F931F9287E7E82EEF9234
:10B32000C8010296A1E0B0E0AC0FBD1F8A0F9B1FC1
:10B330009F938F930E94DB9B080F191FC8010E94E7
:10B340009D4F0FB6F894DEBF0FBECDBF892B11F015
:10B350000C9418508091C52D9091C62D93FF38C83C
:10B360008091DA318F938091D9318F938091D83148
:10B370008F938091D7318F9383EC97E09F938F9336
:10B380001F92EF92C801029621E030E02C0F3D1F82
:10B39000820F931F9F938F930E94DB9B080F191FAF
:10B3A000C8010E949D4F0FB6F894DEBF0FBECDBFFF
:10B3B000892B11F00C9418500C94E8518091BC2901
:10B3C0008F938091BB298F938091BA298F9380911D
:10B3D000B9298F9385ED97E09F938F931F9287E70D
:10B3E0008F93C8010296A1E0B0E0AC0FBD1F8A0F99
:10B3F0009B1F9F938F930E94DB9B080F191FC8010F
:10B400000E949D4F0FB6F894DEBF0FBECDBF892BB3
:10B4100011F00C9418500C94F951809184368F934C
:10B42000809183368F93809182368F93809181367D
:10B430008F9380EE97E09F938F931F9287E78F9370
:10B44000C801029621E030E02C0F3D1F820F931FB0
:10B450009F938F930E94DB9B080F191FC8010E94C6
:10B460009D4F0FB6F894DEBF0FBECDBF892B11F0F4
:10B470000C9418500C940B5281E00E9441102091C2
:10B4800085023091860240918702509188020E9485
:10B4900024969F938F937F936F938DEE97E09F9366
:10B4A0008F931F9287E78F93C8010296A1E0B0E0C7
:10B4B000AC0FBD1F8A0F9B1F9F938F930E94DB9B36
:10B4C000080F191FC8010E949D4F0FB6F894DEBFE8
:10B4D0000FBECDBF892B11F00C9418500C94205244
:10B4E00082E00E94411020918102309182024091BD
:10B4F0008302509184020E9424969F938F937F939E
:10B500006F938AEF97E09F938F931F9287E78F93B4
:10B51000C801029621E030E02C0F3D1F820F931FDF
:10B520009F938F930E94DB9B080F191FC8010E94F5
:10B530009D4F0FB6F894DEBF0FBECDBF892B11F023
:10B540000C9418500C94335283E00E9441109F9346
:10B550008F937F936F9387E098E09F938F931F92D1
:10B5600087E78F93C8010296A1E0B0E0AC0FBD1F42
:10B570008A0F9B1F9F938F930E94DB9B080F191FBD
:10B580008C98C8010E949D4F0FB6F894DEBF0FBE85
:10B59000CDBF892B11F00C9418500C94415229996D
:10B5A00003C089E495E002C086E495E09F938F9301
:10B5B00084E198E09F938F931F9287E78F93C80150
:10B5C000029621E030E02C0F3D1F820F931F9F93C6
:10B5D0008F930E94DB9B080F191FC8010E949D4F8B
:10B5E0000FB6F894DEBF0FBECDBF892B11F00C94BF
:10B5F00018500C9454522A9903C089E495E002C073
:10B6000086E495E09F938F938CE198E09F938F93CE
:10B610001F9287E78F93C8010296A1E0B0E0AC0FBC
:10B62000BD1F8A0F9B1F9F938F930E94DB9B080F68
:10B63000191FC8010E949D4F0FB6F894DEBF0FBEC0
:10B64000CDBF892B11F00C9418500C946752809147
:10B65000C52D9091C62D92FD02C00C947A5221E026
:10B6600042E161E080ED0E94EA659F938F937F93B2
:10B670006F9384E298E09F938F931F9287E78F9355
:10B68000C801029621E030E02C0F3D1F820F931F6E
:10B690009F938F930E94DB9B080F191FC8010E9484
:10B6A0009D4F0FB6F894DEBF0FBECDBF892B11F0B2
:10B6B0000C9418500C947A528091C52D9091C62DFF
:10B6C00092FD02C00C948D5221E042E162E080EDD7
:10B6D0000E94EA659F938F937F936F9382E398E034
:10B6E0009F938F931F9287E78F93C8010296A1E0E3
:10B6F000B0E0AC0FBD1F8A0F9B1F9F938F930E94DA
:10B70000DB9B080F191FC8010E949D4F0FB6F894CC
:10B71000DEBF0FBECDBF892B11F00C9418500C94D6
:10B720008D528091C52D9091C62D92FD02C00C9432
:10B73000A05221E042E163E080ED0E94EA659F9320
:10B740008F937F936F9380E498E09F938F931F92E2
:10B7500087E78F93C801029621E030E02C0F3D1F50
:10B76000820F931F9F938F930E94DB9B080F191FDB
:10B77000C8010E949D4F0FB6F894DEBF0FBECDBF2B
:10B78000892B11F00C9418500C94A0528091C52D67
:10B790009091C62D92FD02C00C94B35221E042E17B
:10B7A00064E080ED0E94EA659F938F937F936F938F
:10B7B0008EE498E09F938F931F9287E78F93C80141
:10B7C0000296A1E0B0E0AC0FBD1F8A0F9B1F9F93B4
:10B7D0008F930E94DB9B080F191FC8010E949D4F89
:10B7E0000FB6F894DEBF0FBECDBF892B11F00C94BD
:10B7F00018500C94B3528091C52D82FD02C00C9458
:10B80000C85246E061E083E00E94CA190C94C85215
:10B810008091A81E8F938091A71E8F938091A61E62
:10B820008F938091A51E8F938CE598E09F938F93C3
:10B830001F9287E78F93C801029641E050E04C0FBA
:10B840005D1F840F951F9F938F930E94DB9B080FB2
:10B85000191FC8010E949D4F0FB6F894DEBF0FBE9E
:10B86000CDBF892B11F00C94185020E030E040E05F
:10B870005C2D60E070E080E090E0A0E00E948892A3
:10B8800011F40C94FB528091C52D82FD02C00C94E2
:10B89000FB528091AC1E8F938091AB1E8F93809151
:10B8A000AA1E8F938091A91E8F9384E698E09F93A0
:10B8B0008F931F9287E78F93C8010296E1E0F0E033
:10B8C000EC0FFD1F8E0F9F1F9F938F930E94DB9B9A
:10B8D000080F191FC8010E949D4F0FB6F894DEBFD4
:10B8E0000FBECDBF892B11F00C9418500C94FB5255
:10B8F0008091C52D9091C62D93FD02C00C940E53DE
:10B9000080E090E00E9415259F938F937F936F9323
:10B910008FE698E09F938F931F9287E78F93C801DC
:10B92000029641E050E04C0F5D1F840F951F9F93DE
:10B930008F930E94DB9B080F191FC8010E949D4F27
:10B940000FB6F894DEBF0FBECDBF892B11F00C945B
:10B9500018500C940E538091C52D9091C62D93FDD7
:10B9600002C00C94215381E090E00E9415259F9322
:10B970008F937F936F938FE798E09F938F931F929E
:10B9800087E78F93C8010296E1E0F0E0EC0FFD1F1E
:10B990008E0F9F1F9F938F930E94DB9B080F191F91
:10B9A000C8010E949D4F0FB6F894DEBF0FBECDBFF9
:10B9B000892B11F00C9418500C9421538091C52DB3
:10B9C0009091C62D93FD02C00C94345381E090E019
:10B9D0000E9415254B015C0180E090E00E94152536
:10B9E0009B01AC01C501B4010E9410239F938F936A
:10B9F0007F936F9380E998E09F938F931F9287E7DF
:10BA00008F93C801029641E050E04C0F5D1F840FF8
:10BA1000951F9F938F930E94DB9B080F191FC801EE
:10BA20000E949D4F0FB6F894DEBF0FBECDBF892B8D
:10BA300011F00C9418500C9434538091C52D9091B2
:10BA4000C62D93FD02C00C94475381E090E00E9404
:10BA500015254B015C0180E090E00E9415259B01BB
:10BA6000AC01C501B4010E9471239F938F937F9312
:10BA70006F938BE998E09F938F931F9287E78F9343
:10BA8000C8010296E1E0F0E0EC0FFD1F8E0F9F1F52
:10BA90009F938F930E94DB9B080F191FC8010E9480
:10BAA0009D4F0FB6F894DEBF0FBECDBF892B11F0AE
:10BAB0000C9418500C9447538091C52D9091C62D2D
:10BAC00093FD02C00C945A5381E090E00E9415252A
:10BAD0004B015C0180E090E00E9415259B01AC01C8
:10BAE000C501B4010E94D6239F938F937F936F93D8
:10BAF00089EA98E09F938F931F9287E78F93C801FD
:10BB0000029641E050E04C0F5D1F840F951F9F93FC
:10BB10008F930E94DB9B080F191FC8010E949D4F45
:10BB20000FB6F894DEBF0FBECDBF892B11F00C9479
:10BB300018500C945A538091C52D9091C62D94FDA8
:10BB400002C00C946D530E942F1E9F938F937F937E
:10BB50006F938CEB98E09F938F931F9287E78F935F
:10BB6000C8010296E1E0F0E0EC0FFD1F8E0F9F1F71
:10BB70009F938F930E94DB9B080F191FC8010E949F
:10BB80009D4F0FB6F894DEBF0FBECDBF892B11F0CD
:10BB90000C9418500C946D53E0E00C94BE538091BB
:10BBA000C52D85FD02C00C94D153E11103C081E085
:10BBB0000E94836860919D3670919E3680919F3679
:10BBC0009091A0360E942A9420E030E040E85AE3A9
:10BBD0000E9424969F938F937F936F938EED98E0AE
:10BBE0009F938F931F9287E78F93C8010296E1E09E
:10BBF000F0E0EC0FFD1F8E0F9F1F9F938F930E940D
:10BC0000DB9B080F191FC8010E949D4F0FB6F894C7
:10BC1000DEBF0FBECDBF892B11F00C941850E1E0B0
:10BC20000C94D1538091C52D85FD02C00C94E45332
:10BC3000E11103C081E00E9483686091A136709198
:10BC4000A2368091A3369091A4360E942A9420E0D7
:10BC500030E040E85BE30E9424969F938F937F93AC
:10BC60006F9380EF98E09F938F931F9287E78F9356
:10BC7000C801029641E050E04C0F5D1F840F951FF4
:10BC80009F938F930E94DB9B080F191FC8010E948E
:10BC90009D4F0FB6F894DEBF0FBECDBF892B11F0BC
:10BCA0000C9418500C94E453C057DF4FE881F9818D
:10BCB000C059D04086811F928F9385811F928F93A8
:10BCC00083811F928F9382811F928F9381E099E0ED
:10BCD0009F938F931F9287E78F93C801029621E06D
:10BCE00030E02C0F3D1F820F931F9F938F930E9474
:10BCF000DB9B080F191FC8010E949D4F0FB6F894D7
:10BD0000DEBF0FBECDBF892B11F00C9418500C94E0
:10BD1000F653779A80917D1490917E14A0917F14B0
:10BD2000B091801492FF22C0749A20C08E2D0E9480
:10BD3000ED71739A80917B1490917C14892B11F092
:10BD40000E941A708091580B8F5F8093580B8091DE
:10BD50007D1490917E14A0917F14B091801482FD87
:10BD600002C00C941850739A0C94185080917D1452
:10BD700090917E14A0917F14B091801482FD0CC02C
:10BD80008091660280FD08C081FD02C00C9432548F
:10BD90001D9902C00C94325440E050E060E070E025
:10BDA000CE0101960E94AC0E8091AE1E90E02091D3
:10BDB0007314309174148217930710F40C94325456
:10BDC00040E050E062E180E192E00E949E780C94B5
:10BDD0003254E5E8FE120C94DD5400E010E00C94BF
:10BDE0008D548CE49BE00E946F76892B11F40C94A7
:10BDF000DD540E941A708091660287FD02C00C9487
:10BE000018502B9A0C94185020E030E04D2D50E043
:10BE100060E070E080E090E0A0E00E94889211F085
:10BE20000C94F5520C94FB52C756DF4F0FB6F894A2
:10BE3000DEBF0FBECDBFDF91CF911F910F91FF905D
:10BE4000EF90DF90CF90BF90AF909F908F907F90BA
:10BE50006F905F904F903F902F9008950C94057DC8
:10BE60004F925F926F927F929F92AF92BF92CF92CA
:10BE7000DF92EF92FF920F931F93CF93DF93CDB793
:10BE8000DEB760970FB6F894DEBF0FBECDBF5B0183
:10BE90000E94DC71E82FF0E0EE0FFF1FEE53F24E30
:10BEA0008081918101969183808380917D1490910E
:10BEB0007E14A0917F14B091801481FD74984090FD
:10BEC00066025090670260906802709069020E945A
:10BED000B97E6C01FC018081982F92959F70913002
:10BEE00099F48F7051F48091A61D9091A71D019631
:10BEF0009093A71D8093A61D3EC1B50187EE98E3E0
:10BF00000E94D67F892B51F08091A41D9091A51D90
:10BF100001969093A51D8093A41D2DC1D301C2014C
:10BF20003EE0B695A795979587953A95D1F7F82F66
:10BF3000F1709F2E8FE69BE00E9475797C01892B22
:10BF400009F44BC0B501C70102960E94D67F892B28
:10BF500009F43FC087012BE53EE040E054E660E095
:10BF600070E0C7010F960E941E77F6019181F701DC
:10BF70008481981321C082858F5F82878091A21D62
:10BF80009091A31D01969093A31D8093A21D84E020
:10BF90000E94A27FF701208530E02817390708F0BA
:10BFA0007AC184E00E94A27FF7018087F601808138
:10BFB0008F70F7018187DFC0F701128684E00E944D
:10BFC000A27FF7018087F60180818F70F70181875A
:10BFD00063C1C7010E94D679B1CF88E092E00E9488
:10BFE000CB7A7C01892B09F4C6C0B501C701029642
:10BFF0000E94CF7FF60181818150F701848380E028
:10C0000091E0A0E0B0E083879487A587B687128689
:10C0100084E00E94A27FF7018087F60180818F7003
:10C02000F7018187B7018FE69BE00E94B079870115
:10C030002BE53EE040E054E660E070E0C7010F967B
:10C040000E941E7711E0F6018181F7018483F601D9
:10C0500080818F70F701878384E00E94A27FF701BF
:10C06000858383E00E94A27FF701868387818F30DA
:10C0700009F010E0F6014180F7018481481A512C43
:10C08000612C712C86E0440C551C661C771C8A952B
:10C09000D1F72385348545855685A0ECB0E00E9414
:10C0A000E790BB27A92F982F872F480E591E6A1E8D
:10C0B0007B1E4386548665867686A501B701C60138
:10C0C0000E94AC0E8091AE1E90E0209173143091CE
:10C0D00074148217930738F040E050E062E180E189
:10C0E00092E00E949E78809173149091741402974C
:10C0F00008F44DC08091C52D9091C62D91FF2AC0A6
:10C100000E943965C60105960E940565F601818188
:10C110001F928F93F70186811F928F9385811F92C3
:10C120008F9389E299E09F938F931F9280E18F9381
:10C13000CE0101965C019F938F930E94DB9B82E06E
:10C140000E941F65C5010E9405650FB6F894DEBF09
:10C150000FBECDBF8091660290916702A0916802E8
:10C16000B091690297FD4DC0809173149091741441
:10C17000029708F47AC080917D1490917E14A0916A
:10C180007F14B091801481FF89C0749A87C0809118
:10C19000660290916702A0916802B091690296FFD1
:10C1A000A9CF992009F4A6CFF6019081892F8F702D
:10C1B0008230E8F0907F8150892B808384E69BE079
:10C1C0000E942E5F8091A01D9091A11D01969093D9
:10C1D000A11D8093A01D80917D1490917E14A0914B
:10C1E0007F14B091801496FF85CF739883CF809190
:10C1F000A61D9091A71D01969093A71D8093A61D43
:10C2000079CF8FE89DE120918F1D222309F4ACCFD7
:10C210009F938F938CE399E09F938F93CE01019628
:10C220003C019F938F930E94189C5C01B301C6014F
:10C2300002960E94EA9A0F900F900F900F900F9025
:10C240000F90009709F490CFEFEFAE1ABE0A8A0D57
:10C250009B1DAC010196FA0120812032D1F362E1ED
:10C260008AE192E00E949E787FCF112309F483CF68
:10C2700082E08093E0311092E2311092E131F0924D
:10C28000E431E092E33140EE51E362E182E492E096
:10C290000E949E7870CF912C10E0D5CE60960FB69C
:10C2A000F894DEBF0FBECDBFDF91CF911F910F91EC
:10C2B000FF90EF90DF90CF90BF90AF909F907F90D6
:10C2C0006F905F904F9008958115910511F001973F
:10C2D000F1F70895E091AD36F091AE3690818091FE
:10C2E000AC3689230895E091AA36F091AB3690815F
:10C2F0008091AC36892B8083E091AF36F091B036D7
:10C3000090818091AC36892B808308951F93CF93C1
:10C31000DF93E091AA36F091AB3690818091AC36F4
:10C32000809589238083E091AF36F091B03690817B
:10C330008091AC36892B80838FE897E00E946461FE
:10C340001FB7F894E091AF36F091B03690818091AC
:10C35000AC3680958923808389E091E00E946461F6
:10C36000E091AD36F091AE36D081C091AC361FBFB2
:10C37000789485E896E00E946461E091AD36F09192
:10C38000AE3690818091AC36892319F08D2F8C23A5
:10C3900001C081E0DF91CF911F9108955093B03695
:10C3A0004093AF367093AB366093AA369093AE3617
:10C3B0008093AD3681E001C0880F2A95EAF780931B
:10C3C000AC360C948661CF93DF93C82FDFB7F89417
:10C3D000E091AF36F091B03690818091AC36892BE8
:10C3E000808387E090E00E946461CC2351F0E0916B
:10C3F000AF36F091B03690818091AC36809589232C
:10C40000808384E390E00E946461E091AD36F09116
:10C41000AE3690818091AC36892309F4C0E085EB7B
:10C4200090E00E946461E091AF36F091B036908167
:10C430008091AC36809589238083DFBF88E790E0C8
:10C440000E9464618C2FDF91CF910895CF93DF9389
:10C45000C82FD8E08C2F81700E94E361C6958111AE
:10C46000C068D150B9F78C2FDF91CF9108958FEF2D
:10C470000C942662DF92EF92FF920F931F93CF935B
:10C48000DF93E82E8B010E948661811135C080EF19
:10C490000E942662D0E0C0E488EFD82EDC0E81E056
:10C4A0000E94E361F82E81E00E94E361882319F085
:10C4B000FF2071F023C0F1100BC0CE1530F0F80151
:10C4C000808180FF05C0CE1519F0DC2FFF24F39486
:10C4D0008F2D0E94E361F80180818695FF2011F085
:10C4E0008068F8018083C150CD11D9CF0F5F1F4FF5
:10C4F000C111D2CF8D2F03C08FEF01C08EEFDF911E
:10C50000CF911F910F91FF90EF90DF900895EF92E0
:10C51000FF921F93CF93DF93182FEB010E94866148
:10C52000209771F085E50E9426627E0188E0E80E82
:10C53000F11C89910E942662CE15DF05D1F703C058
:10C540008CEC0E942662812FDF91CF911F91FF908A
:10C55000EF900C9426620F931F93CF93DF93DB0130
:10C56000ED91FC911197803161F4EE7F63E0EE0F65
:10C57000FF1F6A95E1F716969C911697E91BF10942
:10C580003C96F7FF07C091E0EA019883F195E195A9
:10C59000F10902C0EA011882883279F414968C916C
:10C5A000982F9076903649F086FF02C0EE7F05C046
:10C5B00085FF02C0EC7F01C0E87FCF0144E0969583
:10C5C00087954A95E1F7D9018C93EF70E801E883EC
:10C5D00080E0DF91CF911F910F9108950F931F93EA
:10C5E000CF93DF93EC018B01B80188810E943A62FE
:10C5F000888381508D3F30F4F8018081883211F0BA
:10C60000803191F7DF91CF911F910F910895CF93D2
:10C61000DF93EC010E948661BE0184EB0E94876279
:10C6200081E00E94E361C82F0E94866181E0C11110
:10C6300001C080E0DF91CF9108950F931F93CF93B6
:10C64000C82F8B010E9486610E946A61882349F08D
:10C65000B80184E40E948762C13029F00E947361AE
:10C6600002C082E001C080E0CF911F910F91089538
:10C670004F925F926F927F928F929F92AF92BF92F2
:10C68000CF92DF92EF92FF920F931F93CF93DF939E
:10C69000CDB7DEB729970FB6F894DEBF0FBECDBF7A
:10C6A0006C013B015A0189010E948661B6018EEB43
:10C6B0000E948762CE0101967C014E019AE0890EAC
:10C6C000911C27010E943762F70181937F01E815D1
:10C6D000F905C1F769E070E0C2010E941D83F82EE0
:10C6E000811108C09501A301B201F60180810E9469
:10C6F000AB6202C083E0F82E8F2D29960FB6F89416
:10C70000DEBF0FBECDBFDF91CF911F910F91FF9084
:10C71000EF90DF90CF90BF90AF909F908F907F90E1
:10C720006F905F904F900895EF92FF920F931F9339
:10C73000CF93DF93CDB7DEB72B970FB6F894DEBF5C
:10C740000FBECDBF182F092F682F792F88E0810FDA
:10C750000E941D63882319F084E391E244C06CE8D1
:10C7600072E88EE190E00E9400647E0189E0E80EAC
:10C77000F11C9701AE01465F5F4FBE01655F7F4FC1
:10C78000812F902F0E9438638111E6CF88E0E1EE7F
:10C79000F2E0DE01119601900D928A95E1F729856C
:10C7A00041E752E0249FC001259F900D112464E6CB
:10C7B00070E00E946C908A8594E6899F600D711DDF
:10C7C0001124FE0131968191281303C06F5F7F4FC2
:10C7D00003C0EE15FF05B9F78B85882319F0719515
:10C7E00061957109CB012B960FB6F894DEBF0FBE91
:10C7F000CDBFDF91CF911F910F91FF90EF900895E2
:10C80000DC01CB0181159105A105B10529F081500D
:10C810009040A040B040D9F708959B01AC01109220
:10C82000B90060E074E284EF90E00E948090DA0149
:10C83000C9014097A109B109B695A7959795879524
:10C840008093B800089594EA9093BC0040EA56E8BB
:10C8500061E070E09091BC0097FD07C04150510924
:10C8600061097109B9F781E008959091B900987F45
:10C87000983011F09031B9F78093BB0084E8809331
:10C88000BC0080EA96E8A1E0B0E02091BC0027FD62
:10C8900005C00197A109B109C1F7E5CF8091B900A1
:10C8A000887F883111F08034F1F680E0089524EA21
:10C8B00034E844E92093BC009091BC0097FFFCCF82
:10C8C0009091B900987F983011F0903199F780934A
:10C8D000BB003093BC009091BC0097FFFCCF9091BF
:10C8E000B900987F903211F0983539F44093BC002C
:10C8F0009091BC0094FDFCCFDDCF08950C9423648F
:10C9000084E98093BC008091BC0084FDFCCF089535
:10C910008093BB0084E88093BC008091BC0087FFBB
:10C92000FCCF9091B900987F81E0983209F480E0C3
:10C93000089584EC8093BC008091BC0087FFFCCFFD
:10C940008091BB00089584E88093BC008091BC0076
:10C9500087FFFCCF8091BB000895CF93DF93FC014C
:10C960007096EC01A991CE01A0933F01EC17FD0751
:10C97000C1F780913C018F7D80933C0180913C0107
:10C98000877F80933C01DB015096FB01819180936E
:10C990003E01EA17FB07D1F780913C018068809344
:10C9A0003C0180913D0180FFFCCF405151098091B5
:10C9B0003C01806280933C0180913C01877F8093A1
:10C9C0003C01141615069CF4FB01819180933E01F5
:10C9D000AE17BF07D1F780913C01806880933C017E
:10C9E00080913D0180FFFCCF40515109EACFF90110
:10C9F000C901409620913E0121938E179F07D1F7E0
:10CA000081E090E0DF91CF9108950F931F93CF9332
:10CA1000DF93EC018CE70E9457648CE70E948864E6
:10CA20008E01005F1F4F89910E948864C017D10753
:10CA3000D1F7DF91CF911F910F910C9480648130D9
:10CA400019F440E050E002C040EC50E060E070E0DB
:10CA50008CE790E00C943E16813019F44EE050E0E3
:10CA600002C048E050E060E070E08CE790E00C9499
:10CA70003E1641E050E060E070E08CE790E00E94FC
:10CA80003E1664ED74E180E090E00C94006448E3AD
:10CA900050E060E070E08CE790E00E943E1649E3D1
:10CAA00050E060E070E08CE790E00E943E1644E1C8
:10CAB00050E060E070E08CE790E00E943E1648E7AE
:10CAC00050E060E070E08CE790E00E943E164EE59A
:10CAD00050E060E070E08CE790E00E943E164DE68A
:10CAE00050E060E070E08CE790E00E943E1668E362
:10CAF00074E38CE090E00E9400644CE050E060E061
:10CB000070E08CE790E00E943E1641E050E060E06B
:10CB100070E08CE790E00E943E1646E050E060E056
:10CB200070E08CE790E00E943E1664ED74E180E0D6
:10CB300090E00C940064CF93DF93CDB7DEB7A2975B
:10CB40000FB6F894DEBF0FBECDBF81E1EBECF9E08C
:10CB5000DE01529601900D928A95E1F781E1ECEDAC
:10CB6000F9E0DE01119601900D928A95E1F70E949D
:10CB70004765CE0142960E94056582E00E941F65CE
:10CB800064ED74E180E090E00E940064CE010196C3
:10CB90000E94056560E27CE581E590E00E9400640A
:10CBA00080E00E942C6560E27CE581E590E00E94D7
:10CBB00000644EE050E060E070E08CE790E00E949E
:10CBC0003E16A2960FB6F894DEBF0FBECDBFDF9122
:10CBD000CF910895CF92DF92EF92FF920F931F9320
:10CBE000CF93DF9300D0CDB7DEB7042F122F2130C3
:10CBF00031F0223031F0243031F0283031F090E043
:10CC000005C091E003C092E001C093E0E82FF0E09E
:10CC10008160F82E0C3009F4E1C00E3011F49460FC
:10CC2000DDC0003111F49860D9C0023109F0D6C0DE
:10CC3000292F2C60613009F4B6C0623011F42062F3
:10CC400007C0633011F4206403C0643009F4206627
:10CC50002068622F70E023E030E0AE014F5F5F4F4D
:10CC6000CF010E944E1662E174E380E090E00E94E2
:10CC700000648F2D0E9423640E94996489830E941E
:10CC800099648A83023119F40E9499648B830E940B
:10CC9000996487FDF1CF0E94A3640E94806462E1E1
:10CCA00074E380E090E00E9400648F2D0E94236472
:10CCB0000E94996489830E9499648A83023119F4DD
:10CCC0000E94A3648B830E94A3640E948064698194
:10CCD0002A81023139F5862F90E0A0E0B0E04B8147
:10CCE00030E0322F2227DC0199278827820F931FFB
:10CCF000A11DB11D61FF09C0840F911DA11DB11DB2
:10CD0000BC01CD018C6F9F6F06C0BC01CD01640FCB
:10CD1000711D811D911D0E942C9420E83FEF4FEF63
:10CD200057E41FC070E0762F6627620F711D072E33
:10CD3000000C880B990B0E942C940C3029F420E0F5
:10CD400030EE4FEF54E40DC00E3029F420E038EF00
:10CD50004FEF55E406C0003131F420E03EEF4FEFD5
:10CD600056E40E9478932FE632E143E050E40E94BB
:10CD700024966B017C01612F70E080E090E00E94BE
:10CD80002C949B01AC01C701B6010E9478930F90CF
:10CD90000F900F90DF91CF911F910F91FF90EF9027
:10CDA000DF90CF9008959C68692F70E023E030E019
:10CDB000AE014F5F5F4FCF010E944E1662E174E3F8
:10CDC00080E090E00E9400648F2D0E9423640E9406
:10CDD000996489830E9499648A8356CF6130D9F41B
:10CDE0009068692F70E023E030E0AE014F5F5F4F45
:10CDF000CF010E944E1662E174E380E090E00E9451
:10CE000000648F2D0E9423640E94996489830E948C
:10CE100099648A833CCF292F10CF8F929F92AF9233
:10CE2000BF92CF92DF92EF92FF920F931F93E1E8B0
:10CE3000F4E10081118120E030E06B017C0144E0ED
:10CE4000F594E794D794C7944A95D1F7C01AD10ABC
:10CE5000E20AF30ADC01CB0153E0B595A79597955B
:10CE600087955A95D1F7000F111F221F331F4C01D0
:10CE70005D01801A910AA20AB30AA5019401A28158
:10CE8000B3810E94F2904B015C017BE0B594A794C2
:10CE9000979487947A95D1F7A7019601C701B601B7
:10CEA0000E943C909B01AC01ACE0559547953795AD
:10CEB0002795AA95D1F7A481B5810E94F290DC0153
:10CEC000CB011EE0B595A795979587951A95D1F753
:10CED000A5019401280F391F4A1F5B1F21A332A30C
:10CEE00043A354A3A5E0B0E00E94E790DC01CB018E
:10CEF00080589F4FAF4FBF4F692F7A2F8B2F9927A5
:10CF000087FD9A951F910F91FF90EF90DF90CF9042
:10CF1000BF90AF909F908F900895CF92DF92EF9245
:10CF2000FF921F93CF93DF93CDB7DEB76A970FB60B
:10CF3000F894DEBF0FBECDBF182F21E030E0CE0148
:10CF400001967C01AC0160ED70E08EEE90E00E94F5
:10CF50004E168981803609F0C8C046EB50E060EE7D
:10CF600070E08EEE90E00E943E163CE2C32EDD247F
:10CF7000D39488EE93E00E94C06D91E0C91AD10865
:10CF8000C1F78AE1F70111928A95E9F72AE130E0C9
:10CF9000A70168E870E08EEE90E00E944E1689814D
:10CFA0009A8190938214809381148C8190E0982FC1
:10CFB00088272B81822B90938414809383148E81F5
:10CFC00090E0982F88272D81822B90938614809350
:10CFD00085148F81988590938814809387148A850F
:10CFE00090E0982F88272985822B90938A1480932C
:10CFF00089148C8590E0982F88272B85822B90931D
:10D000008C1480938B148E8590E0982F88272D8523
:10D01000822B90938E1480938D14888990E0982FA2
:10D0200088272F85822B9093901480938F148A8960
:10D0300090E0982F88272989822B909392148093CF
:10D0400091148C8990E0982F88272B89822B9093BC
:10D050009414809393148E8990E0982F88272D89BB
:10D06000822B9093961480939514888D90E0982F3E
:10D0700088272F89822B90939814809397148A8DF8
:10D080008093991428E030E0A70161EE70E08EEE05
:10D0900090E00E944E168A8190E0982F882729817F
:10D0A000822B90939B1480939A148B8180939C1471
:10D0B0008D812C81F0E12F9F90011124982F9F707A
:10D0C000292B30939E1420939D142E812F7030E1D4
:10D0D000839FC0011124822B9093A01480939F14EE
:10D0E0008F818093A1141093A6146A960FB6F894BA
:10D0F000DEBF0FBECDBFDF91CF911F91FF90EF90AC
:10D10000DF90CF9008952F923F924F925F926F924F
:10D110007F928F929F92AF92BF92CF92DF92EF92C7
:10D12000FF920F931F93CF93DF93CDB7DEB7A497F2
:10D130000FB6F894DEBF0FBECDBF9E012F5F3F4FED
:10D14000790198E0D9011D929A95E9F7813009F0AB
:10D1500015C38091A614813009F010C341E050E05E
:10D1600062EF70E08EEE90E00E943E1640E050E0EC
:10D1700065EF70E08EEE90E00E943E1646E250E0D1
:10D1800064EF70E08EEE90E00E943E1600E416E040
:10D1900088EE93E00E94C06D01501109C9F70CE2BE
:10D1A00011E021E030E0AE01475F5F4F63EF70E0D8
:10D1B0008EEE90E00E944E168985897089878823BB
:10D1C00041F088EE93E00E94C06D0150110949F7CB
:10D1D000D5C228E030E0A70167EF70E08EEE90E066
:10D1E0000E944E16F981FAA32A812BA33B813CA30E
:10D1F000CF80D884DC24CD24DC24E12CF12C6C817C
:10D20000862F90E0A0E0B0E0AC01BD01ECE0440F5F
:10D21000551F661F771FEA95D1F78D8190E0A0E03A
:10D22000B0E0F4E0880F991FAA1FBB1FFA95D1F751
:10D23000842B952BA62BB72B2E8122952F70BC010A
:10D24000CD01622B0E940D676093993670939A36D8
:10D2500080939B3690939C368090A2149090A31458
:10D26000A090A414B090A514D501C4019C52A14073
:10D27000B1098A879B87AC87BD87AEE0CC0CDD1CEB
:10D28000EE1CFF1CAA95D1F780919D1490919E14DD
:10D29000092E000CAA0BBB0B14E1880F991FAA1FC3
:10D2A000BB1F1A95D1F7C81AD90AEA0AFB0AA0913E
:10D2B0009F14B091A0142A853B854C855D850E9402
:10D2C000F290C61AD70AE80AF90A90E4D90EE11CCE
:10D2D000F11C0FE0F594E794D794C7940A95D1F721
:10D2E000A0919C14B0E00E94E7902B013C018BE0E0
:10D2F00075946794579447948A95D1F7A0E85A0E8D
:10D30000611C711CA091A1140A2E000CBB0B0E9481
:10D31000F2902AE095958795779567952A95D1F7AC
:10D32000A30192010E943C90DC01CB013AE0B5954B
:10D33000A795979587953A95D1F79C01AD01405EE9
:10D340005F4FA0919A14B0919B140E94F290DC015F
:10D35000CB01905EAF4FBF4FBC01CD014EE0959524
:10D360008795779567954A95D1F7A70196010E9411
:10D370003C906B017C015FE095958795779567956B
:10D380005A95D1F79B01AC010E943C909B01AC01E6
:10D3900067E055954795379527956A95D1F7A09100
:10D3A0009914B0E00E94E790DC01CB0174E0B595E0
:10D3B000A795979587957A95D1F7A7019601281B90
:10D3C000390B4A0B5B0BDA01C90157FF03C080E040
:10D3D00090E0DC0181309105A10539E1B30724F02B
:10D3E00080E090E0A0E0B9E12CE0B595A795979595
:10D3F00087952A95D1F780939D3690939E36A0937A
:10D400009F36B093A03675016401FF0CCC08DC2C6C
:10D4100076019401A5016C2D7C2D8C2D9C2D345F03
:10D420004140510961097109810991092A873E87A3
:10D430004F87588B698B7A8B8B8B9C8B59016A0138
:10D440007B018C010E94FA902D8B3E8B4F8B5D8F60
:10D450006E8F7F8F88A399A330918A1420918914AD
:10D46000932F990F990B492F592F692F792F892FB6
:10D470000E94FA900CE00E942A92922E832E742E23
:10D48000652E562E472E382E292E30918C14209141
:10D490008B14932F990F990BAD88BE88CF88DD8CA4
:10D4A000EE8CFF8C08A119A1492F592F692F792FD4
:10D4B000892F0E94FA9008E00E944392A92CB82C70
:10D4C000C72CD62CE52CF42C032D122D0E94619232
:10D4D00070588F4F9F4F20908714309088145101BF
:10D4E000C12CD12CE12CF12C00E010E00E94FA902C
:10D4F00001E20E944392288F398F4A8F5B8F6C8F95
:10D50000272E382E492EA0E00E94889209F42AC1C5
:10D510003091921420919114932F990F990BAD880B
:10D52000BE88CF88DD8CEE8CFF8C08A119A1492F15
:10D53000592F692F792F892F0E94FA902D8B3E8BBE
:10D540004F8B552E3B014C013091901420918F143C
:10D55000932F990F990BAA84BE84CF84D888E98829
:10D56000FA880B891C89492F592F692F792F892F08
:10D570000E94FA9001E10E942A92AD88BE88CF886D
:10D58000D52C730184010E94619259016A017B01CB
:10D59000582E192FBBA14B2F50E060E070E0E4E063
:10D5A000440F551F661F771FEA95D1F78CA182950E
:10D5B0008F70482BEAA18E2F90E0A0E0B0E0FCE055
:10D5C000880F991FAA1FBB1FFA95D1F7482B592B1B
:10D5D0006A2B7B2B80E090E0A0E1B0E0841B950BF0
:10D5E000A60BB70B3C014D01990C6608762C430144
:10D5F0009C01AD01662D762D862D962D0FE10E94A2
:10D600002A9239014A01B62FA72FF82FE92F30911E
:10D610008E1420918D14932F990F990B492F592F08
:10D62000692F792F892F03E20E942A92052D0E94EB
:10D63000619259016A017B018C019301A4016B2F56
:10D640007A2F8F2F9E2F0E947692E5E3AE2EFCE07C
:10D65000BF2EC12CD12CE12CF12C00E010E00E9457
:10D66000FA90A88CB98CCA8CDB8CEC8CF22C032D34
:10D67000142D0E9455912A873E874F87588B698BBE
:10D680007A8B8B8B9C8B0DE00E944392922E832E83
:10D69000742E652E562E472E382E292E3091981432
:10D6A00020919714932F990F990BA92CB82CC72C64
:10D6B000D62CE52CF42C032D122D492F592F692F30
:10D6C000792F892F0E94FA900E94FA9009E10E9416
:10D6D0004392AA84BE84CF84D888E988FA880B89CB
:10D6E0001C890E94619219012A013B014C01309171
:10D6F000961420919514932F990F990B492F592F18
:10D70000692F792F892F0E94FA9003E10E9443929A
:10D7100059016A017B018C019101A201B301C4018D
:10D720000E94619208E00E94439259016A017B01C4
:10D73000E82F192F3091941420919314932F990F5F
:10D74000990B492F592F692F792F892F04E00E94B7
:10D750002A920E2F0E946192722F632F942F852F91
:10D760009B0104C030E020E090E080E03093A136DF
:10D770002093A2369093A3368093A436A4960FB636
:10D78000F894DEBF0FBECDBFDF91CF911F910F91F7
:10D79000FF90EF90DF90CF90BF90AF909F908F90D1
:10D7A0007F906F905F904F903F902F900895CF9310
:10D7B000E6E4F1E0C081908180812081C07C2295E7
:10D7C000269526952370C20F969596959073C90F4E
:10D7D00082958C70C80F1F92CF938DED93E19F932C
:10D7E0008F930E94839B0F900F900F900F908C2F20
:10D7F000CF910895CF93C82F8DEE99E09F938F938B
:10D800000E946F9B0F900F90C0FF04C08AEF99E0B9
:10D810000E94AB9BC1FF04C089E09AE00E94AB9BD1
:10D82000C2FF04C088E19AE00E94AB9BC3FF04C022
:10D8300087E29AE00E94AB9BC4FF05C086E39AE0B2
:10D84000CF910C94AB9BCF9108951F93CF93DF930F
:10D8500046E069E180E00E94A26E80E00E94F76EDF
:10D860000E947C6D81E49AE09F938F9382EC93E118
:10D870009F938F930E94839B8EB30E94FA6B0E94AA
:10D88000F7780E942E7860E070E08BEA92E00E94C8
:10D89000CA780E941277E091850AF091860A19955C
:10D8A0000E94D76B90E00E94286F0E94BB7F82E0AD
:10D8B0008093E7388093E8380E94746D47EE58E310
:10D8C000BC018DEC9BEA0E94F2710E94E66C0E9402
:10D8D000DF710E94786D0E94F2720E94447EE09196
:10D8E000FF0AF091000B1995E091D70AF091D80A40
:10D8F0001995E091BB0AF091BC0A19950E94F47247
:10D90000182FC0910B0BD0910C0BFE0119950F90A5
:10D910000F900F900F90892B49F0FE011995BC01D3
:10D9200080E890E00E945890EB0102C0C0E8D0E08F
:10D930000E94DC711F921F93DF93CF931F928F93EE
:10D940008091FE0A8F938091FD0A8F938091D60A71
:10D950008F938091D50A8F9380E993E19F938F9362
:10D960000E94839B83E893E19F938F930E94839B04
:10D9700082E793E19F938F930E94839B60E070E026
:10D9800087ED92E00E94CA7889EB99E00E942F759A
:10D990008AE693E19F938F930E94839B8DB79EB7F6
:10D9A00042960FB6F8949EBF0FBE8DBFDF91CF9108
:10D9B0001F91089580E880936100109261000E9499
:10D9C000256C0E943E780E941A6FFBCFEF92FF9267
:10D9D0000F931F93CF93DF93CDB7DEB7A0970FB60A
:10D9E000F894DEBF0FBECDBF83E690E00E94349E68
:10D9F000182F282F35EF380F303108F0982F9095D9
:10DA0000291709F463C08CEE93E19F938F930E94D2
:10DA1000839BE1E3F4E18E010F5F1F4FCE01099676
:10DA20000F900F90D801780124912D933196A8176B
:10DA3000B907D1F7F89448E050E06FE770E0C8010B
:10DA40000E943A9EE3E2F4E1CE010F96D8012491C0
:10DA50002D933196A817B907D1F74EE050E061E752
:10DA600070E0C8010E943A9EE9E1F4E1CE010B9614
:10DA70002491D8012D938D013196A817B907C1F7CC
:10DA80004AE050E067E670E0C7010E943A9E6DEC04
:10DA90007BEA81E690E00E94529E60E070E08FE5B4
:10DAA00090E00E94529E60E08EE590E00E94449ECD
:10DAB00060E070E085E690E00E94529E1AE16AE123
:10DAC00075EE83E690E00E94529E7894812FA09696
:10DAD0000FB6F894DEBF0FBECDBFDF91CF911F917F
:10DAE0000F91FF90EF9008958FE590E00C94349E95
:10DAF0008EE590E00C942C9EF8941092B60016BC23
:10DB000089E787BD82E084BD95E095BD95B395BB5F
:10DB100080936E00789408950F931F936091A914D9
:10DB20007091AA148091AB149091AC140091A91437
:10DB30001091AA142091AB143091AC1460177107A6
:10DB40008207930759F71F910F9108950F931F9321
:10DB50006091B9367091BA368091BB369091BC36DF
:10DB60000091B9361091BA362091BB363091BC364F
:10DB7000601771078207930759F71F910F91089556
:10DB8000009731F0880F991F880F991F0197F1F7BF
:10DB900008951F920F920FB60F9211240BB60F9299
:10DBA0002F933F934F935F936F937F938F939F93A5
:10DBB000AF93BF93EF93FF938091A9149091AA1410
:10DBC000A091AB14B091AC140196A11DB11D80932E
:10DBD000A9149093AA14A093AB14B093AC148091A1
:10DBE000A8148F5F8093A81487FF15C01092A81403
:10DBF0008091B9369091BA36A091BB36B091BC36BF
:10DC00000196A11DB11D8093B9369093BA36A093A9
:10DC1000BB36B093BC36809158388823E1F08091B0
:10DC2000A7148F5F8093A71487FF15C01092A714C5
:10DC30008091B1369091B236A091B336B091B4369E
:10DC40000196A11DB11D8093B1369093B236A09379
:10DC5000B336B093B4360E947A76892B11F00E94C5
:10DC60009B75FF91EF91BF91AF919F918F917F91A4
:10DC70006F915F914F913F912F910F900BBE0F903D
:10DC80000FBE0F901F9018951F920F920FB60F9214
:10DC900011240BB60F922F933F934F935F936F9383
:10DCA0007F938F939F93AF93BF93EF93FF93809155
:10DCB000C600E091BF36F091C036309709F0199553
:10DCC000FF91EF91BF91AF919F918F917F916F9154
:10DCD0005F914F913F912F910F900BBE0F900FBE10
:10DCE0000F901F9018951F920F920FB60F9211244C
:10DCF0000BB60F922F933F934F935F936F937F9346
:10DD00008F939F93AF93BF93EF93FF938091CE0038
:10DD1000E091BD36F091BE36309709F01995FF912C
:10DD2000EF91BF91AF919F918F917F916F915F9193
:10DD30004F913F912F910F900BBE0F900FBE0F9000
:10DD40001F90189581110EC01092C5006093C400F9
:10DD500088E98093C1004093C2001092C0361092AF
:10DD6000BF360895813069F41092CD006093CC00E5
:10DD700088E98093C9004093CA001092BE36109281
:10DD8000BD360895811107C08091C00085FFFCCF8A
:10DD90006093C6000895813031F48091C80085FFFA
:10DDA000FCCF6093CE000895CF93C82F8A3031F412
:10DDB0006DE08091AD140E94C26E02C08D3029F0DA
:10DDC0006C2F8091AD140E94C26E80E090E0CF91E4
:10DDD0000895811105C07093C0366093BF360895D1
:10DDE000813021F47093BE366093BD3608958093E0
:10DDF000AD1483E992E09093043B8093033B089534
:10DE000084B7877F84BF0FB6F894A895809160008F
:10DE1000886180936000109260000FBE08959FE0BB
:10DE200088E10FB6F894A895809360000FBE909398
:10DE300060000895A89508950FB6F894A89580916C
:10DE40006000886180936000109260000FBE0895AA
:10DE50000C9442970C943E978091C63690E00895BA
:10DE60008091390181FF09C0809139018D7F8093B4
:10DE7000390189E190E00197F1F723E040E06FE19B
:10DE800082E491E00E944F7485E090E00197F1F701
:10DE900008959091390191FD0AC0282F803108F032
:10DEA0002FE040E06FE085E491E00C944F7408951A
:10DEB0008091390181FD09C040E06FE181E491E08A
:10DEC0000E9444748F7E813019F080E090E00895C4
:10DED00081E090E008958091390181FF02C081E0E6
:10DEE000089540E06FE181E491E00E9444748F3135
:10DEF00021F08F7E8150823090F780E008958091EC
:10DF0000390181FD04C00E946B6F8823C1F308951D
:10DF1000109258388091390181FD8BC00E947F6F2B
:10DF20008091390181FD85C00E94306F8091390157
:10DF3000826080933901809190388823D9F1809153
:10DF40009400909195004091A1385091A238841787
:10DF50009507A0F480916D3890916E38A0916F383C
:10DF6000B0917038875F924CAF4FBF4F80936D3840
:10DF700090936E38A0936F38B093703820919400CE
:10DF800030919500241B350B80916D3890916E383F
:10DF9000A0916F38B0917038820F931FA11DB11DF1
:10DFA00080936D3890936E38A0936F38B09370382B
:10DFB00010929038809192388823D9F18091940002
:10DFC000909195004091A5385091A63884179507F7
:10DFD000A0F48091753890917638A0917738B091FF
:10DFE0007838875F924CAF4FBF4F809375389093CE
:10DFF0007638A0937738B093783820919400309198
:10E000009500241B350B8091753890917638A0913E
:10E010007738B0917838820F931FA11DB11D80937E
:10E02000753890937638A0937738B09378381092FB
:10E030009238089580915838882321F00E946B6FA0
:10E040000E94886F80E090E0089522E0260F27FF6D
:10E050000CC080915638909157380196909357385C
:10E06000809356388FEF9FEF0895AB01BC018EEA85
:10E0700094E10E94B09A80E090E0089540E06FE162
:10E0800081E491E00C944474282F40E06FEF86E522
:10E0900091E00E944F740895CF93DF9398EF980F0B
:10E0A000923038F0982F9F7E963019F0893109F020
:10E0B0004BC09091390191FD4AC0C82F0E947F6FDB
:10E0C0000E943E70D82FC81709F43BC0C83029F40D
:10E0D000809139010E94306F27C0C93119F486310F
:10E0E00081F404C0C63169F4893159F429E040E073
:10E0F0006FE182E491E00E944F7485E090E0019727
:10E10000F1F72C2F40E06FE182E491E00E944F7420
:10E11000D83031F48FEF0E94447081ED92E002C05C
:10E1200085E090E00197F1F70E943E70C81749F032
:10E13000C63019F4813071F404C0C63159F481310C
:10E1400049F480E490E008C082E490E005C084E4F3
:10E1500090E002C083E490E0DF91CF910895809138
:10E160009400909195009093A6388093A53881E013
:10E1700080939238809358389091390191FF1EC056
:10E1800020919400309195003093A2382093A138CB
:10E1900080939038809353382FB7789480913901C9
:10E1A000809139018D7F8093390180E197E2309130
:10E1B0005338332311F00197D1F72FBF86E10E9426
:10E1C0004C700C947F6F80915838811102C00E946E
:10E1D000AF7081E090E008950F931F93CF93DF938A
:10E1E0001F92CDB7DEB780915838882361F08091B7
:10E1F000390181FF02C080E07BC00E946B6F8823E1
:10E20000D1F300E003C00E94E37001E0809194002C
:10E21000909195009093A03880939F3811E01093CF
:10E220008F3880E88093550186E00E944C701093EF
:10E23000C7368FB789837894109247018091C7368B
:10E240008111FCCF89818FBF8091470111E08E3011
:10E2500008F010E0119586E10E944C701092550173
:10E2600080918F388823D9F1809194009091950006
:10E2700040919F385091A03884179507A0F4809161
:10E28000693890916A38A0916B38B0916C38875F8B
:10E29000924CAF4FBF4F8093693890936A38A093E8
:10E2A0006B38B0936C382091940030919500241B0A
:10E2B000350B8091693890916A38A0916B38B09194
:10E2C0006C38820F931FA11DB11D80936938909304
:10E2D0006A38A0936B38B0936C3810928F38011164
:10E2E0000E941A70812F8295869586958370817021
:10E2F00090E00F90DF91CF911F910F9108958FEFD4
:10E3000080934E0121E044E060EF8CE691E00E94B2
:10E310004F7425E041E06EE08CE691E00E944F747E
:10E3200080E880936F018091460180936D0121E028
:10E3300045E060E284E491E00C944F74CF93DF9366
:10E34000C9EFD7E0CE010197F1F70E944374109214
:10E35000CD3610924F371092D1371092CC361092A2
:10E36000CB36E9E3F1E080818E7F808380818D7FF1
:10E37000808381EC93E00197F1F780818160808355
:10E3800023E040E06FE182E491E00E944F74219726
:10E39000F1F780915D0180915E010E947F7160E0E4
:10E3A00070E081EA92E00E94CA780E94AF7081E03A
:10E3B00090E0DF91CF91089580912F150895CF932C
:10E3C000C82F0E947F6FC0932F152C2F40E06FE164
:10E3D00088E491E0CF910C944F740E94DF7186E045
:10E3E0000C944C70EF92FF920F931F93CF93DF9397
:10E3F0007C018B01EA011F936F93FF928F938BE552
:10E400009AE09F938F930E946F9BE0926201F0923B
:10E41000630100936001109361010F900F900F90C2
:10E420000F900F900F902097C1F0888180936B011F
:10E43000898180936A018A81809369018B818093AD
:10E4400068018C81809367018D81809366018E8144
:10E45000809365018F8180936401DF91CF911F913B
:10E460000F91FF90EF90089581EA92E00E94EB787F
:10E4700081E08093C6368091C8369091C936019666
:10E480009093C9368093C83681E090E008950F9349
:10E490001F93CF932091CC36C2E8C29F90011124E4
:10E4A000F901E353F94C4081442309F44FC047FD7F
:10E4B00009C0433038F050E08A010250110960175A
:10E4C000710710F4108242C0B9016253794C0E9466
:10E4D000B09A8091CC36C89FF0011124E353F94CD7
:10E4E000DF01A058BF4F9C919093C13610828F5F7F
:10E4F000833018F48093CC3602C01092CC36E09171
:10E50000CC3682E8E89FF0011124E353F94C808176
:10E51000882319F00E94347202C01092C6366091AE
:10E5200047016093C2368091C536882311F0681781
:10E5300010F46093C53670E084E00E94977F60918C
:10E54000C13670E083E00E94977F02C000E010E0D7
:10E55000C801CF911F910F9108950F931F93CF93EF
:10E56000DF931F92CDB7DEB78C01FC0180819181D2
:10E57000009709F18334954029F0F8011182108247
:10E5800083E02AC06238E1F40E944F7F8FB789830D
:10E59000F8940E94B97E60E870E00E944772298179
:10E5A0002FBF1816190674F40E94B47EE091050B73
:10E5B000F091060B199583E495E0F801918380832F
:10E5C00081E00AC08091C3369091C4360196909341
:10E5D000C4368093C336EFCF0F90DF91CF911F9158
:10E5E0000F9108950C94496F8091390181FD06C007
:10E5F00040E06FE085E491E00C94447480E108957C
:10E60000EF92FF921F93CF93DF931F92CDB7DEB7A8
:10E61000182F8091390181FD07C00E947F6F809182
:10E62000583881111CC05AC0809194009091950077
:10E630009093A2388093A13881E0809390388093A2
:10E640005338809139018D7F8093390180E197E2C1
:10E6500020915338222309F30197D1F7DECF80911F
:10E6600092388823D9F1809194009091950040913F
:10E67000A5385091A63884179507A0F48091753875
:10E6800090917638A0917738B0917838875F924C26
:10E69000AF4FBF4F8093753890937638A0937738FB
:10E6A000B09378382091940030919500241B350B5D
:10E6B0008091753890917638A0917738B0917838FC
:10E6C000820F931FA11DB11D8093753890937638EA
:10E6D000A0937738B09378381092923889E10E94ED
:10E6E0004C7086E00E94A27F892B51F00E94F47248
:10E6F000E82E86E00E94A27F81500E94496F02C0EE
:10E70000E12CF12C80919400909195009093A43885
:10E710008093A33881E0809391388FB78983F894F0
:10E7200080913901826080933901809139018D7F18
:10E730008093390162E0610F8EEA94E10E94957442
:10E7400089818FBF8091543890915538019690936C
:10E750005538809354380E947F6F45E060EE82E424
:10E7600091E00E944474182F86E00E94A27F892BBA
:10E7700019F08E2D0E94496F809191388823D9F12C
:10E7800080919400909195004091A3385091A438C5
:10E7900084179507A0F48091713890917238A091F8
:10E7A0007338B0917438875F924CAF4FBF4F8093EE
:10E7B000713890937238A0937338B0937438209165
:10E7C000940030919500241B350B80917138909105
:10E7D0007238A0917338B0917438820F931FA11DC5
:10E7E000B11D8093713890937238A0937338B093B1
:10E7F00074381092913880915838882371F0809144
:10E800009400909195009093A6388093A53881E06C
:10E81000809392380E94AF7002C00E94886F1230BD
:10E8200028F48CE00E94A27F10E00BC0133031F07E
:10E83000153031F0173029F411E003C012E001C0A7
:10E8400013E0812F90E00F90DF91CF911F91FF9007
:10E85000EF900895CF93DF93EB010E94257000970E
:10E8600029F4CE010E940073009751F02091563890
:10E87000309157382F5F3F4F309357382093563899
:10E88000DF91CF9108950895FC0180816823862F40
:10E8900090E002C0959587954A95E2F70895CF9349
:10E8A000DF931F92CDB7DEB7FC01922F8FB789831C
:10E8B000F8942081562F50955223292F01C0220F02
:10E8C0004A95EAF72623252B208389818FBF0F9055
:10E8D000DF91CF910895CF93DF93E0917B012DEFEE
:10E8E0002E0F2D3740F0FC011082E058FF4F1082B0
:10E8F0003196108217C0DC01ED932E2FC0E8D1E0D5
:10E9000038813D93215021962111FACFE150F0E05A
:10E91000E058FE4F2181FC01E058FF4F20833196E3
:10E9200021E02083DF91CF910895609380016250B0
:10E93000E1E8F1E0DC012D91CD01208361503196B9
:10E940006111F8CF08951F920F920FB60F92112404
:10E950000BB60F922F933F934F935F936F937F93D9
:10E960008F939F93AF93BF93EF93FF938091470152
:10E970008093C2368091CB3622E8829FC001112459
:10E980008353994C0E946B748091CB368F5F833098
:10E9900018F48093CB3602C01092CB360E943472AA
:10E9A000FF91EF91BF91AF919F918F917F916F9167
:10E9B0005F914F913F912F910F900BBE0F900FBE23
:10E9C0000F901F9018951F920F920FB60F9211245F
:10E9D000109253380F900FBE0F901F9018951F92F2
:10E9E0000F920FB60F9211241092CA360F900FBEDD
:10E9F0000F901F9018951F920F920FB60F9211242F
:10EA00000F900FBE0F901F9018951F920F920FB688
:10EA10000F9211240F900FBE0F901F9018951F9208
:10EA20000F920FB60F9211240F900FBE0F901F90F0
:10EA300018951F920F920FB60F9211240F900FBED0
:10EA40000F901F9018951F920F920FB60F921124DE
:10EA50001092C7360F900FBE0F901F901895CF934E
:10EA6000DF93EC0189919991009729F060E070E0C3
:10EA70000E94CA78F7CFDF91CF910895CF92DF92AD
:10EA8000EF92FF920F931F9380913415909135155B
:10EA9000892B49F4109230151092311510923215CD
:10EAA0001092331541C00E948C6D8B019C01E09146
:10EAB0003415F091351540815181628173818481D3
:10EAC0009581A681B781840F951FA61FB71F801B54
:10EAD000910BA20BB30B0084F185E02D3097C1F0B0
:10EAE000C080D180E280F380448155816681778146
:10EAF0004C0D5D1D6E1D7F1D401B510B620B730B7A
:10EB0000481759076A077B0730F7DB01CA01E3CFD3
:10EB1000800F911FA21FB31F809330159093311562
:10EB2000A0933215B09333151F910F91FF90EF9082
:10EB3000DF90CF9008958BEA92E00C94EB78EF92FF
:10EB4000FF920F931F93CF93DF938C01FC01808181
:10EB50009181009799F089359105D9F0F8011182DA
:10EB6000108283E068C0828593854817590709F0B1
:10EB700049C00084F185E02D3097A9F71092351532
:10EB80001092341589E590E0F8019183808381E04B
:10EB900052C0673891F16238A9F7C0913415D0910D
:10EBA0003515E12CF12C209769F3CE010E944679AE
:10EBB000892BF1F0AE0168E88A859B850E949E78DA
:10EBC000892BA1F41B861A8688859985E114F104A6
:10EBD00021F0F7019187808704C0909335158093C9
:10EBE0003415198618860E943E75D7CF0E949B75F2
:10EBF0007E010884D985C02DD6CFE0913415F091DF
:10EC00003515BACFF0933515E0933415A085B1854D
:10EC1000109709F4B7CF1A968D919C911B974817BE
:10EC2000590739F418968D919C911997918780878F
:10EC3000EDCFFD01EBCFDF91CF911F910F91FF90B1
:10EC4000EF900895CF93DF93EC010E949B752A8586
:10EC50003B859091341580913515232B91F0E92F48
:10EC6000F82F309771F0EC17FD0739F48091E21519
:10EC70009091E3159387828710C00084F185E02D81
:10EC8000F0CF2091E2153091E3153B872A879887D2
:10EC90008987D0933515C0933415DF91CF910C94AB
:10ECA0003E75CF93DF93EC010E941879CE01DF917E
:10ECB000CF910C942276CF93DF93EC010E942879B8
:10ECC000CE01DF91CF910C942276CF93DF93EC01AC
:10ECD0000E943A79CE01DF91CF910C94227621E007
:10ECE00030E0FC0182859385892B11F020E030E033
:10ECF000C901089581E090E02091341530913515D7
:10ED0000232B11F480E090E00895CF93DF93EC0182
:10ED1000E0913415F0913515E817F90769F4888505
:10ED2000998590933515809334150DC08085918514
:10ED3000C817D90721F0FC013097C1F706C08885B4
:10ED40009985918780870E943E75198618861B8653
:10ED50001A86DF91CF910895EF92FF920F931F9340
:10ED6000CF93DF938C017A01FC0180819181009720
:10ED700041F08A34910511F1F8011182108283E08B
:10ED80004AC087E395E10E947579EC01209761F014
:10ED90004E815F8168857985CE0102960E94517609
:10EDA0000990D881C02DF2CF81E0809336158AE496
:10EDB00090E0F8019183808381E02DC06838E1F70D
:10EDC00087E395E10E947579EC01209781F3CE01EC
:10EDD0000296E816F906D9F4BE0187E395E10E9490
:10EDE0009579E090E215F090E3158E859F859093DC
:10EDF000E3158093E215E889F989309719F08A893B
:10EE00009B891995F092E315E092E215D0CF099015
:10EE1000D881C02DDACFDF91CF911F910F91FF9054
:10EE2000EF9008951092361587E395E10E9471796D
:10EE300060E070E085EB92E00C94CA78EF92FF926C
:10EE40000F931F93CF93DF93EC01E090E215F090C6
:10EE5000E315FF86EE86398B288B1B8B0A8B8091FE
:10EE60003615882379F085EB92E09093E315809333
:10EE7000E215CE0102960E945176F092E315E092DF
:10EE8000E21504C04E835F8368877987BE0187E3FC
:10EE900095E10E949579BE0187E395E1DF91CF91DD
:10EEA0001F910F91FF90EF900C94B079CF93DF9367
:10EEB000EC0180913615882329F0CE0102960E943C
:10EEC000857604C01B861A861D861C86BE0187E3D4
:10EED00095E1DF91CF910C9495791F93CF93DF93B8
:10EEE000DC011496ED91FC9115973097E1F0162F07
:10EEF000EC019093E3158093E21582E08887CD01C1
:10EF000006961995082E000C990B0297029710F09F
:10EF1000133839F4BE01CE01DF91CF911F910C94CB
:10EF20009D7781E08887DF91CF911F910895FC0143
:10EF3000208520FD0C946D770895CF92DF92EF929B
:10EF4000FF920F931F93CF93DF93E090E215F09021
:10EF5000E3150091E4151091E515F801E817F9079C
:10EF600039F0309709F44BC00190F081E02DF6CFD5
:10EF7000009709F444C06B01EC018885882309F1EE
:10EF800018860115110561F00C171D0729F0AE0157
:10EF900067E8C8010E949777F80100811181F1CFDD
:10EFA000EC81FD81309769F0CC15DD0551F0D093EF
:10EFB000E315C093E21540E050E063E8CE01069609
:10EFC0001995E091E415F091E515CE17DF0741F4AE
:10EFD000888199819093E5158093E4150CC0FC011C
:10EFE000309749F080819181C817D907C1F788818E
:10EFF000998191838083F092E315E092E215DF918D
:10F00000CF911F910F91FF90EF90DF90CF900895D7
:10F010001F93CF93DF9310923E15C091E415D091CA
:10F02000E51511E0209779F08985882341F018874C
:10F03000198640E050E062E8CE010E946D770990A9
:10F04000D881C02DEFCFDF91CF911F91089580918E
:10F05000E11591E0980F9093E11508958AE8809367
:10F06000E1151092DF151092E0151092E51510923F
:10F07000E4151092E3151092E215089580913E1563
:10F0800081110E9408789091E015992309F44EC0EF
:10F09000E091DF152E2F30E085E0E89FF00111248C
:10F0A000E15CFA4E608160933D154181528150933D
:10F0B0003C1540933B150380F481E02D2F5F3F4FBB
:10F0C0002F7133272093DF1591509093E0153097DF
:10F0D00031F58091E4159091E51590933A15809360
:10F0E00039158091391590913A15892BF9F0809155
:10F0F0003E1581110E94087840913B1550913C15B6
:10F1000060913D158091391590913A150E9497773D
:10F11000E0913915F0913A1580819181DECF613807
:10F1200011F481E08087CF010E94977780913E158E
:10F130002091E01590E0820F911D08959C0190911F
:10F14000E0159032A9F0E091DF15E90FEF7185E04D
:10F15000E89FF0011124E15CFA4E60835283418301
:10F16000348323839F5F9093E01580E090E00895BF
:10F1700081E090E00895CF93DF93C091E215D091A4
:10F18000E3150E949777D093E315C093E215DF91C2
:10F19000CF910895AB013091E4152091E515E32F4F
:10F1A000F22FE817F907B1F0309721F00190F081C4
:10F1B000E02DF7CF009771F0FC013083218390930D
:10F1C000E5158093E41521E020871782168261E817
:10F1D0000C94BB780895009749F0FC0120852150DC
:10F1E000223020F421E0218720933E1508950C94CD
:10F1F000AD838091E6159091E7150097C1F01092CC
:10F20000E7151092E615DC0114966D917C91159727
:10F210001296ED91FC9113971995E091E615F091F6
:10F22000E715309721F0808191810C94C783089570
:10F23000CF93DF93EC014C835D836E837F830E94C9
:10F240008C6D688379838A839B83DF91CF91089546
:10F25000FC01408151816281738184819581A68105
:10F26000B781840F951FA61FB71F80839183A28348
:10F27000B3830895CF93DF93EC010E948C6D688374
:10F2800079838A839B83DF91CF910895CF92DF9218
:10F29000EF92FF92CF93DF93EC010E948C6DC880B8
:10F2A000D980EA80FB80DC01CB018C199D09AE0975
:10F2B000BF090196A11DB11D21E030E0CC80DD80A9
:10F2C000EE80FF80C816D906EA06FB0610F020E0A3
:10F2D00030E0C901DF91CF91FF90EF90DF90CF90A8
:10F2E0000895FC01118210820895FC0180819181B2
:10F2F0000895DC01ED91FC91309741F0808191817E
:10F30000009711F0FC01FACFCF01089580E090E062
:10F310000895DC01ED91FC911197309721F0208147
:10F3200031812D933C93CF010895DC01ED91FC9147
:10F330003097A9F0A0E0B0E0208131816E177F07FF
:10F3400041F4109709F4DC012D933C931182108253
:10F350000895DF012115310511F0F901EDCF089570
:10F360000F931F93CF93DF938C01EB010E9495794C
:10F3700019821882C8010E947979009711F4F80166
:10F3800001C0FC01D183C083DF91CF911F910F9108
:10F390000895DC01ED91FC9180E090E0309729F038
:10F3A00001960190F081E02DF9CF0895009721F0AA
:10F3B000FC0180819181089580E090E008952F9272
:10F3C0003F924F925F926F927F928F929F92AF92F5
:10F3D000BF92CF92DF92EF92FF920F931F93CF9342
:10F3E000DF93CDB7DEB768970FB6F894DEBF0FBED8
:10F3F000CDBFE9E5F8E354A445A436A427A490A41E
:10F4000081A472A463A4248D2983858D8A83B68CFC
:10F41000A78C908D9B83218D2C83828D8D83938DE2
:10F420009E8324892F838589888796899987278950
:10F430002A8780898B8791899C8722892D87838958
:10F440008E8794859F872585288B8685898B9785D0
:10F450009A8B20852B8B81858C8B92859D8B238528
:10F460002E8BF480E580D680C78080818F8B918140
:10F47000988F128103810E94A66D2F923F924F9226
:10F480005F926F927F928F929F92AF92BF922A81EA
:10F490002F9329812F932E812F932D812F932C81B0
:10F4A0002F932B812F932A852F9329852F9328859E
:10F4B0002F932F812F932E852F932D852F932C857E
:10F4C0002F932B852F932A892F9329892F9328896E
:10F4D0002F932F852F932E892F932D892F932C894E
:10F4E0002F932B892F93CF92DF92EF92FF920F935E
:10F4F0001F93288D2F932F892F939F938F937F9303
:10F500006F93E7EEF8E381811F928F9380811F92C2
:10F510008F9389E394E19F938F930E94839B0FB60F
:10F52000F894DEBF0FBECDBF68960FB6F894DEBF6D
:10F530000FBECDBFDF91CF911F910F91FF90EF9044
:10F54000DF90CF90BF90AF909F908F907F906F9003
:10F550005F904F903F902F900895CF93DF93EC01F1
:10F560004A815B8160E070E08C819D810E94B99A44
:10F57000288139818A819B81289FA001299F500D74
:10F58000389F500D112460E070E08E819F81DF91E3
:10F59000CF910C94B99AFC018281938120E030E0F4
:10F5A00028173907D1F0A481B581A20FB31F4C9160
:10F5B000411110C081E08C9380819181289FA0012E
:10F5C000299F500D389F500D112486819781840FFB
:10F5D000951F08952F5F3F4FE3CF80E090E008959F
:10F5E000FC01868197814281538120E030E024171D
:10F5F0003507D1F08617970781F4A481B581A20F52
:10F60000B31F8C91181614F481508C9384819581CA
:10F61000FC01E20FF31F80810895A081B1818A0F60
:10F620009B1F2F5F3F4FE3CF8FEF0895FC01268193
:10F63000378162177307A0F0A281B38140815181A5
:10F64000A49FC001A59F900DB49F900D1124280F79
:10F65000391F81E090E06217730720F080E0089581
:10F6600080E090E00895CF92DF92EF92FF920F93A7
:10F670001F93CF93DF937C018B016A0188EE95E1A4
:10F680000E947579EC01892B51F0EC81FD81309756
:10F6900011F0C8011995CE010E94D679F3CFA601C9
:10F6A000B801C701DF91CF911F910F91FF90EF90AB
:10F6B000DF90CF900C94137D0F931F93CF93DF9324
:10F6C0000E945F7D8C0188EE95E10E947579EC01C6
:10F6D000892B49F0EA81FB81309709F01995CE0119
:10F6E0000E94D679F4CF0115110539F0C801DF91D8
:10F6F000CF911F910F910C94077DDF91CF911F91B6
:10F700000F910895CF92DF92EF92FF920F931F9384
:10F710000E94447E0E944F7F0E941F7D0E945D7D5B
:10F72000C12C88E0D82E87E0E82EF12C00E01EE105
:10F7300020E030E040E052E060E070E082E090E005
:10F740000E94B17C1F910F91FF90EF90DF90CF90BE
:10F750000895CF93DF93EC010E94727D009761F0D2
:10F760000E94D27EE091D90AF091DA0ABE0183E3C9
:10F770009BE7199581E090E0DF91CF91089508957E
:10F780000F931F93CF93DF93C9E2D6E1488159814C
:10F790006A817B8100E010E02AEE3BE789E096E198
:10F7A0000E941E770E942A6FBC0180E090E02881B1
:10F7B00039814A815B810E948090AB01BC012FE0BE
:10F7C0003CE785EF95E10E941E77DF91CF911F9175
:10F7D0000F9108958091291690912A16A0912B16C9
:10F7E000B0912C164091251650912616609127163F
:10F7F00070912816880F991FAA1FBB1F4817590719
:10F800006A077B0710F4DB01CA01809329169093E5
:10F810002A16A0932B16B0932C160C94C07BCF9372
:10F82000DF930E944F7F0E94B97EEC0119821882FB
:10F830000E94287D28813981009719F1FC014085BB
:10F840004423F9F0FC0142815381F901EE0FFF1FBF
:10F85000EE0FFF1FEC0FFD1F53834283FC01448119
:10F8600055812F5F3F4FF901EE0FFF1FEE0FFF1F76
:10F87000EC0FFD1F51834083398328830E94D67982
:10F88000D9CFC901880F991F880F991F02960E942E
:10F89000B47E88819981892B31F08AEE95E1DF91E0
:10F8A000CF910C941F7EDF91CF910895AF92BF92BC
:10F8B000CF92DF92EF92FF920F931F93CF93DF933C
:10F8C0001F921F92CDB7DEB75B010E94B97E8C01FB
:10F8D000FC01E080F180FA82E9820E94017F9701B9
:10F8E000220F331F220F331F2E5F3F4F82179307C4
:10F8F00098F0C12CD12CCE14DF0471F0F8014481B2
:10F90000558162817381C5010E942C7DFFEFCF1A62
:10F91000DF0A0C5F1F4FEFCF0F900F90DF91CF9159
:10F920001F910F91FF90EF90DF90CF90BF90AF901D
:10F9300008950F93013099F480911D1690911E1631
:10F94000A0911F16B09120168093291690932A1625
:10F95000A0932B16B0932C160F910C94C07B0F9193
:10F9600008954F925F926F927F928F929F92AF9283
:10F97000BF92CF92DF92EF92FF920F931F932A01D3
:10F980003B01480159014FEB5AE0BC018AEE95E179
:10F990000E94027EEAEEF5E143AA54AA65AA76AA7D
:10F9A00087AA90AEA1AEB2AEC3AED4AEE5AEF6AE0F
:10F9B00089E99CE71F910F91FF90EF90DF90CF9026
:10F9C000BF90AF909F908F907F906F905F904F907F
:10F9D0000C94237DEF92FF920F931F93CF93DF93AD
:10F9E0008C01EB017A010E94967DF801F086E78296
:10F9F00063EC7AE0CE01DF91CF911F910F91FF90E0
:10FA0000EF900C94BA7D0C949E7D0C94A97BDC0144
:10FA10001796ED91FC9118970190F081E02D3097A9
:10FA200009F019940895DC011796ED91FC9118974F
:10FA30000280F381E02D309709F01994089581E355
:10FA400096E10C9471799093301680932F16089557
:10FA500081E396E10C947579EF92FF920F931F93D7
:10FA6000CF93DF938C01EB017A0181E396E10E9451
:10FA700075790097D9F0DC0112962D913C9113977E
:10FA80002C173D0781F41696ED91FC91179730974E
:10FA900069F09701AE01B801DF91CF911F910F91ED
:10FAA000FF90EF9019940E94D679E3CFDF91CF9128
:10FAB0001F910F91FF90EF9008950C94927DCF933A
:10FAC000DF93E091150BF091160B1995EC01892B42
:10FAD00029F06A817B8181E00E94977FCE01DF91CE
:10FAE000CF9108950F931F93CF93DF93EC01E09193
:10FAF000170BF091180B19958C016A817B8181E0BD
:10FB00000E94977F81E090E0012B11F480E090E06B
:10FB1000DF91CF911F910F910895E091190BF09112
:10FB20001A0B199483E396E10C947179FC017383A9
:10FB30006283BC0183E396E10C94B079BC0183E35A
:10FB400096E10C949579CF93DF93EC0183E396E1F2
:10FB50000E947579009749F0FC01228133812C17AE
:10FB60003D0729F00E94D679F5CF80E090E0DF9143
:10FB7000CF9108950F931F93CF93DF938B010E9432
:10FB8000A37DEC01892B31F01D830C83C8010E94F9
:10FB90008D7D8E83DF91CF911F910F910895DC01B0
:10FBA0001996ED91FC911A970280F381E02D309720
:10FBB00009F0199408950F931F93CF93DF931F9229
:10FBC0001F92CDB7DEB78C0188E10E94B57FBC01E2
:10FBD000CE0101960E94CF7FD8011996ED91FC913C
:10FBE0001A970190F081E02D309729F0BE016F5FE8
:10FBF0007F4FC80119950F900F90DF91CF911F9102
:10FC00000F910895EF92FF920F931F93CF93DF937D
:10FC10008C01EB017A0145EC5AE00E94EA7CF80184
:10FC2000F286E18669EC7AE0CE01DF91CF911F91F7
:10FC30000F91FF90EF900C94BA7D0C94037DCF93BD
:10FC4000DF93EC0167EE78E388E10E94AB7FCE01A1
:10FC5000DF91CF910C94057DE091010BF091020BA7
:10FC60001994E091BD0AF091BE0A1994E091070B36
:10FC7000F091080B1994E091090BF0910A0B19947B
:10FC800080E090E0089508958FEB92E00E94AD7AB5
:10FC90008FEC92E00E94AD7A87EC92E00C94AD7A02
:10FCA0000F931F93CF93DF93EC01BC018FEC92E095
:10FCB0000E94167B892BA9F00990D881C02DFE01E6
:10FCC00061917191CF010E94627FBE016E547F4F9E
:10FCD000CE018E579F4FDF91CF911F910F910C94C2
:10FCE000867FBE0187EC92E00E94167B892BD1F0C3
:10FCF0000E944F7F688179818A819B810E94627F07
:10FD00008CA990E00E94137F0CA910E00E94C07E95
:10FD1000BE016C5F7F4FA801DF91CF911F910F91C2
:10FD20000C94B09ADF91CF911F910F91089520917B
:10FD3000481D3091491D2817390798F04091461DFC
:10FD40005091471D480F591F5093471D4093461D22
:10FD5000281B390B3093491D2093481D81E090E00A
:10FD6000089580E090E008959093491D8093481D88
:10FD700008958091461D9091471D8D53934E08958F
:10FD80008091451D90E08D56934E089581E090E05E
:10FD90002091911C3091921C235C3C4111F480E035
:10FDA00090E008950E94C67E892B61F06091911CBD
:10FDB0007091921C4091481D5091491D83EC9CE12B
:10FDC0000C94B09A2091461D3091471D21153105A4
:10FDD000B9F08091481D9091491DC096E3ECFCE17B
:10FDE000AF0143595C414817590734F4DF01A20FB2
:10FDF000B31F4C914193F4CF1092471D1092461DB2
:10FE000008958091481D9091491D08958091451D48
:10FE100090E3981B2091481D3091491DA901490F7D
:10FE2000511DCA0108951F93CF93DF931091451D73
:10FE3000212F30E02817390774F0EC010E94067F6B
:10FE40008C0F9D1F8138910530F41C1B1093451DAC
:10FE500081E090E002C080E090E0DF91CF911F91BF
:10FE600008950F931F93CF93DF93E7EBF8E311927D
:10FE7000119288E3E73EF807D1F7CFEAD8E307EB22
:10FE800018E363EE7AE0CE010E94CF7F22960C1732
:10FE90001D07B9F7DF91CF911F910F91089510922F
:10FEA000471D1092461D1092491D1092481D80E377
:10FEB0008093451D83EC9CE19093921C8093911C50
:10FEC0000C94317FEF92FF920F931F93CF93DF93A8
:10FED0008C017B010E944F7FE701C138D10510F0F2
:10FEE000C0E8D0E0AE01B8018091911C9091921CC5
:10FEF0000E94B09AD093491DC093481DCE01DF9156
:10FF0000CF911F910F91FF90EF900895FC0190E326
:10FF1000A7EBB8E301900D929A95E1F788E0FB0119
:10FF2000AFEAB8E301900D928A95E1F70895E82FC2
:10FF3000F0E0EE0FFF1FE954F74C7183608381E01E
:10FF400090E00895E82FF0E0EE0FFF1FE954F74C22
:10FF500080819181089590E0880F991F8158974C76
:10FF60000E94CF7F81E090E0089590E0880F991F74
:10FF70008158974C0895E091850AF091860A199569
:10FF8000E091FF0AF091000B1995E091D70AF091EA
:10FF9000D80A1995E091BB0AF091BC0A1994FB01AB
:10FFA00020813181FC0131832083089542E050E0BB
:10FFB0000E94A39A21E030E0892B11F020E030E08C
:10FFC000C9010895BC0187EE98E30C94CF7F81E6C8
:10FFD0009DE10E946F76892B21F081E69DE10C94D2
:10FFE00065760895E0914D1DF0914E1D309709F012
:10FFF000199480E00895EF92FF920F931F93CF938F
:020000021000EC
:10000000DF938C01EA01FC0180819181009741F02E
:100010008A33934081F1F8011182108283E0F8C0A5
:1000200080E024E0829FF0011124E15BF24E118216
:1000300010828F5F8430A9F780934C1D8091E21568
:100040009091E3159093601D80935F1D0E94277827
:100050008093E93840E450E060E070E081E69DE1A3
:100060000E9451760E948F848AE393E0F801918385
:10007000808381E0CDC06230D9F48091EA389091DC
:10008000EB38892B89F38091FB38863029F48091F5
:10009000133981FD0E94E77F81E00E94D684809120
:1000A000EA389091EB38892BF9F20E945581DCCF28
:1000B000633060F5611114C02097B1F2D093E83934
:1000C000C093E73983E00E94D6848091EA3890910A
:1000D000EB38892B11F00E94F27F0E94E77FC4CF9A
:1000E000613011F6209709F4BFCFD093E439C09363
:1000F000E33985E00E94D6848091EA389091EB380C
:10010000892B09F4B1CF0E94F27FAECF673809F096
:1001100040C010924B1D8FE4E82E8DE1F82E8091A7
:100120004B1D8430C0F4F70182819381C817D90731
:1001300049F4808191810E94BB84F7011182108271
:1001400013821282F4E0EF0EF11C80914B1D8F5F41
:1001500080934B1DE4CFE9EEF9E3848D958DC817AC
:10016000D90719F4158E148E118EB0962AE3E9364C
:10017000F20799F7EFE7FAE381859285C817D90767
:1001800011F4158214823D968BE3E130F807A1F754
:100190006BCF683809F068CFC156DD4109F064CFF4
:1001A00081E69DE10E946F76892B09F45DCF109264
:1001B0004B1DE0914B1DE43008F056CF20E2E29F4A
:1001C000F0011124E751F64C818D8823D9F081E6A6
:1001D0009DE10E94657680914B1DE0E28E9FC001FB
:1001E00011248751964C9093E8398093E73982E047
:1001F0000E94D6848091EA389091EB38892B11F0D7
:100200000E94F27F80914B1D8F5F80934B1DD1CF59
:10021000DF91CF911F910F91FF90EF900895CF93B1
:10022000DF93A091E739B091E839109719F0ED010B
:100230006C9605C0C091E339D091E439299680913C
:10024000E23986FF23C010924A1D80E0EFE4FDE111
:100250008430C1F04081518114962D913C911597C5
:100260004217530761F4228133812115310539F09A
:1002700080934A1D398328831B821A8205C03496D5
:100280008F5FE6CF80934A1D0E94E77F8881998126
:10029000009741F04A815B816091E938DF91CF910D
:1002A0000C94BB78DF91CF9108950F931F93CF9358
:1002B000DF938091FB38863009F07AC08091EA386C
:1002C0009091EB38803F910508F472C08897EC015B
:1002D000D695C7959E01220F331F8E012817390727
:1002E00010F40F5F1F4FCE0188969093EB388093E8
:1002F000EA389093F4388093F538109217391092B9
:1003000016390E948984809590959093173980932F
:1003100016391092FD381092FC380E94788480952E
:1003200090959093FD388093FC380E94F27FC8012D
:1003300088969093EB388093EA389093F4388093C2
:10034000F5388091E5399091E639BC016C0F7D1F3D
:10035000A8010E94B09ABE018AE099E30E94258418
:100360008091EE3880930A398091EF3880930B3971
:100370008091F03880930C398091F13880930D3959
:1003800010921739109216390E94898480959095A1
:1003900090931739809316391092FD381092FC38DB
:1003A0000E947884809590959093FD388093FC38D6
:1003B000DF91CF911F910F910C94F27FE091950AFC
:1003C000F091960A199480E090E00895AF92BF9260
:1003D000CF92DF92EF92FF920F931F93CF93DF9311
:1003E000CDB7DEB7E1970FB6F894DEBF0FBECDBF35
:1003F0007C016B01CE0101965C0181E3F501119254
:100400008A95E9F781E089838CE00E94A27F8C8342
:100410001D821F8280916D1D91E0980F90936D1D3C
:10042000898713E018878DEC9BEA9B878A8789E18F
:100430000E94B57F63EE7AE00E94D67F892B31F06F
:1004400082E08E838FEF8C878D8709C089E10E94BF
:10045000B57FBC01CE010C960E94CF7F1E838DEC30
:100460009BEA9D8B8C8B67EE78E3CE0146960E94CB
:10047000CF7F0E94B97E9FA78EA70E94017F99AB74
:1004800088ABC5010E94608E8C011127C8010E94B3
:10049000137F892B31F10E94C07EA801BC01C501E8
:1004A0000E94838E00918B0A10918C0A0E94067F15
:1004B0005C010E94C07EB501F8011995E114F104B8
:1004C00081F0009739F0019761F441E050E064E079
:1004D00070E004C041E050E060E070E0C601F70168
:1004E0001995E1960FB6F894DEBF0FBECDBFDF9130
:1004F000CF911F910F91FF90EF90DF90CF90BF9021
:10050000AF9008950F931F93CF93DF93411551053B
:1005100079F0FA018B01EC01828193810E94507E77
:10052000B801CE01DF91CF911F910F910C94E6811C
:10053000DF91CF911F910F910895EF92FF920F934A
:100540001F93CF93DF93CDB7DEB7E1970FB6F89443
:10055000DEBF0FBECDBF0E94017F7C010E94B97E2D
:100560008E010F5F1F4FA801B7010E94728F892B68
:1005700009F441C088A999A99701281B390BC90121
:100580000E94977E892BB9F18E8181110CC0BE012A
:100590006A5E7F4F88E10E94AB7FE091DB0AF091B9
:1005A000DC0A199528C02A853B852D3C9BEA390732
:1005B00019F02F3F3F4FF9F4823019F0E8E0F0E0F6
:1005C00002C0E2E0F0E0E00FF11FE017F107F9F2FE
:1005D000319783858F3FC9F3BE01645F7F4F89E107
:1005E0000E94AB7F89E10E94B57F67EE78E30E94AD
:1005F000D67F892B61F6E1960FB6F894DEBF0FBE69
:10060000CDBFDF91CF911F910F91FF90EF90089593
:100610000E942A6F80936D1DE091950AF091960AD1
:100620001994892B29F0E091950AF091960A04C05B
:10063000E091970AF091980A1994FC01680F791FCC
:1006400080E048E1E617F70781F0219198E0382F24
:100650003227532F517030FD84278695513009F48D
:1006600080682695915099F7EDCF08951F920F92CB
:100670000FB60F9211240BB60F922F933F934F9307
:100680005F936F937F938F939F93AF93BF93EF93FA
:10069000FF93809194009091950090939C38809363
:1006A0009B3881E080938D3880917100807D8093AC
:1006B00071000E94F97880918D388823D9F180915A
:1006C00094009091950040919B3850919C388417EC
:1006D0009507A0F48091613890916238A0916338B9
:1006E000B0916438875F924CAF4FBF4F80936138B1
:1006F00090936238A0936338B0936438209194004B
:1007000030919500241B350B8091613890916238AF
:10071000A0916338B0916438820F931FA11DB11D61
:100720008093613890936238A0936338B0936438B3
:1007300010928D38FF91EF91BF91AF919F918F9162
:100740007F916F915F914F913F912F910F900BBED1
:100750000F900FBE0F901F9018959FB7F894E1E788
:10076000F0E08081807D808388B38F6288BB1092A7
:100770009000E1E9F0E01082109292001092950052
:10078000109294008081856080839FBF08959C01B2
:100790009FB7F894309399002093980088B38F62A4
:1007A00088BBE1E7F0E08081826080839FBF08958D
:1007B000FB0141505109460F571FE417F50778F424
:1007C000208130E0322F22276181260F311D820FD8
:1007D000931F8217930708F401963296EECFE41721
:1007E000F50751F4208130E0322F2227820F931F2A
:1007F0008217930708F401960895CF93DF93C09171
:10080000F438D0E0DC2FCC272091F53830E02451AB
:100810003109C20FD31F48E050E06EEF78E39E012C
:10082000280F311DC9010E94D883AE0166E079E32B
:100830000E94D883009721F098278927982702C023
:100840008FEF9FEFDF91CF910895FC012381260F59
:100850002093F138A72FBB2792819A0F9093F038FD
:1008600031813093EF3840814093EE38E92FF0E04A
:10087000EA17FB0748F481E0830F8093EF3881117A
:1008800003C04F5F4093EE3830E0772726173707D5
:1008900088F49F5F9093F03891110CC08091EF38ED
:1008A0008F5F8093EF38811105C08091EE388F5FA4
:1008B0008093EE3808952091E7393091E839BC01F2
:1008C000C90108960E942584E091E739F091E83942
:1008D000AEEEB8E38C91808711968C911197818749
:1008E00012968C911297828713968C918387089524
:1008F00044E150E062EF78E380E090E00E94D8832A
:10090000009721F098278927982708958FEF9FEF68
:10091000089586E00C94FD8381E10C94FD8380E0D2
:10092000E82FF0E0EE0FFF1FE759F54C118210821F
:100930008F5F8430A9F780E090E2899FF001112455
:10094000E751F64C118E8F5F8430B1F780E094E070
:100950009093721D8093711D80E09DE0989FF0013F
:100960001124E158F54C158214828F5F8A30B1F75B
:100970008093701D08959C0190E09430A1F0E92FC0
:10098000F0E081E0890FEE0FFF1FE759F54C408141
:1009900051814217530729F49093701D11821082E0
:1009A0000895982FEACF9093701D0895AF92BF924B
:1009B000CF92DF92EF92FF920F931F93CF93DF932B
:1009C000843009F4DFC1C091E739D091E8392AE1D8
:1009D00039E33093E6392093E5393093ED382093AD
:1009E000EC38833059F4898D8F70833009F06AC0F8
:1009F00088899989892B09F0BFC67EC0823009F0A9
:100A00007FC08091761D8F5F8093761D811113C00A
:100A10008091751D8F5F8093751D81110CC0809131
:100A2000741D8F5F8093741D811105C08091731DAB
:100A30008F5F8093731D1092EB381092EA381092FA
:100A40007E3A10927D3A898D982F9D7F953041F4A2
:100A50008A8D8F5F8A8F843109F08EC6198E8CC67D
:100A6000882309F489C628893989232B09F440C0D1
:100A70009A8D2FEF290F2A8F91117EC69B8D98306A
:100A800031F02FEF280F223048F4953039F4198EC9
:100A900080E88093E2390E940F8128C5953038F4B0
:100AA00023E0092E01C0220F0A94EAF701C020E3D7
:100AB0002A8F9F5F9B8F8F708330A1F048F4813025
:100AC00009F43AC3823009F057C61092133937C37C
:100AD000863009F4A8C4883009F4A5C4843009F02C
:100AE0004BC6A1C484E08093E2390E940F8130C5D7
:100AF0008F70833009F040C688E08093E239EBC400
:100B0000853019F5E091E339F091E43984819581DC
:100B1000892B09F431C61092E8391092E7398EE03A
:100B200099E39093E6398093E5399093ED3880937B
:100B3000EC3810927E3A10927D3A1092EB38109277
:100B4000EA3888E08093E2391BC18091F23885341D
:100B500009F012C60091F43810E0102F00278091A0
:100B6000F538080F111D8091EA389091EB38801705
:100B7000910708F401C61093EB380093EA3880918E
:100B8000F8388F7309F0F8C5F090F938F110F4C512
:100B90008091793A90917A3AC0910D0BD0910E0BD9
:100BA0008C179D0759F440917B3A50917C3A2091E3
:100BB0000F0B3091100B42175307A1F0209102390F
:100BC000309103398217930709F0D6C52091043973
:100BD0003091053980917B3A90917C3A28173907FA
:100BE00009F0CAC50E947884019609F0C5C58091B4
:100BF000FB38863009F429C18131E9F1813009F0EF
:100C0000BBC580910639883009F0B6C51092063907
:100C10008091083990910939873F6FEF960710F05E
:100C2000099601C0089690930939809308398091FC
:100C3000FE389091FF38A0910039B091013980932E
:100C4000023990930339A0930439B0930539809108
:100C5000793A90917A3AA0917B3AB0917C3A80931C
:100C6000FE389093FF38A0930039B093013980E4A7
:100C70008093FA385EC50C5111091093EB3800933C
:100C8000EA388EE099E39093E6398093E5398091D4
:100C90000C3990910D39892B29F00E948C84019692
:100CA00009F06AC5209108393091093921153105BB
:100CB00009F462C58FE79AE39093E4398093E339AE
:100CC000A0900639B0900739E0900F0BF090100B10
:100CD0004091110B5091120BA091FE38B091FF384A
:100CE00000910039109101396091130B7091140B30
:100CF000E091E339F091E4398BE3E130F80708F053
:100D00003BC584819581009721F12817390709F5A2
:100D100086819781009719F08A159B05D1F480810F
:100D20009181C817D90729F4C280D380CE14DF047B
:100D3000B1F08417950729F4C280D380C616D70670
:100D400071F08A179B0729F482819381081719078C
:100D500031F03D96F093E439E093E339C9CF109236
:100D6000E8391092E73982E08093E2398EE099E326
:100D70009093ED388093EC3810927E3A10927D3A41
:100D80000E940F8180917D3A90917E3A009709F4FC
:100D9000F3C49C01245E3F4F3093EB382093EA3834
:100DA0003093F4382093F538E091E339F091E43949
:100DB00020852093FA3821E12093FB380896982764
:100DC0008927982790930B3980930A3910920D390F
:100DD00010920C398481958190930739809306395C
:100DE0008681978190930939809308398091793A67
:100DF00090917A3AA0917B3AB0917C3A8093FE38F8
:100E00009093FF38A0930039B0930139808191818C
:100E1000A281B3818093023990930339A09304395E
:100E2000B09305398AE199E39093E6398093E539E7
:100E30000E948C8480959095009711F48FEF9FEF1E
:100E400090930D3980930C3974C40E948984019663
:100E500009F092C440910839509109394115510562
:100E600009F48AC48091063990910739009709F4F2
:100E700083C46091FE387091FF38E0910039F091A1
:100E80000139C9EED9E3298D2223A9F0AC81BD81B6
:100E90004A175B0781F4AE81BF818A179B0759F41B
:100EA000A881B9816A177B0731F4AA81BB81EA174F
:100EB000FB0709F45CC1A0962AE3C936D20719F7EB
:100EC000809113398F738230D9F450936F1D409302
:100ED0006E1D80E0843091F0E82FF0E0EE0FFF1FF0
:100EE000E759F54C208131818F5F4217530791F705
:100EF0001092701D80E0C0E0D0E07CC08093701D37
:100F00008091133982FD38C484E18093133988E2DB
:100F100090E09093EB388093EA3880E58093123923
:100F200030910D398091113980930D3920910C3910
:100F30008091103980930C392093103990910B399E
:100F400080910F3980930B3990930F3980910A3932
:100F50008093701D40910E3940930A3980930E3969
:100F60003F5F3093113931110DC02F5F209310393D
:100F7000211108C09F5F90930F39911103C08F5FBB
:100F800080930E39809106399091073990936F1DA7
:100F900080936E1D209108393091093930930739BB
:100FA0002093063990930939809308398091FE384F
:100FB0009091FF38A0910039B091013980930239A6
:100FC00090930339A0930439B09305398091793A0D
:100FD00090917A3AA0917B3AB0917C3A8093FE3816
:100FE0009093FF38A0930039B093013987C39730AD
:100FF00089F08F5F8430C1F060E2869F90011124F8
:10100000F901E751F64C918D9111F1CF8093701D4C
:10101000EF010FC0209721F0428D9A8D941748F769
:10102000E901C751D64CE5CF8093701D209709F494
:10103000A3C3D093E839C093E73983E08A8F888FC0
:101040001E8A84E08F8B1B8E80910839909109391C
:101050009D838C8380910639909107399F838E837D
:101060008091FE389091FF38A0910039B0910139FC
:1010700088839983AA83BB8381E0898F8091731DC4
:101080008C878091741D8D878091751D8E878091CE
:10109000761D8F8781E090E0998B888B80910D3948
:1010A0008B8780910C398A8780910B398987809151
:1010B0000A39888781E090E00E945B848091123930
:1010C000982F907F9135C0F182958F7090E00597B1
:1010D000880F991F880F991FEF2DF0E0E817F90787
:1010E0004CF5EE50F74C20A5222321F1213011F4CC
:1010F000F394F2CF2230C9F421A52430B1F4F09258
:10110000701D82A590E0982F882723A5822B9093AD
:101110006F1D80936E1D893C910510F088EC90E066
:101120009B8B8A8B9D8B8C8B07C021A5222311F072
:10113000F20ED2CFF092701D80E18093133980912E
:10114000133982608093133982E080931A3984E0E6
:1011500080931B3910921C3988EC80931D398CE2E6
:1011600090E09093EB388093EA3880E675C2D09394
:10117000E839C093E7391092E23980911339782F1A
:101180007470F72E82FF03C0198E80E20EC2909118
:10119000123992959F70990F990F9093701D091BAA
:1011A0001109045111091093EB380093EA38922F7A
:1011B0009F70923029F4982F9F73923139F41FC099
:1011C000913021F4982F9F739230C9F0012B19F4BC
:1011D000982F9370A1F020910A399885291332C273
:1011E00020910B39998529132DC220910C399A85AC
:1011F000291328C220910D399B85291323C284FF0E
:1012000049C0688979896115710509F443C0CE0127
:101210000C960E94258430910E398091EE38381357
:1012200039C020910F398091EF38281333C0909145
:1012300010398091F03898132DC080911139409168
:10124000F138841327C03C872D879E878F878B8D2D
:10125000811119C09E89888D2A8D821B292F269580
:1012600026952695821B980F9E8B87FD81952F8949
:10127000322F36953695231B820F8F8B9695969538
:101280009695890F888F81E08093E239888D8A8FC7
:10129000198A188A298DE22FEF708E2F90E0FC01B9
:1012A0003197E830F10508F067C28827E656FF4F0E
:1012B0008F4F0C94C1908091E23980FF14C083E07D
:1012C000898F80E48093E239198A188A8091EA38FC
:1012D0009091EB38009709F4FAC022E42093E239A8
:1012E0000E945B84F4C0809113398F73823009F0BF
:1012F00043C222CF8091E23980FF60C080911339D0
:101300008F73823109F05AC080911239982F907FE3
:101310009135C0F182958F7090E00597880F991FE5
:10132000880F991FEF2DF0E0E817F9074CF5EE5004
:10133000F74C20A5222321F1213011F4F394F2CFB0
:101340002230C9F421A52430B1F4F092701D82A599
:1013500090E0982F882723A5822B90936F1D809370
:101360006E1D893C910510F088EC90E09B8B8A8B78
:101370009D8B8C8B07C021A5222311F0F20ED2CFBA
:10138000F092701D83E0898F80910A39888780915F
:101390000B39898780910C398A8780910D398B8729
:1013A00081E090E00E945B8482E48093E239198AB4
:1013B000188A1092EB381092EA3889C080E2809344
:1013C000E2390E940F81E091E739F091E839118EFE
:1013D00097CD8091133980FF28C024FD26C08889CD
:1013E0009989892B09F0C8C18091EA389091EB382E
:1013F00001960E945B848091E239982F90619093CE
:10140000E2392091EA383091EB38232B19F08261D0
:101410008093E2390E940F8181E090E0998B888B64
:1014200088E0898F1B8E81E10EC185FF1CC08091F1
:101430001839909119399827892798274091E539CB
:101440005091E639480F591F5093E6394093E539DA
:101450004091EA385091EB38BA01681B790B7093D0
:10146000EB386093EA384091EA385091EB384115F7
:10147000510551F024FD08C09091E239926090939B
:10148000E239CA010E945B848091143990E0982F60
:10149000882720911539820F911D90936F1D80939D
:1014A0006E1D2C893D892817390710F0892B21F4EE
:1014B00030936F1D20936E1D80916E1D90916F1D56
:1014C0009B8B8A8B8091E239837009F455C110920D
:1014D0007E3A10927D3A0E940F818091E23985FF19
:1014E00007C010927E3A10927D3A198E84E1ABC00B
:1014F00084FF0AC010927E3A10927D3A81E090E01B
:10150000998B888B84E08DCF20917D3A30917E3A03
:1015100021153105E1F080FF02C0198A188A8889F7
:101520009989009781F48A899B898217930720F40F
:1015300090937E3A80937D3A80917D3A90917E3A65
:10154000998B888B04C090937E3A80937D3A1B8E52
:101550008091EC389091ED389093E6398093E5399D
:1015600080917D3A90917E3A892B59F088899989AA
:10157000009739F088969093EB388093EA3888E1A9
:101580000BC08091E23981FFF7C088E290E0909330
:10159000EB388093EA3880E1809313395CC0809106
:1015A000E23980FFE9C0198E80E18093E2390E9420
:1015B0000F81E2C08091EA389091EB38009711F0EA
:1015C0000E945B84909113398091E23990FF0BC0A7
:1015D00080FF06C087E0898F1A8E198A188A19C081
:1015E00086E0898F16C080FF1EC085E0898F198A2A
:1015F000188AC2C08091EA389091EB38009711F0B8
:101600000E945B848091133980FF0DC087E0898F31
:101610001A8E81E090E00E945B8480E18093E23941
:101620000E940F810FC08091EA389091EB38892B8E
:1016300049F4A2C08091E23980FF9EC087E0898F83
:101640001A8E9AC080E18093133988E290E09093DB
:10165000EB388093EA3880E580931239888580934F
:101660000E39898580930F398A85809310398B854F
:10167000809311398C8580930A398D8580930B393D
:101680008E8580930C398F8580930D3986E0809309
:10169000FB388C819D8190930739809306398E8128
:1016A0009F8190930939809308398091793A90917C
:1016B0007A3AA0917B3AB0917C3A8093FE3890932D
:1016C000FF38A0930039B093013988819981AA81AC
:1016D000BB818093023990930339A0930439B0936E
:1016E0000539898D84FF05C010921539109214397F
:1016F00005C01092143988EC8093153980E48093EA
:10170000FA388091EA389091EB389093F4388093CE
:10171000F538109219391092183910921739109221
:1017200016390E94898480959095909317398093FB
:10173000163985E48093F2381092F3381092F93814
:101740001092F8388091771D9091781D01969093B2
:10175000781D8093771D9093F6388093F738109218
:10176000FD381092FC380E94788480959095909373
:10177000FD388093FC3804C01092EB381092EA38A0
:101780001092E239DF91CF911F910F91FF90EF906E
:10179000DF90CF90BF90AF900895FC0180E090E083
:1017A0002081222329F02181820F911D3296F8CFCA
:1017B0000895EF92FF920F931F93CF93DF937A01D7
:1017C0002830310514F5DB014D915C9154274527F4
:1017D000542702C0440F551FEA94E2F7452F5527BE
:1017E000F901E55EF44FC081D0E04C235D2368E051
:1017F00070E0EB01C21BD30BFA0102C0F695E7952E
:10180000CA95E2F7DC01EC9376C0D90153E0B595B7
:10181000A7955A95E1F7E114F10431F0AB01FC0111
:101820008C010A0F1B1F2FC0FB01AC017B01EA0ECC
:10183000FB1EEE16FF0629F06191EA016993AE01E5
:10184000F8CF8901077011270115110509F453C05C
:10185000FC01EA0FFB1FD7012C9130E0D801A55EF7
:10186000B44F9C91492F50E042235323C8E0D0E06D
:101870009E01201B310BEA0102C0D695C7952A951F
:10188000E2F7C08338C0E017F10781F0EA018881F0
:1018900099819827892798270E2C02C0880F991FB5
:1018A0000A94E2F791934F5F5F4FEDCF2770332794
:1018B0002115310501F1A60FB71F8D919C91982735
:1018C0008927982702C0880F991FEA94E2F7892F89
:1018D0009927D901A55EB44F4C9150E084239523FC
:1018E00048E050E0BA01621B730B02C096958795E1
:1018F0006A95E2F78083DF91CF911F910F91FF905E
:10190000EF9008958F929F92AF92BF92CF92DF9205
:10191000EF92FF920F931F93CF93DF931F921F922B
:10192000CDB7DEB70E94B97E8C0182E090E00E94C4
:10193000977E892B19F480E090E05DC0F8018181E9
:1019400090E0982F88272081820F911D0E94A37D0F
:101950007C01892B81F30E94B97E4C01F7019681AD
:10196000892F877021E030E011F420E030E0969577
:1019700096959695A901490F511DCA010E94977E1F
:10198000892BC9F2F70104811581A12CB12CF80132
:101990008081882379F1F801C180D12CA50147709D
:1019A0005527B50193E0759567959A95E1F7680D10
:1019B000791D883168F09601CE0101960E94D98B7D
:1019C000BE016F5F7F4FF80180810E94AB7F0DC029
:1019D0001A8219829601CE0101960E94D98B6981E3
:1019E0007A81F80180810E94977FAC0CBD1C0E5F4C
:1019F0001F4FCDCFC7010F900F90DF91CF911F9157
:101A00000F91FF90EF90DF90CF90BF90AF909F909D
:101A10008F900895DF92EF92FF920F931F93CF93D1
:101A2000DF93FC012830310544F4DA018C9190E019
:101A300040E150E0461B570B6BC0C901A3E09595F0
:101A40008795AA95E1F76115710549F08A017F0133
:101A5000E80EF91EC8E0D0E0C61BD70B2EC0DA0195
:101A6000EF01480F591FA417B50719F06D9169933D
:101A7000FACFA901477055274115510509F456C001
:101A8000E80FF91F2C9130E088E090E0841B950B63
:101A900002C0359527958A95E2F780E190E0841B96
:101AA000950B02C0220F331F8A95E2F78081832BAA
:101AB00080838181282B218339C0EE15FF0591F0A9
:101AC000D801DD908D01AD2DB0E00C2E02C0AA0F23
:101AD000BB1F0A94E2F7D080BD29B193B081AB2B34
:101AE000A083EBCF2770332721153105F9F0DA01F8
:101AF000A80FB91F8C9190E0621B730B685F7F4F3A
:101B000002C0959587956A95E2F7992740E150E0E4
:101B1000BA01621B730B02C0880F991F6A95E2F726
:101B20002081922B90839181892B8183DF91CF91AA
:101B30001F910F91FF90EF90DF9008956F927F9229
:101B40008F929F92AF92BF92CF92DF92EF92FF92CD
:101B50000F931F93CF93DF931F921F92CDB7DEB7E2
:101B60007C01FC018681982F977001E010E011F450
:101B700000E010E0869586958695080F111DC80136
:101B800002960E94137F009709F446C00E94C07E0F
:101B9000F7012281FC012083F7012381FC012183CD
:101BA0000E94C07E02964C01A80160E070E00E9495
:101BB000B99AF701C480D580A12CB12CF60180819F
:101BC000882341F1F601E180F12C3501F7E06F2225
:101BD0007724850193E0159507959A95E1F7080D0F
:101BE000191D883128F00E94B57F9701AC0108C00B
:101BF0000E94A27F9A8389839701AE014F5F5F4F56
:101C0000B301C8010E940A8DAE0CBF1C82E0C80E51
